:020000040800F2
:1000000000000120D9740008EF330008F133000824
:10001000F3330008F5330008F73300080000000050
:10002000000000000000000000000000F93300089C
:10003000FB33000800000000FD330008FF33000818
:100040002975000829750008013400082975000881
:1000500029750008297500080D3400081D340008B2
:10006000297500082D34000829750008353400086A
:10007000413400084D34000829750008297500082E
:10008000593400085D3400082975000829750008F6
:10009000000000002975000869340008297500086F
:1000A00029750008297500082975000829750008B8
:1000B00029750008297500082975000829750008A8
:1000C00029750008297500086D3400082975000895
:1000D0002975000879340008297500082975000879
:1000E000297500082975000885340008297500085D
:1000F00029750008000000000000000029750008B4
:100100002975000829750008913400082975000830
:100110002975000829750008297500082975000847
:100120002975000829750008297500082975000837
:0801300029750008297500087B
:1001400010B5054C237833B9044B13B10448AFF311
:1001500000800123237010BDC807002000000000AC
:10016000D419030808B5034B1BB103490348AFF387
:10017000008008BD00000000CC070020D41903084F
:1001800014214160704714207047406A7047000096
:1001900081010008870100088B010008A101000807
:1001A00010B5044604F1100000F05CFCC4F8F8003F
:1001B0000148C4F87C0110BD90010008F8B5E6B014
:1001C00004460D4616461F460A4906A800F0CAFE18
:1001D00070996F9A05910492009733466E996D9AC3
:1001E000039102922A466C990191214600F060F831
:1001F00067B0F0BD9C010008F8B5E6B004460D46B6
:1002000016461F46094906A800F0ACFE6F996E9A83
:100210000491039200976D996C9A02910192334672
:100220002A46214600F087F867B0F0BD9C0100081F
:1002300038B500281CBF01680029184A23D1184B83
:100240001C684FF6F0710C404CF24025AC421FBFC9
:100250001B6819404CF27024A14212D1114D29683B
:1002600079B911490B68C3F30B03B3F58A6F1FBF4C
:100270000968C1F30B0140F28343994204BF012195
:10028000117028B905E0094B994204BF0121117092
:100290004068BDE8324002F073BC00BFE4070020B4
:1002A00000ED00E0002004E00010005C0000374892
:1002B0002DE9F04104460D46216816464A681F465E
:1002C00090478046B8F5403F2ED122680A9993683E
:1002D000204698478046B8F5403F25D12368089AC4
:1002E0000799D3F80CC02046E0478046B8F5403F58
:1002F0001AD12368069A39461F692046B8478046B6
:10030000B8F5403F10D1236829465D693246204642
:10031000A8478046B8F5403F06D123680B9A099953
:100320009D692046A847804621680A682046904774
:100330004046BDE8F0812DE9F04104460D462168B4
:1003400016464A681F4690478046B8F5403F2ED172
:1003500022680A999368204698478046B8F5403F3E
:1003600025D12368089A0799D3F80CC02046E047A6
:100370008046B8F5403F1AD12368069A39461F696E
:100380002046B8478046B8F5403F10D1236829463B
:100390005D6932462046A8478046B8F5403F06D101
:1003A00023680999DD6900222046A8478046216814
:1003B0000A68204690474046BDE8F0814FF440303F
:1003C00070470000F0B50C4685B0114600281A466B
:1003D0001CBF0568002D0B4B11D082B104B971B957
:1003E0000D9860B10F9E0E9F0A9B02900496039792
:1003F0000B980C9E009001962046A847034618468D
:1004000005B0F0BD020003002DE9F04F0646D0B064
:100410000868F56DD6F860E0726EB76EF36E00BADC
:1004200000906C46486800BA60600DF1400888682A
:1004300000BAA060C86800BAE060086900BA20612C
:10044000486900BA6061886900BAA061C86900BAE9
:10045000E061086A00BA2062486A00BA6062886A8D
:1004600000BAA062C86A00BAE062086B00BA2063F2
:10047000486B00BA6063886B00BAA063C86B00BAAF
:10048000E063402058F80C1C58F820CC58F838ACE1
:100490008CEA010158F840CC8AEA01018CEA010992
:1004A0004FEAF979401E48F8049BEBD187EA020035
:1004B00000EA0E00784010EBF5610098DFF824C4E4
:1004C00041186144C81882EABE032B404FEAF0612C
:1004D00053405918636859186144CF194FEAB5035E
:1004E00083EABE01014081EABE0111EBF765A16814
:1004F0004D196544A91883EAB0023A404FEAF16504
:100500005A405519E26855194FEAB70282EAB00716
:1005100065440F4005EBBE0E97EAB00717EBFE658A
:1005200027697D194FEAB10782EA0701654401EAAC
:100530000E01EB18514011EBF36561694D194FEA5B
:10054000BE0187EA010E65440EEA030E15EBB0000A
:100550008EEA070E0EEBF065D4F818E0754465449A
:10056000AA1881EAB30505404FEAF26E4D40AE4449
:10057000E569AE44E64477444FEAB00080EAB30E42
:100580000EEA020E8EEAB30E0EEBF765D4F820E009
:1005900075446544691880EAB2053D404FEAF16E42
:1005A0004540AE44656AAE44E6440EEBB3034FEA01
:1005B000B70787EAB20E0EEA010E8EEAB20E0EEB14
:1005C000F365D4F828E075446544281887EAB10536
:1005D0001D404FEAF06E7D40AE44E56AAE44E6440D
:1005E0000EEBB2024FEAB30383EAB10E0EEA000E3D
:1005F0008EEAB10E0EEBF265D4F830E07544654436
:10060000EF1983EAB00515404FEAF76E5D40AE443E
:10061000656BAE44E6440EEBB1014FEAB20282EAEA
:10062000B00E0EEA070E8EEAB00E0EEBF165D4F8AE
:1006300038E075446544EB1882EAB7050D404FEA8F
:10064000F36E5540AE44E56BAE44E6440EEBB000AD
:100650004FEAB10181EAB70E0EEA030E8EEAB70E39
:100660000EEBF065D4F840E07544654481EAB30EC2
:10067000AA180EEA000E4FEAF2658EEA010E7544E2
:10068000DDF844E04FEAB000754480EAB30E6544FB
:100690000EEA020E15EBB7078EEAB30E0EEBF76506
:1006A000DDF848E04FEAB202754480EA020E654484
:1006B0000EEA070E69188EEA000E0EEBF165DDF802
:1006C0004CE07544654405EBB3034FEAB70E1427BD
:1006D0000DF1500CDFF810528EEA010B82EA0B0B81
:1006E0000BEBF36A5CF804BBDA44AA44504483EA97
:1006F000B10B4FEAF06A8EEA0B0BDA445CF804BBEC
:10070000DA44AA44524480EAB30B4FEAF26A8BEA15
:10071000B10BDA445CF804BBDA444FEAB000AA44F7
:1007200080EA020BD6448BEAB30B0BEBFE6A5CF853
:1007300004BBDA444FEAB202AA4482EA0E0B0AEB87
:10074000B10180EA0B0B0BEBF16A5CF804BBDA44F5
:100750007F1DAA44282F0AEBB3034FEABE0EBBD37A
:100760003C2F61D3502F4DD204EB870CC7F15407B7
:100770005E4CA7FB04A504465D4FA8088EEA010A5B
:1007800082EA0A0A5CF804BB0AEBF3655D447D1952
:100790002C1983EAB10A4FEAF4658EEA0A0A554435
:1007A0005CF804AB5CF804BB55447D19AA1884EAD4
:1007B000B30A4FEAF2658AEAB10A55445D444FEA4A
:1007C000B4047D1984EA020AAE448AEAB30A0AEB49
:1007D000FE655CF804AB55444FEAB2027D1982EA2B
:1007E0000E0A15EBB10184EA0A0A5CF804BB0AEBB5
:1007F000F1655D447D1915EBB303401E4FEABE0E53
:10080000BCD12046F46D1B19F365336EC9183166EF
:10081000716E71447166B36ED218B266F16E401893
:10082000F06650B0BDE8F08F4EEA010B0EEA010A07
:100830000BEA020B4BEA0A0A0AEBF36554F827A00D
:10084000DFF8B0C0554443EAB10B654403EAB10A8E
:100850000BEA0E0B28184BEA0A0A7F1C0AEBF0651C
:1008600054F827A0554440EAB30B654400EAB30AA4
:100870000BEAB10BAA184BEA0A0A7F1C0AEBF265D5
:1008800054F827A055444FEAB00040EA020B6544F3
:1008900000EA020A0BEAB30BAE444BEA0A0A7F1CD9
:1008A0000AEBFE6554F827A055444FEAB20242EA2B
:1008B0000E0B654402EA0E0A0BEA000B15EBB101C0
:1008C0004BEA0A0A7F1C0AEBF16554F827A055444D
:1008D0007F1C65443C2F05EBB3034FEABE0EA3D348
:1008E00040E700BF9979825AA1EBD96ECDCCCCCC30
:1008F000D6C162CADCBC1B8F00B581B00168074A53
:10090000914200D110B9064801B000BD7C212DF004
:1009100012FE4FF4003001B000BD00BF040A000811
:10092000030002002DE9F0410B4A92E8F85188B02B
:10093000694681E8F8510268084B9A4200D118B91B
:10094000074808B0BDE8F0811422083000F04FFBE2
:1009500008B0BDE8F08100BFE4090008040A0008FF
:1009600003000200152904D20268044B9A4200D108
:1009700008B903487047083000F048BB040A000873
:100980000300020010B481B013460268074CA24273
:1009900000D118B901B010BC0548704701B000F192
:1009A000240210BC083000F035BB00BF040A000868
:1009B0000300020010B481B013460268074CA24243
:1009C00000D118B901B010BC054870470A4601B003
:1009D00000F1240110BC083000F070BB040A0008CC
:1009E000030002000123456789ABCDEFFEDCBA9816
:1009F00076543210F0E1D2C3000000000000000085
:100A000000000000F9080008250900086509000831
:100A100085090008B509000809040008810F0008CD
:100A2000CD0F0008890F0008F0B5A3B004460B48AD
:100A300002900D4616461F46094B0822402104A885
:100A400000F0D1FA28980190009733462A462146B3
:100A500002A800F01BF823B0F0BD00BF040A000894
:100A6000180A000810B5040008BF002408D0054883
:100A7000054B20600822402104F1080000F0B3FA81
:100A8000204610BD040A0008180A00082DE9F041AC
:100A900004460E46216817464A681D469047804620
:100AA000B8F5003F19D12268069993682046984707
:100AB0008046B8F5003F10D123683146DE683A46DB
:100AC0002046B0478046B8F5003F06D12368079A14
:100AD00029461D692046A847804621680A682046A5
:100AE00090474046BDE8F08110B500F033FA4FF46E
:100AF000403400280EBF034C4FF4C0712DF01BFD95
:100B0000204610BD0200030010B5044600F022FA92
:100B100008B9054810BD0021A160D0F87C211168FA
:100B200088474FF4403010BD0200030070B5044602
:100B30000D4600F00FFA064E40B1D0F87C01416836
:100B40008847A84224BF65604FF44036304670BDE8
:100B5000020003002DE9FF4715000C4600D02CB120
:100B6000064600F0F7F95FEA000801D16448C3E0E7
:100B7000D8F8F80001684A689047B0F5003F17D1EF
:100B8000D8F87C118A68404690478146B9F1810FB8
:100B900080F09E80A94508F1FC0A17D2D8F8F80029
:100BA0000368D3F80CC02A462146E047B0F5003F61
:100BB00040F08E80D8F8F8000368D3F810C06A4679
:100BC0005146E047B0F5003F76D10AE0002004E04E
:100BD000215C0AF800100098401C00900098A84280
:100BE000F6D34FF0000C4749474A484B01AC0098F8
:100BF000844558D2D3E9007001ADC5E90070107882
:100C000000281ABF042086464FF0000E085854F8FA
:100C10000E5028443E4D05600127D0F800E0876063
:100C2000019D4F681AF80C007D408EEA050585F09D
:100C3000040E65680F687D4085F0FC05754485F0FD
:100C4000A30568400AF80C000CF1010CCFE7D3E9CA
:100C5000004501A8C0E9004510782E4D002814BFBA
:100C60004FF0040E4FF0000E01A8744651F80EE04C
:100C70000459A6440127CEF80050DEF80040CEF813
:100C800008704D68019F40687D406C400D68684069
:100C900084F0040480F0FC00041984F057040AF87E
:100CA0000C400CF1010CCC45D1D3D8F8F800016808
:100CB0004A689047B0F5003F0AD1D8F8F8000368B9
:100CC000D3F80C804A465146C047B0F5003F01D0EA
:100CD000114811E0002006E05AF8201081F06A3136
:100CE0004AF82010401CB0EB990FF5D3B06840F0E3
:100CF0000100B0604FF4403004B0BDE8F08700BFA1
:100D0000020003000C5B0308E40700202C0F00081E
:100D1000ADBE4ED70DBE75A10100030038B50C461F
:100D2000017A1546CA0702D500F014F908B9084837
:100D300032BDD0F8F80003682146DC682A46A04797
:100D4000B0F5003F01D0034832BD4FF4403032BD12
:100D500002000300010003002DE9F84191B00546AF
:100D60000E461746402101A82DF0E5FB297AC80759
:100D700004D5284600F0EEF8040002D1DFF8A48084
:100D80004BE0D4F8F800DFF8A0800368D3F810C077
:100D90006A4601A9E047B0F5003F3ED1D4F8F8001B
:100DA00001684A689047B0F5003F36D1D4F87C110D
:100DB0008A6820469047D4F8F830024618461B68E7
:100DC000D3F80CC004F1FC01E047B0F5003F24D19A
:100DD000D4F87C0141688847D4F8F83002461846B8
:100DE0001B68D3F80CC001A9E047B0F5003F14D14F
:100DF000D4F8F8000268696893689847B0F5003F36
:100E00000BD1D4F8F80003681C693A463146A04774
:100E1000B0F5003F08BF4FF44038404612B0BDE87F
:100E2000F08100BF02000300010003002DE9F8413A
:100E3000A5B0074688461646402115A82DF07BFB35
:100E400000220492402105A82DF075FB387AC107D5
:100E50005ED5384600F07EF8050059D0D5F8F80088
:100E60002D4C0368D3F810C06A4605A9E047B0F5D9
:100E7000003F3CD1D5F8F80001684A689047B0F5CA
:100E8000003F34D1D5F87C118A6828469047D5F8C0
:100E9000F830024618461B68D3F80CC005F1FC0177
:100EA000E047B0F5003F22D1D5F87C014168884782
:100EB000D5F8F830024618461B68D3F80CC005A9CF
:100EC000E047B0F5003F12D1D5F8F8000268796824
:100ED00093689847B0F5003F09D1D5F8F80003684A
:100EE0001D6904AA15A9A847B0F5003F01D0204606
:100EF0000FE00A4B0A490B4A0396029101924046C1
:100F00001C68049B009415AA796800F0E5F900E0DC
:100F1000054826B0BDE8F08101000300145B03081A
:100F2000936E030026C703000200030004B0010112
:100F300000170145E90A0008090B00082D0B0008FD
:100F4000BD030008550B00081D0D0008590D0008D1
:100F50002D0E00080168024A914218BF0020704718
:100F6000340F000810B5040008BF002404D0034863
:100F70002060204609688847204610BD340F0008CD
:100F800020225C302DF0D3BAF0B58468A30800228B
:100F900004F0030407E000F15C0555F8226035BA5F
:100FA00041F82250521C9A42F5D300220BE000F186
:100FB0005C0502EB830755F82360D500C5F11805E1
:100FC000EE40CE55521CA242F1D3F0BD30B5C468FC
:100FD00003690022E31AD5188C5C0544521C082AC8
:100FE0002C77F8D330BD0360C1600261704738B51B
:100FF000044615460022626023685A689047002024
:101000006061A061A5604FF4003032BD81604FF493
:10101000003070472DE9F84304462079D4F80C805D
:10102000450748BF244845D466691D46A8F101001C
:1010300000EAD60306EBC506B6EBC50F666102D221
:10104000A669761CA6611746A66906EB5576A661C9
:101050000E46E918884225D2A8EB03094A463146D4
:10106000F8182DF064FA2268136839460FE04246FA
:1010700038462DF05CFA23681A68394620469047B6
:1010800007E0311811F00300F1D1226813682046FF
:101090009847484600EB0809A9F10101A942F0D39D
:1010A000002300E000202A1A3118F8182DF03FFA2A
:1010B0004FF40030BDE8F283040002002DE9FC4F3C
:1010C000024685B0D0681369DFF86CC1DFF86C8127
:1010D000A0EB030A506840F004005060002703A80A
:1010E00002900DF10C0ED8E9003403A8544DC0E96C
:1010F00000342878534D00280CBF00230423994660
:101100005CF803305EF80940234401261D601C682A
:101110009E60DCF80430039DDCF80090DEF804608B
:101120005D406540484C654089EA0606474C66408C
:101130007519474C6540D8E9006B03AC0028C4E939
:10114000006B0EBF002404200424029E5CF8000003
:10115000345920183F4C04600126046886600398C7
:10116000029E43406340384C7068634089EA000047
:10117000364C6040034438484340280018BF0120E3
:101180005B1E9B41042F2CBFC0B2D80F02F1140389
:1011900053F8200007F00303C3F10303DB00D8403A
:1011A0000DF807007F1C082F9DD315460C466A6971
:1011B000AB69E868D20842EA4372401E00EA0207BF
:1011C000002302409B420AD8524508D28020E055B5
:1011D0007F1C574516D2AAEB0701E01910E08020CA
:1011E000E05500E0E355E8687F1C8742FAD32A689F
:1011F000136828469847BAF1000F03D0514620469D
:101200002DF099F92A68069E059F9368694628463D
:1012100098472A68D2F8009021462846C8472B688C
:10122000DA683946284690470EB1A86830604FF416
:10123000003007B0BDE8F08F0C5B03085C120008BB
:10124000E40700205FC5109304850012FC68017A52
:10125000C0F524FF24AF33D426AF698B04B001015D
:1012600000170145F8B501240094002300240DE087
:10127000009D065D0F5D7E40F643761CF60F86F0FE
:10128000010635400095641C009DEB189442EFD395
:101290001846F2BDF8B5002301240094002A11E09D
:1012A000009C85188F1815F8016C17F8015C6E40CA
:1012B000F643761CF60F86F0010634400094009C3D
:1012C000E318521EECD11846F2BD0000651200086A
:1012D00095120008010000002DE9F84F1D46DDF8C9
:1012E00028900B9F0D9C4FF0FF3300930E469246C3
:1012F000D9F800B0804632465146D847834664B399
:10130000D9F8043032465146404698476FEA0B02FE
:10131000521C42EA0B0200996FEAD2735B1C19401F
:10132000C2430091521C024300996FEAD2735B1CC6
:101330001940009186F05531484087EA000181F05C
:101340005531216080F05531C943491C0843009A4A
:101350006FEAD070401C82430092D9F8080001283F
:1013600009D17540E943491C0D4300986FEAD572D5
:10137000521C90430AE0F11C85EA9102D243521CB0
:10138000154300986FEAD5735B1C984386F0AA3624
:10139000009086EA0B0686F0AA33F243DB430C98F2
:1013A000C2F3C0725B1C42EAD3720099D243521C52
:1013B00091430091774000998843009987F0AA37BC
:1013C0000F403843BDE8F28F00000000000000002D
:1013D00001F0FF01102A2BDB10F0070F08D010F8E6
:1013E000013B013A8B422DD010F0070F42B3F6D1EA
:1013F000F0B441EA012141EA014122F007047FF003
:1014000000070023F0E80256083C85EA010586EA59
:10141000010685FA47F5A3FA87F586FA47F6A5FA95
:1014200087F68EB9EED1F0BC01F0FF0102F00702A1
:1014300032B110F8013B013A83EA010313B1F8D14C
:101440000020704701387047002D06BF354603382D
:10145000073815F0010F07D1013015F4807F02BF66
:10146000013015F4C03F0130F0BC0138704700BFB7
:10147000034613F8012B002AFBD1181A01387047D4
:1014800081F0004102E000BF83F0004330B54FEA35
:1014900041044FEA430594EA050F08BF90EA020FA2
:1014A0001FBF54EA000C55EA020C7FEA645C7FEA35
:1014B000655C00F0E2804FEA5454D4EB5555B8BF58
:1014C0006D420CDD2C4480EA020281EA030382EAC9
:1014D000000083EA010180EA020281EA0303362D5B
:1014E00088BF30BD11F0004F4FEA01314FF4801C2E
:1014F0004CEA113102D0404261EB410113F0004F40
:101500004FEA03334CEA133302D0524263EB4303F6
:1015100094EA050F00F0A780A4F10104D5F1200E94
:101520000DDB02FA0EFC22FA05F2801841F10001EF
:1015300003FA0EF2801843FA05F359410EE0A5F1C3
:1015400020050EF1200E012A03FA0EFC28BF4CF0F4
:10155000020C43FA05F3C01851EBE37101F00045AA
:1015600007D54FF0000EDCF1000C7EEB00006EEBB7
:101570000101B1F5801F1BD3B1F5001F0CD3490841
:101580005FEA30004FEA3C0C04F101044FEA445298
:1015900012F5800F80F09A80BCF1004F08BF5FEA1F
:1015A000500C50F1000041EB045141EA050130BDFF
:1015B0005FEA4C0C404141EB0101013C28BFB1F511
:1015C000801FE9D291F0000F04BF01460020B1FA5C
:1015D00081F308BF2033A3F10B03B3F120020CDA2F
:1015E0000C3208DD02F1140CC2F10C0201FA0CF00D
:1015F00021FA02F10CE002F11402D8BFC2F1200C72
:1016000001FA02F120FA0CFCDCBF41EA0C01904027
:10161000E41AA2BF01EB0451294330BD6FEA040470
:101620001F3C1CDA0C340EDC04F11404C4F120025B
:1016300020FA04F001FA02F340EA030021FA04F36D
:1016400045EA030130BDC4F10C04C4F1200220FAC4
:1016500002F001FA04F340EA0300294630BD21FA02
:1016600004F0294630BD94F0000F83F4801306BFC8
:1016700081F480110134013D4EE77FEA645C18BFBC
:101680007FEA655C29D094EA050F08BF90EA020F53
:1016900005D054EA000C04BF1946104630BD91EA4B
:1016A000030F1EBF0021002030BD5FEA545C05D14E
:1016B0004000494128BF41F0004130BD14F580048D
:1016C0003CBF01F5801130BD01F0004545F0FE4101
:1016D00041F470014FF0000030BD7FEA645C1ABF36
:1016E000194610467FEA655C1CBF0B46024650EA6D
:1016F000013406BF52EA033591EA030F41F4002199
:1017000030BD00BF90F0000F04BF0021704730B51E
:101710004FF4806404F132044FF000054FF00001F3
:1017200050E700BF90F0000F04BF0021704730B5B4
:101730004FF4806404F1320410F0004548BF404289
:101740004FF000013EE700BF42004FEAE2014FEADE
:1017500031014FEA02701FBF12F07F4393F07F4FB9
:1017600081F06051704732F07F4208BF704793F0BC
:101770007F4F04BF41F40021704730B54FF46074CF
:1017800001F0004521F000411CE700BF50EA0102D2
:1017900008BF704730B54FF000050AE050EA01027B
:1017A00008BF704730B511F0004502D5404261EBEB
:1017B00041014FF4806404F132045FEA915C3FF42C
:1017C000D8AE4FF003025FEADC0C18BF03325FEAC9
:1017D000DC0C18BF033202EBDC02C2F1200300FA7A
:1017E00003FC20FA02F001FA03FE40EA0E0021FA9F
:1017F00002F11444BDE600BF70B54FF0FF0C4CF48D
:10180000E06C1CEA11541DBF1CEA135594EA0C0F3E
:1018100095EA0C0F00F0DEF82C4481EA030621EA79
:101820004C5123EA4C5350EA013518BF52EA0335B4
:1018300041F4801143F4801338D0A0FB02CE4FF066
:101840000005E1FB02E506F00042E0FB03E54FF096
:101850000006E1FB03569CF0000F18BF4EF0010E8E
:10186000A4F1FF04B6F5007F64F5407404D25FEA8A
:101870004E0E6D4146EB060642EAC62141EA55513D
:101880004FEAC52040EA5E504FEACE2EB4F1FD0C7F
:1018900088BFBCF5E06F1ED8BEF1004F08BF5FEAFD
:1018A000500E50F1000041EB045170BD06F00046AF
:1018B00046EA010140EA020081EA0301B4EB5C045C
:1018C000C2BFD4EB0C0541EA045170BD41F4801154
:1018D0004FF0000E013C00F3AB8014F1360FDEBF79
:1018E000002001F0004170BDC4F10004203C35DA55
:1018F0000C341BDC04F11404C4F1200500FA05F3D8
:1019000020FA04F001FA05F240EA020001F0004278
:1019100021F0004110EBD37021FA04F642EB0601EE
:101920005EEA430E08BF20EAD37070BDC4F10C0418
:10193000C4F1200500FA04F320FA05F001FA04F2DC
:1019400040EA020001F0004110EBD37041F10001C8
:101950005EEA430E08BF20EAD37070BDC4F12005D3
:1019600000FA05F24EEA020E20FA04F301FA05F23B
:1019700043EA020321FA04F001F0004121FA04F2E3
:1019800020EA020000EBD3705EEA430E08BF20EAB3
:10199000D37070BD94F0000F0FD101F000464000ED
:1019A00041EB010111F4801F08BF013CF7D041EA6F
:1019B000060195F0000F18BF704703F00046520073
:1019C00043EB030313F4801F08BF013DF7D043EA44
:1019D0000603704794EA0C0F0CEA135518BF95EAFA
:1019E0000C0F0CD050EA410618BF52EA4306D1D181
:1019F00081EA030101F000414FF0000070BD50EAA0
:101A0000410606BF1046194652EA430619D094EA29
:101A10000C0F02D150EA013613D195EA0C0F05D113
:101A200052EA03361CBF104619460AD181EA030167
:101A300001F0004141F0FE4141F470014FF000001F
:101A400070BD41F0FE4141F4780170BD70B54FF0BA
:101A5000FF0C4CF4E06C1CEA11541DBF1CEA13553A
:101A600094EA0C0F95EA0C0F00F0A7F8A4EB05041C
:101A700081EA030E52EA03354FEA013100F0888013
:101A80004FEA03334FF0805545EA131343EA1263DC
:101A90004FEA022245EA111545EA10654FEA002691
:101AA0000EF000419D4208BF964244F1FD0404F54A
:101AB000407402D25B084FEA3202B61A65EB0305A6
:101AC0005B084FEA32024FF480104FF4002CB6EB63
:101AD000020E75EB030E22BFB61A754640EA0C00E3
:101AE0005B084FEA3202B6EB020E75EB030E22BF23
:101AF000B61A754640EA5C005B084FEA3202B6EB64
:101B0000020E75EB030E22BFB61A754640EA9C0022
:101B10005B084FEA3202B6EB020E75EB030E22BFF2
:101B2000B61A754640EADC0055EA060E18D04FEAB0
:101B3000051545EA16754FEA06164FEAC30343EA50
:101B400052734FEAC2025FEA1C1CC0D111F4801F1D
:101B50000BD141EA00014FF000004FF0004CB6E716
:101B600011F4801F04BF01430020B4F1FD0C88BFB5
:101B7000BCF5E06F3FF6AFAEB5EB030C04BFB6EBC0
:101B8000020C5FEA500C50F1000041EB045170BDB3
:101B90000EF0004E4EEA113114EB5C04C2BFD4EBE0
:101BA0000C0541EA045170BD41F480114FF0000E64
:101BB000013C90E645EA060E8DE60CEA135594EAE0
:101BC0000C0F08BF95EA0C0F3FF43BAF94EA0C0FE3
:101BD0000AD150EA01347FF434AF95EA0C0F7FF458
:101BE00025AF104619462CE795EA0C0F06D152EAAC
:101BF00003353FF4FDAE1046194622E750EA410690
:101C000018BF52EA43067FF4C5AE50EA41047FF4A0
:101C10000DAF52EA43057FF4EBAE12E74FF0FF3C05
:101C200006E000BF4FF0010C02E000BF4FF0010CD6
:101C30004DF804CD4FEA410C7FEA6C5C4FEA430C4F
:101C400018BF7FEA6C5C1BD001B050EA410C0CBF9E
:101C500052EA430C91EA030F02BF90EA020F002000
:101C6000704710F1000F91EA030F58BF994208BF67
:101C700090422CBFD8176FEAE37040F00100704724
:101C80004FEA410C7FEA6C5C02D150EA013C07D17B
:101C90004FEA430C7FEA6C5CD6D152EA033CD3D0C6
:101CA0005DF8040B704700BF8446104662468C46C0
:101CB0001946634600E000BF01B5FFF7B7FF0028F3
:101CC00048BF10F1000F01BD4DF808EDFFF7F4FF1C
:101CD0000CBF012000205DF808FB00BF4DF808EDA7
:101CE000FFF7EAFF34BF012000205DF808FB00BFCA
:101CF0004DF808EDFFF7E0FF94BF012000205DF8EC
:101D000008FB00BF4DF808EDFFF7CEFF94BF0120A0
:101D100000205DF808FB00BF4DF808EDFFF7C4FF99
:101D200034BF012000205DF808FB00BF4FEA410CE2
:101D30007FEA6C5C02D150EA013C0AD14FEA430CC5
:101D40007FEA6C5C02D152EA033C02D14FF0000002
:101D500070474FF0010070474FEA410212F5001240
:101D600015D211D56FF47873B3EB625212D94FEAE2
:101D7000C12343F0004343EA505311F0004F23FACC
:101D800002F018BF404270474FF00000704750EA21
:101D9000013005D111F0004008BF6FF000407047DE
:101DA0004FF00000704700BF4FEA4102B2F1E0433C
:101DB00024BFB3F5001CDCF1FE5C0DD901F0004C32
:101DC0004FEAC0024CEA5070B2F1004F40EB830082
:101DD00008BF20F00100704711F0804F21D113F1AE
:101DE0003872BCBF01F00040704741F480114FEAE7
:101DF0005252C2F11802C2F1200C10FA0CF320FA70
:101E000002F018BF40F001004FEAC1234FEAD3238C
:101E100003FA0CFC40EA0C0023FA02F34FEA4303F6
:101E2000CCE77FEA625307D150EA01331EBF4FF07F
:101E3000FE4040F44000704701F0004040F0FE409A
:101E400040F40000704700BF80F0004002E000BF97
:101E500081F0004142001FBF5FEA410392EA030F95
:101E60007FEA226C7FEA236C6AD04FEA1262D2EBDF
:101E70001363C1BFD218414048404140B8BF5B42E4
:101E8000192B88BF704710F0004F40F4000020F07D
:101E90007F4018BF404211F0004F41F4000121F093
:101EA0007F4118BF494292EA030F3FD0A2F10102DD
:101EB00041FA03FC10EB0C00C3F1200301FA03F11B
:101EC00000F0004302D5494260EB4000B0F5000F3E
:101ED00013D3B0F1807F06D340084FEA310102F1FD
:101EE0000102FE2A51D2B1F1004F40EBC25008BFAF
:101EF00020F0010040EA03007047490040EB000079
:101F0000013A28BFB0F5000FEDD2B0FA80FCACF179
:101F1000080CB2EB0C0200FA0CF0AABF00EBC250A6
:101F200052421843BCBFD0401843704792F0000F94
:101F300081F4000106BF80F400000132013BB5E7E7
:101F40004FEA41037FEA226C18BF7FEA236C21D05D
:101F500092EA030F04D092F0000F08BF08467047C2
:101F600090EA010F1CBF0020704712F07F4F04D190
:101F7000400028BF40F00040704712F100723CBFA3
:101F800000F50000704700F0004343F0FE4040F4CD
:101F9000000070477FEA226216BF08467FEA23638B
:101FA0000146420206BF5FEA412390EA010F40F476
:101FB000800070474FF0000304E000BF10F00043C2
:101FC00048BF40425FEA000C08BF704743F09643A9
:101FD00001464FF000001CE050EA010208BF7047C4
:101FE0004FF000030AE000BF50EA010208BF70474B
:101FF00011F0004302D5404261EB41015FEA010C60
:1020000002BF84460146002043F0B64308BFA3F157
:102010008053A3F50003BCFA8CF2083AA3EBC25339
:1020200010DB01FA02FC634400FA02FCC2F1200258
:10203000BCF1004F20FA02F243EB020008BF20F08F
:102040000100704702F1200201FA02FCC2F12002F5
:1020500050EA4C0021FA02F243EB020008BF20EAEA
:10206000DC7070474FF0FF0C1CEAD0521EBF1CEA18
:10207000D15392EA0C0F93EA0C0F6FD01A4480EA06
:10208000010C400218BF5FEA41211ED04FF00063EF
:1020900043EA501043EA5111A0FB01310CF000401B
:1020A000B1F5000F3EBF490041EAD3715B0040EA41
:1020B000010062F17F02FD2A1DD8B3F1004F40EB11
:1020C000C25008BF20F00100704790F0000F0CF0E4
:1020D000004C08BF49024CEA502040EA51207F3AA8
:1020E000C2BFD2F1FF0340EAC250704740F4000083
:1020F0004FF00003013A5DDC12F1190FDCBF00F074
:1021000000407047C2F10002410021FA02F1C2F121
:10211000200200FA02FC5FEA310040F1000053EABD
:102120004C0308BF20EADC70704792F0000F00F00B
:10213000004C02BF400010F4000F013AF9D040EA11
:102140000C0093F0000F01F0004C02BF490011F4A5
:10215000000F013BF9D041EA0C018FE70CEAD153A3
:1021600092EA0C0F18BF93EA0C0F0AD030F0004C23
:1021700018BF31F0004CD8D180EA010000F00040D7
:10218000704790F0000F17BF90F0004F084691F095
:10219000000F91F0004F14D092EA0C0F01D14202CF
:1021A0000FD193EA0C0F03D14B0218BF084608D198
:1021B00080EA010000F0004040F0FE4040F40000E2
:1021C000704740F0FE4040F4400070474FF0FF0C75
:1021D0001CEAD0521EBF1CEAD15392EA0C0F93EABC
:1021E0000C0F69D0A2EB030280EA010C49024FEA0E
:1021F000402037D04FF0805343EA111143EA1013C7
:102200000CF000408B4238BF5B0042F17D024FF47E
:10221000000C8B4224BF5B1A40EA0C00B3EB510F59
:1022200024BFA3EB510340EA5C00B3EB910F24BF42
:10223000A3EB910340EA9C00B3EBD10F24BFA3EBC7
:10224000D10340EADC001B0118BF5FEA1C1CE0D18F
:10225000FD2A3FF650AF8B4240EBC25008BF20F042
:10226000010070470CF0004C4CEA50207F32C2BF96
:10227000D2F1FF0340EAC250704740F400004FF033
:102280000003013A37E792F0000F00F0004C02BF64
:10229000400010F4000F013AF9D040EA0C0093F02E
:1022A000000F01F0004C02BF490011F4000F013B88
:1022B000F9D041EA0C0195E70CEAD15392EA0C0FF0
:1022C00008D142027FF47DAF93EA0C0F7FF470AF28
:1022D000084676E793EA0C0F04D14B023FF44CAF6B
:1022E00008466EE730F0004C18BF31F0004CCAD100
:1022F00030F000427FF45CAF31F000437FF43CAF3C
:102300005FE700BF4FF0FF3C06E000BF4FF0010C5D
:1023100002E000BF4FF0010C4DF804CD4FEA40023F
:102320004FEA41037FEA226C18BF7FEA236C11D089
:1023300001B052EA530C18BF90EA010F58BFB2EB3C
:10234000030088BFC81738BF6FEAE17018BF40F0BC
:10235000010070477FEA226C02D15FEA402C05D170
:102360007FEA236CE4D15FEA412CE1D05DF8040BF5
:10237000704700BF844608466146FFE70FB5FFF788
:10238000C9FF002848BF10F1000F0FBD4DF808ED40
:10239000FFF7F4FF0CBF012000205DF808FB00BF31
:1023A0004DF808EDFFF7EAFF34BF012000205DF88B
:1023B00008FB00BF4DF808EDFFF7E0FF94BF0120D8
:1023C00000205DF808FB00BF4DF808EDFFF7D2FFD5
:1023D00094BF012000205DF808FB00BF4DF808ED18
:1023E000FFF7C8FF34BF012000205DF808FB00BFE5
:1023F0004FEA40024FEA41037FEA226C02D15FEAD2
:10240000402C08D17FEA236C02D15FEA412C02D133
:102410004FF0000070474FF0010070474FEA400254
:10242000B2F1FE4F0FD34FF09E03B3EB12620DD902
:102430004FEA002343F0004310F0004F23FA02F06C
:1024400018BF404270474FF00000704712F1610F13
:1024500001D1420205D110F0004008BF6FF00040EA
:1024600070474FF00000704742000ED2B2F1FE4FAD
:102470000BD34FF09E03B3EB126209D44FEA002353
:1024800043F0004323FA02F070474FF0000070471A
:1024900012F1610F01D1420202D14FF0FF307047BB
:1024A0004FF00000704700BF53B94AB9002908BF78
:1024B00000281CBF4FF0FF314FF0FF3000F06AB929
:1024C000ADF1080C6DE904CE00F006F8DDF804E08B
:1024D000DDE9022304B070472DE9F047089D0C4662
:1024E000002B4ED194468C458646B2FA82F262D9D0
:1024F0004AB1C2F12003914020FA03F30CFA02FC26
:10250000194300FA02FE4FEA1C471FFA8CF6B1FB92
:10251000F7F44FEA1E4307FB141143EA014304FB9F
:1025200006F199420AD91CEB030304F1FF3080F055
:102530001281994240F20F81023C6344591A1FFAFA
:102540008EF3B1FBF7F007FB101143EA014300FBE8
:1025500006F69E420AD91CEB030300F1FF3180F01E
:10256000FC809E4240F2F980634402389B1B40EAA3
:10257000044000211DB1D3400022C5E90032BDE86E
:10258000F0878B4205D90DB1C5E90001002108464D
:10259000F5E7B3FA83F1002946D1A34202D3904272
:1025A000C0F0F080861A64EB03030120002DE6D012
:1025B000C5E90063E3E7002A40F09080A1EB0C043A
:1025C0004FEA1C481FFA8CF70121B4FBF8F64FEADA
:1025D0001E4308FB164443EA044307FB06F09842F7
:1025E00008D91CEB030306F1FF3402D2984200F233
:1025F000CD8026461C1A1FFA8EF3B4FBF8F008FBB8
:10260000104443EA044300FB07F79F4208D91CEB40
:10261000030300F1FF3402D29F4200F2B080204653
:10262000DB1B40EA0640A5E7C1F120068B4022FAF9
:1026300006F71F4320FA06FC04FA01F343EA0C03F1
:10264000F44000FA01F8380C4FEA1349B4FBF0FEED
:102650001FFA87FC00FB1E4449EA04440EFB0CF9F8
:10266000A14502FA01F20AD93C190EF1FF3A80F0B5
:102670008480A14540F28180AEF1020E3C44A4EB7F
:1026800009041FFA83F9B4FBF0F300FB134449EA91
:10269000044403FB0CFCA44507D93C1903F1FF30AB
:1026A00067D2A44565D9023B3C4443EA0E40A0FBF7
:1026B0000293A4EB0C049C42CE469C4651D34ED0D0
:1026C00055B1B8EB0E0364EB0C0404FA06F6CB40EC
:1026D0001E43CC40C5E90064002150E7C2F120034D
:1026E00020FA03F10CFA02FC24FA03F394400C43A1
:1026F0004FEA1C4800FA02FE1FFA8CF7B3FBF8F011
:1027000008FB1031230C43EA014300FB07F1994217
:1027100008D91CEB030300F1FF362CD299422AD9C9
:10272000023863445B1AA4B2B3FBF8F108FB11331F
:1027300044EA034401FB07F3A34208D91CEB040459
:1027400001F1FF3613D2A34211D902396444E41ACD
:1027500041EA004139E70446F0E6084606E7C84585
:10276000AED2B9EB020E63EB070C0138A8E7314695
:10277000EDE7034699E73046D4E7D6467FE7634462
:1027800002384DE70646234608460FE7023E6344FB
:1027900030E700BF704700BF00487047001BB74BD1
:1027A00070B50C4601F02CFA104E05460821304653
:1027B00005F0B6FF012804D001F022FA431BA34222
:1027C00007D30821094805F0ABFF431E5842584182
:1027D00070BD72B60821304605F0A2FF012800D076
:1027E00030BF62B6BFF36F8FE0E700BF0004004860
:1027F00008B5002210214FF0904005F097FF0548E2
:102800000022202105F092FFBDE80840022001F0DF
:10281000FFB900BF0004004810B50C4C0122102184
:10282000204605F083FF052001F0F2F92046012241
:10283000202105F07BFF4FF090400122102105F090
:1028400075FFBDE81040022001F0E2B90004004825
:1028500070B54FF090400C46164610210022144DE2
:1028600005F064FF00232B701248B3B222462146C4
:1028700007F050F9D8B901F0C3F941F287360446A0
:102880002B783BB1BDE87040012210214FF0904001
:1028900005F04CBF01F0B4F9031BB342F2D872B695
:1028A0002B7803B930BF62B6BFF36F8FE8E770BD16
:1028B000E507002048090020014B01221A707047EB
:1028C000E507002000487047185B030813B5114B5B
:1028D0000446186800909B88ADF804300120FFF78B
:1028E0009BFF062269460120FFF7B2FF0120FFF798
:1028F0007FFF9DF80430112B08D19DF80520122A86
:1029000004D101202370627002B010BD00231A466A
:102910001846F7E7F01903080CB4F0B5ADB032ABC8
:1029200006AF53F8042B059305460E46384696210C
:102930002BF050FD9528C1BF42F62E63ADF8AA30AA
:102940002E23ADF8AC3000F037F83C24042D4FF4C2
:102950007A7E1449B0FBFEFCB0FBF1F14EF6602329
:10296000B0FBF3F3B3FBF4F204FB1232BCFBF4F361
:1029700004FB13C30EFB1C049ABF0B48405D3F20B1
:10298000CDE90040CDE9026708482BF0A3FC084BD5
:102990001B6898682BF0C8FB2DB0BDE8F04002B072
:1029A000704700BF80EE3600765B0308545B030877
:1029B000F405002001F02CB901F022B91348144AA3
:1029C00008B54FF00043C0E9002304224261012210
:1029D0000023C2614FF480510722C0E90233C0E9ED
:1029E0000933C0E90C1203610383837680F8203039
:1029F00080F82C30826380F83C30C36404F0E8FD3A
:102A000018B1BDE8084000F099BB08BDE8070020F8
:102A1000002401400268084B9A4282B00AD14FF06C
:102A2000B0431A6E42F400721A661B6E03F4007310
:102A30000193019B02B07047002401400268054BDE
:102A40009A4201BF4FF0B042136E23F40073136635
:102A5000704700BF0024014030B585B00024054612
:102A6000CDE901440394FFF7A9FF144805F044F9A8
:102A700008B100F063FB1148039401A9CDE90154AA
:102A800004F004FF08B100F059FB0C4805F05EF8B3
:102A900008B100F053FB4FF0FF31084804F098FEF6
:102AA000064805F00BF9054804F0ECFE044603481F
:102AB00005F0AEF8204605B030BD00BFE8070020A5
:102AC000014B024A1A607047E807002000240140C9
:102AD00008B50948FFF7C0FF68B1084BB3F8AA3042
:102AE0004FF6FF72934216BF40F6E442044B534345
:102AF000B3FBF0F398B208BD002000B40075FF1FCF
:102B0000D8084C0013B50023ADF80630FFF7E0FFFE
:102B100004461948FFF7A0FF184BB3F8C820B3F8D4
:102B2000A8108A4204FB00F018D040F6E443B0FB42
:102B3000F3F364205B1A4343521A93FBF2F31E3300
:102B40001BB2ADF80630BDF806305BB21B02ADF823
:102B50000630BDF8060000B202B010BD4FF47A7224
:102B600040F6FF73B0FBF3F35343A3F53923A3F50A
:102B70000C6340F6C412E0E7001000B00075FF1FC0
:102B80004FF0B04382B09A6A22F480529A629A6CF3
:102B900042F480529A649B6C03F480530193019B2E
:102BA000002002B070474FF0B04307B59A6C42F076
:102BB00004029A649A6C02F004020192019A9A6CDF
:102BC00042F001029A649B6C002203F0010311465B
:102BD00000930B20009B05F02DF90B2005F05CF90C
:102BE000002211460C2005F025F90C2005F054F9BF
:102BF000002211460D2005F01DF90D2005F04CF9BD
:102C0000002202210F2005F015F90F2005F044F9EC
:102C100000221146102005F00DF9102005F03CF9B6
:102C200000221146112005F005F9112003B05DF8CE
:102C300004EB05F031B9000008B505F071FB10B1E7
:102C40006FF0040008BD064B9A6942F040429A6159
:102C50004CF2FA321A6105F075FB0028F2D0EFE76A
:102C600000400058F0B585B000230D46009306469D
:102C7000A8B3FFF7E1FF044670BB05F051FB88BB2A
:102C80001A481B4A02230193D0F8E01506F1784355
:102C900002EA8121B3FBF1F701FB1733DB0A029350
:102CA000D0F8E00505F178410139314402EA80228B
:102CB000B1FBF2F002FB1011C3EBD12301336946E3
:102CC00001A8039305F0BEFB20B1022814BF6FF0EA
:102CD0000104012405F036FB204605B0F0BD6FF07D
:102CE0000504F9E76FF00404F6E700BF0070FF1F6A
:102CF00000FCFF03014B1860002070474C080020C7
:102D00002DE9F04FB0F1006F89B006460F469046AE
:102D1000C0F0C080DFF89091644DD9F8E03505EA45
:102D2000832303F10063013B984200F2B380002942
:102D300000F0B38040EA02035B0740F0AE80FFF78B
:102D40007BFF044690BB05F0EBFA002840F0A8801A
:102D5000D9F8E015009705EA812106F17842B2FB27
:102D6000F1F301FB132208F17843013B3344B3FB39
:102D7000F1F001FB1033DB0A01334FEAD22AA3EB57
:102D8000D222012A039388BFC6F30A050AF58037C9
:102D9000C6F108038CBFC5F500654546FF02B34682
:102DA0000693039B9A4505D305F0CCFA204609B05B
:102DB000BDE8F08FA6F10803069A1A4495421CD884
:102DC000009B04950193CDF814B04FF00009059BCA
:102DD00009EB0301049B99453DD3009BAB442B4475
:102DE000A8EB0505B5F5006F009328BF4FF400650B
:102DF0000AF1010A07F50067D3E753F8081F5A687C
:102E0000B2F1FF3F08BFB1F1FF3FD5D0284B1868A2
:102E100010B96FF00504C7E727B14FF400623946D7
:102E200011F09CFDDFF888900099D9F80030CBF3C1
:102E30000A001844AAB211F091FD4FF4006138461F
:102E4000FFF710FF00BBD9F8003001934FF4006387
:102E500005970493B9E7019B07914B440293012026
:102E6000D3E9002305F0A8FA88B90799019BD1E9B5
:102E7000000259F80310029B5B689A4208BF88421F
:102E800005D109F10809A2E76FF001048CE76FF0A2
:102E9000030489E74FF0FF3488E76FF0050485E706
:102EA0006FF0040482E700BF0070FF1F00FCFF0307
:102EB0004C080020B1F1006F70B510D30B4BD3F864
:102EC000E0650B4B03EA862303F10063013B994263
:102ED00005D838B192B211F041FD002070BD4FF01D
:102EE000FF30FBE76FF00500F8E700BF0070FF1F41
:102EF00000FCFF03B0F1006F10B40DD3084BD3F802
:102F0000E045084B03EA842303F10063013B984248
:102F100002D810BCFFF7A6BE4FF0FF3010BC7047C0
:102F20000070FF1F00FCFF034FF0B04382B0DA6C6B
:102F30000243DA64DB6C03400193019B02B07047EB
:102F40002DE9F04186B01422002101A82BF060FA8F
:102F50000220464EFFF7E8FF0420FFF7E5FF0120BF
:102F6000FFF7E2FF04213046002205F0DFFB0022DC
:102F700010214FF0904005F0D9FB042300240125D7
:102F800002270DEB03013046CDE901354FF0100863
:102F9000CDE9034705F0A4FA01A93046CDE9018542
:102FA000CDE9037405F09CFA202301A93046CDE950
:102FB0000135CDE9037405F093FA01A94FF0904073
:102FC000CDE90185CDE9034405F08AFA08224FF4E2
:102FD000881301A93046CDE901234FF00308CDE95C
:102FE000034705F07DFA4FF4441301A94FF09040D8
:102FF000CDE90183CDE9035705F072FA4FF4405350
:1030000001A93046CDE90135CDE9034805F068FA5C
:103010004FF404134021CDE901131548039501A98C
:1030200005F05EFA22460F21062004F003FF062079
:1030300004F032FF22460F21072004F0FBFE072098
:1030400004F02AFF22462146092004F0F3FE09205D
:1030500004F022FF22462146092004F0EBFE09205D
:1030600004F01AFF06B0BDE8F08100BF000400487C
:103070000008004800B59BB04822002108A82BF0AA
:10308000C7F91822002102A82BF0C2F905F068FB4D
:103090004FF0B0420120D2F8903023F01803C2F86C
:1030A0009030D2F8003423F4C06343F40073C2F8C4
:1030B0000034D2F8003403F4C0630193019B24234D
:1030C000089381230B930023CDE91003B02208A8B5
:1030D000CDE9122305F0BCFC08B172B6FEE74F2320
:1030E000CDE90230CDE90400CDE90600022102A8B5
:1030F00005F048FF08B172B6FEE71BB05DF804FBAF
:1031000008B504F013FAFFF7B5FFFFF719FFFFF753
:103110004AFD00F0FDFF00F0ADFE00F089F8064822
:103120000122042105F002FB02F02EFC00F048FC15
:1031300002F031FCFCE700BF0004004872B6FEE775
:1031400000B58DB02C22002101A82BF061F91748A1
:10315000174B03601F2383604FF080420023C0E9B8
:103160000433C0E9072383614FF48073436206F0A0
:10317000AFF908B1FFF7E2FF0C4806F0D5FA08B145
:10318000FFF7DCFF4FF00053002207930748089237
:103190004FF4807301A9029206920B9306F0F8F99E
:1031A00008B1FFF7CBFF0DB05DF804FB500800201D
:1031B0000028004010B5044690B03822002102A833
:1031C0002BF026F92268194B9A422CD14FF4803308
:1031D000029302A84FF480730F9305F0F7FF08B134
:1031E000FFF7ACFF4FF0B0430220D3F8902042F439
:1031F0000042C3F890209A6D42F480629A659B6DFC
:10320000002203F4806311460193019B04F012FE37
:10321000022004F041FE00222A20114604F00AFE9A
:103220002A2004F039FE10B010BD00BF0028004075
:103230001148124A08B54FF48273C0E900230023F5
:103240004FF4E062C0E902324FF400712822C0E975
:1032500006120722C0E90433C0E90833C0E90B2392
:1032600083620823436306F0CFFB18B1BDE8084032
:10327000FFF764BF08BD00BF4809002000300140CF
:10328000F0B5054689B01422002103A82BF0C0F840
:103290002A68374B9A4269D14FF0B04302261A6E22
:1032A00042F480521A661A6E02F480520292029A16
:1032B000DA6C42F00102DA64DA6C02F00102019287
:1032C000019ADA6C42F00202DA64DB6C03F002036A
:1032D00000930524009B0327D02303A94FF09040BF
:1032E000CDE90336CDE9067405F0FAF82023CDE9DF
:1032F00003364FF09040002603A90794CDE90567F7
:103300001C4C05F0EDF81C4826620723C4E90003B5
:1033100080232046C4E90266C4E90436C4E906668F
:1033200004F01AFE08B1FFF709FF144AAC65A56264
:10333000134C0823C4E900231021002380222046D7
:10334000C4E90213C4E90423C4E90633236204F088
:1033500003FE08B1FFF7F2FE002222206C65114641
:10336000A56204F067FD222004F096FD09B0F0BDCF
:1033700000300140E80800201C00024030000240FC
:10338000880800207047000008B504F0E5F8044BF9
:103390000120C3F88800BDE8084005F039BA00BF35
:1033A0000004005808B504F0DEF800F0C1FFFFF794
:1033B000C7FDFFF7F8FB00F05DFDBDE80840FFF733
:1033C00037BF08B504F0CFF8FFF7BAFDFFF7EBFB06
:1033D000BDE80840FFF72CBF08B504F0BDF8BDE814
:1033E00008400121002005F0C3B970477047FEE78F
:1033F000FEE7FEE7FEE7FEE770477047704770475D
:10340000014806F0B7B900BF50080020024B012068
:10341000187005F099B900BFAA1E0020024B0122C6
:1034200002201A7005F090B9A91E0020082005F0AE
:103430008BB90000014804F005BF00BF5413002001
:10344000014804F0FFBE00BFE8080020014804F076
:10345000F9BE00BF8808002070470000014804F052
:10346000F1BE00BF0814002070470000014806F0BC
:103470003FBD00BF48090020014807F077BE00BFEC
:1034800068140020014805F0A9BF00BF50080020C3
:10349000014806F0BEBF00BF401300202DE9F043F5
:1034A00089B080460020109E0790894615461F4629
:1034B000FCF7BEFEF0B9104CCDE90090CDE9020456
:1034C00007AB0E480593142304933A464346294616
:1034D0000068FCF777FF2346324604F1140153F8E5
:1034E000044B42F8044B8B42F9D1079B337509B06A
:1034F000BDE8F0830120FAE7C2090020085B030859
:103500007FB5124C00253C2302A86375CDE9025516
:10351000257500F01FFB042303AA009412210C4818
:10352000FFF7BCFF0B49142220462AF061FF064634
:10353000B0FA80F040096075074B00902A46294692
:10354000022011F005F9304604B070BDAC0900202E
:10355000B25B03082E210020945B0308034A044851
:1035600040F21B53002107F077BC00BFD6090020B2
:10357000B4130020312BF0B52DD81825102415FBDD
:103580000343194D00244FF0800C4CFA04F6A3F1CC
:103590001007314205EB470714BF4FF0240E4FF0E0
:1035A000140EA7F806E0A3F10807304205EB470721
:1035B00014BF4FF0240E4FF0140E0134324205EBCD
:1035C0004306A7F806E00CBF14272427082CF78031
:1035D00003F10103D9D1054B1B781BB9BDE8F040BD
:1035E000FFF7BCBFF0BD00BFD6090020F01E0020D1
:1035F00010B500240022E3B2114610460134FFF753
:10360000B9FF322CF6D1BDE81040FFF7A7BF00008C
:1036100070B504460D46FFF7EBFF0F4B04EB440477
:1036200000261C440A2000F0F3FAA2786178207882
:1036300012FB05F211FB05F110FB05F0F3B2D2B25B
:10364000C9B2C0B20136FFF795FF322EEAD1BDE80C
:1036500070400A2000F0DCBA070000202DE9F0419C
:1036600006460F462048904600214FF416622AF085
:10367000CFFE1E4A10254FF0800C2B4600244CFA3A
:1036800004F1A3F110000F4202EB400014BF4FF011
:10369000240E4FF0140EA0F806E0A3F108000E422D
:1036A00002EB400014BF4FF0240E4FF0140E013413
:1036B00018EA010F02EB4301A0F806E00CBF14204A
:1036C0002420082CC88003F10103D8D11835B5F5A2
:1036D000986FD2D1064B1B781BB9BDE8F041FFF7BC
:1036E0003DBFBDE8F08100BFDC090020D609002005
:1036F000F01E002003460846072B1CD8DFE803F025
:1037000004070A0E121417190022114600E00022C5
:10371000104601E000221146FFF7A0BF0A46002133
:103720000020F9E70022F7E70A460021F0E70A4601
:10373000F6E70A46E9E770477FB502AC204611F08C
:1037400069FA94E80300824C824D2378012B85E8C6
:10375000030009D080490B7833B1804A13781BB13C
:103760007F4B1878052823D17E4B1A686AB92968DF
:1037700019607D49186808607C490A601B680093DD
:1037800011467B4B032010F0E3FF7A487A4D037813
:10379000DBB20A2B32D8DFE813F02C004D005100C9
:1037A000570060009700AA00B600C300C300C30022
:1037B0002078012806D1097821B9127812B91B782E
:1037C000052BE2D0694B1A68002ADED129681960FE
:1037D0006A491868086063490A6018681B680968C4
:1037E0005B1ACDE900031146654B032010F0B0FFD2
:1037F000CBE7644B1B78DBB2634A13700378634EEC
:10380000012B06D0624C227802F0FF03002A00F060
:103810008C805D4A002313702B703370FFF7E8FE35
:103820005C4A002313705C4A13705C4B01221A70CF
:1038300004B070BD544B00221A70DFE7584A12786A
:10384000012A08BF0123D7E7237813B94E4B012281
:10385000F2E72378012BD1D146E0444B414A1B6863
:1038600012689B1A042BC9D923783C4A53B93A4BA6
:103870001B78012B06D11378012BD9B202D1424B10
:103880001970BBE72378012B05D0334B1B7813B19C
:103890001378002BB2D13C4B0221197041490C78AE
:1038A000032C03D104212970197008E00C78012C35
:1038B00001D10821F7E70C78022CE1B2F3D012789D
:1038C000002A9BD10822B7E7237833B9344B1B7801
:1038D000012BDAB201D12C4BAEE72378012B03D0B8
:1038E0002F4B1B78002B89D1274B0222A4E723788A
:1038F0001BB92D4B1B78002BA8D02378012BF3D0BC
:10390000294B1B78A6E723781BB9154B1B78042B92
:103910009CD02378012BE7D0114B1B78052B9AE71D
:103920000F4B1A78042AF8D190E7227812B9164B77
:103930001B78DBB22B701D4B28781978FFF7DAFE65
:10394000237803B12B782B78DBB2337068E700BFA4
:103950008B1E0020901E00200A010020090100207B
:10396000891E0020A41E00209C1E0020A01E0020F6
:10397000C45B03080601002005000020981E0020FB
:10398000E75B03080400002006000020010000207F
:10399000F01E00208E1E00208D1E0020E81E00203C
:1039A0002D210020121500208A1E0020000000207A
:1039B000024803680021596307F0C8BAB413002015
:1039C000002270B50F4B1146022010F0C1FE0124F9
:1039D0000A25294620461435FFF78CFEEDB2322029
:1039E00000F016F96E2DF4D10134E4B2FFF700FEB9
:1039F000092CEDD10022BDE87040034B1146022096
:103A000010F0A6BE1E5C0308515C0308054808B50B
:103A10000823036006F01AFB18B1BDE80840FFF761
:103A20008DBB08BD401300204FF0B04307B55A6E60
:103A300042F001025A665B6E002203F0010301931B
:103A400011463220019B04F0F5F9322003B05DF8F5
:103A500004EB04F021BA00000CB407B5054A05AB2D
:103A60001021019311F084FA03B05DF804EB02B069
:103A7000704700BF875C030830B585B0044602A8D4
:103A80000D4611F0A1F8BDF90C30064A0093102143
:103A9000029B2046FFF7E0FF2046FDF7E9FC288067
:103AA00005B030BD875C03084FF0B04210B5936895
:103AB00023F40043936011F00FF9104B01241C70A4
:103AC00000F0ACF810F0DAFD0D4810F0F1FD0D4BF0
:103AD0004FF400421A61022010F0F0FDFEF7F0FFF3
:103AE00000F002F910F0E4FE2146204610F000FF3D
:103AF00021462046BDE8104010F0E4BE4C130020E3
:103B0000793A00080040005810F008BF08B5FEF7E9
:103B1000DFFF40F6B83398420CD8B0F5E16F0BD315
:103B2000FE23A0F5E16058434FF49663B0FBF3F039
:103B3000C0B208BDFE20FCE70020FAE77FB568466A
:103B400000F0B6F80198FEF769FC00B207B05DF826
:103B500004FB0000194A38B5D2F88035591C0446D8
:103B600019D103F007FD054603F010FD054403F0ED
:103B700007FD2B0EE3712B0CA3712B0A6371030E4F
:103B8000E370C0F30742C0F307232571C0B2A270EF
:103B90006370207038BD190AC3718171190C1B0E36
:103BA00041710371D2F88435C370D2F88405C0F333
:103BB0000722C0F30743000EE9E700BF0070FF1FB4
:103BC00038B5094BD3F8803503600133054609D178
:103BD00003F0D0FC044603F0D3FC444003F0D6FCD1
:103BE00044402C6038BD00BF0070FF1F012102203F
:103BF00010F068BE0021022010F064BE0020704763
:103C0000024B187808B100F0BFB970474C13002080
:103C100082B00190019802B000F052BAF0B5224A89
:103C2000224CD2F8903043F4804389B0C2F89030EF
:103C300003F0B2FC03F0B8FC03F0BEFC01230493D4
:103C40000323069300254FF0B04305950795DA6CE2
:103C500042F00202DA64DA6C02F002020292029A84
:103C6000DA6C42F00202DA64DB6C03F002030193C7
:103C70004FF4805703A92046019B03974FF4005649
:103C800004F02EFC03A92046039604F029FC2A46E2
:103C90003946204604F04AFD2A463146204604F0C3
:103CA00045FD09B0F0BD00BF000800580004004801
:103CB00010B50446FEF726FF074BA36040F30F2024
:103CC000FEF77CF9054B064A2360064B6060C4E9A9
:103CD0000323002010BD00BF0000484200007A44CA
:103CE0000D093E00AB03050000207047012070471E
:103CF00008B52AF0EFFB162303604FF0FF3008BD34
:103D000008B52AF0E7FB16230360FEE770B50D4601
:103D100014460E46731B9C4201DC204670BDAFF377
:103D2000008006F8010BF5E730B5104600234FF090
:103D30006042834200DB30BDD2F8804EE50707D5F4
:103D4000D2F8004EE40703D5CC5C156815B11470A9
:103D50000133EEE700BFF8E74FF0FF3070474FF454
:103D600000534B60002070470120704700207047CF
:103D70000B4A116810B5034609B90A491160106869
:103D800009490A4C0344091B8B4206D92AF0A2FBBD
:103D90000C2303604FF0FF3010BD1360FCE700BF41
:103DA00050130020E0400020000001200008000027
:103DB00037B5184B02689A42054628D14FF0B043F8
:103DC000154C1A6E42F400621A661B6E134A03F415
:103DD00000630193019B1723C4E9002310210023F2
:103DE0008020C4E902134FF48073C4E904034FF444
:103DF000806C2023C4E906C320464FF4005323629D
:103E000004F0AAF808B1FFF799F96C62A56203B053
:103E100030BD00BF002C01405413002008000240B8
:103E200010B5044686B01422002101A82AF0F0FA49
:103E300022680F4B9A4218D14FF0B04301A9DA6CB7
:103E400042F00102DA64DB6C03F00103009302220A
:103E5000009B4FF48073CDE901324FF09040012375
:103E6000CDE90332059304F03BFB06B010BD00BF63
:103E7000002C014010B58EB01022002103A82AF0BA
:103E8000C7FA00241C2221460DEB0200CDE90044B4
:103E900002942AF0BDFA1F481F4B8460C0E9003429
:103EA0003B23C0E90334C0E9054406F01BFD08B11B
:103EB000FFF744F94FF480531648039303A906F023
:103EC0002FFE08B1FFF73AF9124806F03BFD08B1A2
:103ED000FFF734F900240F4802946946CDE9004405
:103EE00007F036F808B1FFF729F9602309480D9467
:103EF000002207A9CDE90734CDE90944CDE90B44F7
:103F000006F088FD08B1FFF719F90248FFF788FFAE
:103F10000EB010BDB4130020002C0140014B1868F6
:103F2000704700BF001400200320704708B5014609
:103F30004FF47A7200238002890DFEF7B5FA08BDAE
:103F40004FF47A73A0FB0303800A40EA8350704762
:103F5000034B98689A689042FBD1C043704700BFFA
:103F60000028004008B5FFF7F3FF014B186008BDBB
:103F70000014002008B5FFF7EBFF024B1B68C01AC6
:103F800008BD00BF00140020024B187808B1FFF7ED
:103F9000DFBF70470414002010B5074B074C012207
:103FA000DA654FF48071204605F0DEF94FF0FF33FB
:103FB0002363002010BD00BF0028004050080020EF
:103FC00002460021014805F0E6BB00BF5008002072
:103FD00002460121014805F0DEBB00BF5008002069
:103FE00010B58CB02C220021044601A82AF010FA4A
:103FF000FFF7D2FF0C4B0D481B681C4400230893AD
:1040000006934FF00053E443079301224FF480736B
:1040100001A902940B9305F0BBFA08B1FFF78EF8E3
:1040200000200CB010BD00BF00140020500800207C
:1040300038B50546FFF78CFF02210446074805F016
:10404000B1FBC4F309024FF47A71A2FB0121920A79
:10405000A30A2A8043EA805038BD00BF50080020E0
:104060000148002105F09EBB5008002001480121B5
:1040700005F098BB50080020F8B50F4D2E78CEB94A
:104080000E4C4FF0FF372763FFF75AF8FFF784FF16
:104090004FF48071204605F067F92046276305F04C
:1040A00025FB32462046022105F075FBFFF75AFF3B
:1040B00001232B700020F8BD0414002050080020BC
:1040C000014610B54FF47A7200238002890DFEF785
:1040D000EBF90146FFF73CFF0446FFF739FF031BEE
:1040E0008B4200D310BD00BFF7E710F0FDBE00000B
:1040F00010B5064C0221204605F054FB0221421C5B
:104100002046BDE8104005F046BB00BF5008002027
:104110001648174A08B54FF4E133C0E900230023DD
:104120000C22C0E90233C0E90523C0E90733C0E926
:104130000933036107F0FFFD08B1FEF7FFFF0B48ED
:10414000002107F070FF08B1FEF7F8FF07480021D3
:1041500007F089FF08B1FEF7F1FF044807F043FFBD
:1041600018B1BDE80840FEF7E9BF08BD681400209B
:104170000044004070B596B006461422002103A802
:104180002AF046F93822002108A82AF041F93268BD
:10419000274B9A424AD10223089308A84FF44023A0
:1041A0000A9305F013F808B1FEF7C8FF4FF0B043CB
:1041B00000259A6D1F4C42F400329A659A6D02F404
:1041C00000320292029ADA6C42F00102DA64DB6C8D
:1041D00003F001030193019B0C220223CDE9032389
:1041E00003A907234FF090400793CDE9055504F04C
:1041F00077F9114925621423C4E900131023C4E997
:10420000023520468023C4E90435C4E9065503F08D
:10421000A3FE08B1FEF792FF2520F46700220221D9
:10422000A66203F007FE252003F036FE16B070BD2F
:1042300000440040081400208000024002680C4B3B
:104240009A4210B5044612D14FF0B0420C21936D42
:1042500023F4003393654FF0904004F0EDF9E06FE4
:1042600003F0ECFEBDE81040252003F023BE10BD96
:104270000044004008B50A460146024806F0DAFE4E
:10428000002008BD6814002013B5114B114C1860B4
:104290004FF40013009302AB13E90600204607F029
:1042A00046FE2368DA69D103FCD4DA695202FCD5F0
:1042B0009A68084842F480029A6007F07EFE064938
:1042C0000448012207F0ECFD002002B010BD00BF41
:1042D000FC140020681400200415002008B5074BCA
:1042E0001860FEF760FCFFF713FF054AD2F8803034
:1042F00043F00063C2F88030002008BD00150020A4
:104300000008005808B54FF0B04308489A6B42F4D3
:1043100000329A639A6B22F400329A63FFF78EFFA1
:10432000112003F0C7FD002008BD00BF6814002065
:1043300008B5074807F0FFFC08B1FEF7FFFE054887
:1043400003F00AFE18B1BDE80840FEF7F7BE08BD4D
:1043500068140020081400200268044B9A4203D11C
:10436000034B00201B681847704700BF0044004003
:104370000015002002680B4B9A4210B504460FD17D
:10438000094B1B682BB1D0F8902012B907480121C6
:10439000984720460549BDE81040012207F080BD3E
:1043A00010BD00BF00440040FC1400200415002094
:1043B0002DE9F04F9DB0FEF785FA13F03DFA024665
:1043C00040B90146644B022010F0C2F901201DB033
:1043D000BDE8F08F012013F0D7FA11F0D3FF0446A7
:1043E000039040B9024601465C4B022010F0B0F940
:1043F00013F096FAEAE75A4D296812F013FC69683F
:10440000204612F029FC297A204612F059FC697ADC
:10441000204612F089FC6969204612F015FDE86813
:10442000FEF722F881B2204612F098FC2969204656
:1044300012F060FCA97A204612F028FC02212046E6
:1044400012F0DAFC1021204612F018FD039812F049
:1044500021F80246049040B90146424B022010F078
:1044600077F903A811F0EEFFC2E703A811F0EAFF05
:10447000049812F077FB024640B901463A4B0220FD
:1044800010F066F904A812F023F9B1E7374EDFF80F
:10449000E0A0DFF8E0B0002333604FF0020804989A
:1044A00005AB0A2208A912F04FF9054628BB0246BF
:1044B0000146314B022010F04BF930682C49FDF7D2
:1044C000D1FD4FF07C51FDF7CDFD3060049812F026
:1044D00079FB044604A812F0FBF813F021FA002C33
:1044E0003FF474AF002D3FF471AF0022234B11460F
:1044F000032010F02DF9002069E731680998FDF7D5
:10450000A9FCBDF81890306000221D4BCDF800903A
:104510001146022010F01CF908AC0027BBB29945E7
:1045200004F1080405D8B8F1010FC6D04FF0010816
:10453000B5E754F8040C5146FDF794FDFDF794FFE0
:10454000019034F8083C009300225B46114602209B
:1045500010F0FEF80137E1E7E05C0308F85C0308BF
:10456000200000202D5D0308545D0308AC1E0020D0
:1045700000007A44B75D03087D5D0308CE5D030843
:10458000A65D030830B5044685B0084614491546B3
:10459000FDF768FDFDF742FFCCB1114902902846B6
:1045A000FDF760FDFDF73AFF0E4901902846FDF743
:1045B0004FFC0D49FDF70AFEFDF756FF0022009063
:1045C0000A4B1146032010F0C3F805B030BD00902F
:1045D000074B22462146032010F0BAF8F5E700BF4A
:1045E00000007A44CDCC4C3FCDCCCC3EE75D0308F7
:1045F000145E03082DE9F04FADF2344D4FF4007214
:1046000000210CA829F004FF4FF4007200218CA8AF
:10461000B34E29F0FDFE002537464FF000082C462A
:10462000B9682046FDF716FC796804462846FDF770
:1046300011FC08F10408B8F5007F054607F11007E2
:10464000EED14FF070512046FDF70CFD4FF0705148
:1046500004462846FDF706FD0025DFF8848207465C
:104660004FF00009AA46D8F808002146FDF7F0FBF4
:104670000146FDF7F7FC01465046FDF7EBFB3946D6
:104680008246D8F80400FDF7E3FB0146FDF7EAFC9B
:1046900001462846FDF7DEFB09F10409B9F5007F64
:1046A000054608F11008DED14FF070515046FDF775
:1046B000D9FC4FF070510A902846FDF7D3FC824692
:1046C0000A98FDF741F8874B00222BF015FECDE943
:1046D00004015046FDF738F8824B00222BF00CFE07
:1046E000FDF762FB0DF130090546C84600234FF087
:1046F000000BB168B0690693FDF7AAFBFDF78EFECB
:104700000028B8BF4042FDF759FC48F8040B0146A9
:104710005846FDF79FFB069B0433B3F5FE7F8346A7
:1047200006F11006E5D17049FDF750FD0DF1300896
:10473000064600234FF0000B314658F8040B069351
:10474000FDF786FB0146FDF78DFC069B01461846EA
:10475000FDF780FB0BF1010B1FFA8BFBBBF17F0F09
:104760000346E9D16049FDF731FDFCF7EDFF5D4BF4
:1047700000222BF0C1FDCDE906010DF50C78C346F2
:10478000002200234846D9F8001040680B93089295
:10479000FDF75EFBFDF742FE0028B8BF4042FDF783
:1047A0000DFC089A4BF8040B01461046FDF752FB2E
:1047B0000B9B01339BB27E2B09F104090246E1D128
:1047C0004A49FDF703FD4FF0000B8146002349469F
:1047D00058F8040B0893FDF73BFB0146FDF742FC3C
:1047E000089B01461846FDF735FB0BF1010B1FFA3C
:1047F0008BFBBBF17E0F0346E9D13C49FDF7E6FC9C
:10480000FCF7A2FF374B00222BF076FDCDE9080123
:1048100037492846FDF726FCFDF700FE3449029093
:104820005046FDF71FFCFDF7F9FD31490190384670
:10483000FDF718FCFDF7F2FD002211462D4B00900C
:1048400002200FF085FF2C492C4F2846FDF7B2FDC2
:1048500008B105233B702A4B1A782A4B1B889BB260
:104860009A4280F08C80284B1A78284B1B889BB288
:104870009A4206D226492046FDF7B0FD08B1012331
:104880003B70244FDFF890A03B880A9A01339BB21B
:104890003B803B889BB20A2B04BF00233B803B88B4
:1048A0004FF01C0B9BB20BFB03F3DDE904014AF84C
:1048B00003403B889BB20BFB03A35A603B889BB22F
:1048C0000BFB03A8FDF770FA3B88C8F808009BB201
:1048D0000BFB03A34FF08641DD603D8830461DE0B1
:1048E0002C1600200000E03F0000FE420000FC42C9
:1048F00000007A442A5E030800007A431215002063
:10490000A70300200A150020A60300200815002098
:10491000CDCC4C3F2C1E002014150020FDF7A2FB2F
:10492000ADB20BFB05A528613D88DDE90601FDF769
:104930003BFA4FF08641FDF795FBADB23B880BFB90
:1049400005A59BB26861324D0BFB03AA2A788AF851
:104950001820DDE90801FDF727FA4FF08641FDF741
:1049600081FBFDF781FD2B4BC0B218802B78012B0A
:1049700005D10022284B114602200FF0E9FE274FF7
:10498000234D3B78DFF89880012B24D1DFF89490F9
:10499000254EB9F80030B9F800204FF01C0A9BB240
:1049A00092B20AFB03F30AFB0262F0589168FDF72A
:1049B00051FA2146FDF712FDB0B102232B702B787E
:1049C000022BD8B204D10022184B11460FF0C0FEC2
:1049D0002B78DBB23B702B78DBB23B70C8F8004021
:1049E0000DF2344DBDE8F08FB9F80030D8F80090E2
:1049F0009BB20AFB03662046B168FDF72BFA4946D5
:104A0000FDF7ECFC10B103232B70E4E72870E2E71C
:104A10001215002006150020705E030810150020F6
:104A20000C1500202C1E002014150020B55E030874
:104A30002DE9F04F9FB0FDF745FF12F0FDFE024655
:104A400040B90146A84B03200FF082FE01201FB0A1
:104A5000BDE8F08F012012F097FF10F0ABFB044689
:104A60000D9040B902460146A04B03200FF070FEA6
:104A700012F056FFEAE79E4F3B78012BDDB252D091
:104A8000022D6FD0002D39D1042110F059FF0121E2
:104A9000204610F083FE9749204610F0B3FE964959
:104AA000204610F095FE9549204610F043FE9449AB
:104AB000204610F059FE0221204610F075FF914962
:104AC000204610F057FF214606A810F0B5FE8E4A8A
:104AD00019928E4A1A924FF07C53002218A9204650
:104AE00018931B921C921D9310F0D2FE294620466B
:104AF00010F0F2FE0321204610F008FF0D9800246C
:104B00003C7010F0EDFB02460E9000286DD1804BFA
:104B1000014603200FF01CFE0DA810F0B9FB0EA8F3
:104B200010F06CFCA4E77B4E294610F037FE71496B
:104B3000204610F067FEB168204610F0FBFDF168DA
:104B4000204610F011FE716A204610F041FEF16C13
:104B5000204610F00FFF704B0022114601200FF08D
:104B6000F7FDCBE76B4D012110F018FEE9692046F7
:104B700010F048FE696A204610F02AFEA968204617
:104B800010F0D8FDE968204610F0EEFDA86CFDF7A6
:104B90006BFC81B2204610F007FFE96C204610F054
:104BA000E9FE214606A810F047FE2B6B18936B6BAD
:104BB0001993AB6B1A93EB6B1B932B6C1C9318A97B
:104BC0006B6C1D93204610F063FEA86AFDF74CFC49
:104BD000C1B2204610F080FE286AFDF745FCC1B244
:104BE000204610F0FBFE4D4BB6E710F09DFC38B9A7
:104BF00000224B4B114603200FF0AAFD002026E7B0
:104C00001422214613A829F003FC0026DFF8EC80CB
:104C1000DFF81091DFF810A1212537460E980FA973
:104C200010F0DAFC0246002840F08A8001463F4B33
:104C300003200FF08DFDDFF8F8800E9810F094FC43
:104C4000B8F8003000229BB2114600930320394B84
:104C50000FF07EFD0D9D0121284610F09FFD0421DF
:104C6000284610F06DFE2349284610F0CBFD22495E
:104C7000284610F0ADFD2149284610F05BFD204983
:104C8000284610F071FD0221284610F08DFE1D49C6
:104C9000284610F06FFE294606A810F0CDFD1A4AEE
:104CA0001992254A1B924FF07C534FF07E5218A95F
:104CB00028461C9218931A931D9310F0E9FD0021C9
:104CC000284610F009FE0321284610F01FFE0D991A
:104CD0000EA810F0BDFB0246002840F0848001467B
:104CE000164B022016E700BFE05C0308FA5E0308DB
:104CF000A81E0020000082429A99993FCDCC4C3FDB
:104D0000000020406666263F000020410AD7233C71
:104D10007C5F0308301E00201A5F03084A5F030807
:104D2000975F0308CDCCCC3EA4030020B55F0308F9
:104D30002E1E0020DE5F0308CDCC4C3E136003081E
:104D4000119A10999DF83C00FFF71CFC9DF83C302F
:104D5000FBB1DDF844B038465946FDF77BF81099B1
:104D600007463046FDF776F8414606465846FDF7B9
:104D70006FF84946FDF72AFAFDF776FB1EAB80B2C5
:104D800003EB4000013430F82C3C0133E4B220F84E
:104D90002C3C9AF80030012B1ED1DFF818B2864A5D
:104DA000BBF8003011999BB202EB03139960BBF87A
:104DB00000309BB202EB0312109B5360BBF8003033
:104DC0009BB25A1C92B2802BABF8002004D1FFF7A3
:104DD00011FC0023ABF800300F20FDF7EBFD013D87
:104DE0007FF41CAF27E70E9810F09EFB00283FF4DD
:104DF000FFAE0DA810F04CFADFF8C0B14FF021095A
:104E00000E980FA910F0E8FB054600287CD1024659
:104E100001466B4B03200FF09BFCB8F80030DFF825
:104E2000A491DFF8A4B100229BB2114600930320A5
:104E3000664B0FF08DFC012C94BF0023012389F8F1
:104E4000003099F800300022CDE900431146604B54
:104E500003200FF07DFC0DF14C084FF0000A38F8EC
:104E6000022B3AB1CDE900A200225B461146012097
:104E70000FF06EFC0AF1010ABAF10A0FEFD15549A1
:104E80003846FDF7EFF807462046FDF797F88046CD
:104E900001463846FDF79AF94E4907463046FDF778
:104EA000E1F84146FDF792F94B4B1F604B4B002157
:104EB00018608046FDF76AFA0646A8B942234046C4
:104EC00099F80090CDE90343FDF7A8FA029038461F
:104ED000FDF7A4FA5FFA89F9CDE90090404B32461C
:104EE000314603200FF034FC0E9810F03DFB0446D1
:104EF0000EA810F083FA12F013FD002C3FF4A6ADBB
:104F000085F00100C0B2A2E5119A10999DF83C000D
:104F1000FFF738FB9DF84930002B43D19DF83C301A
:104F2000FBB1DDF844A038465146FCF793FF1099D9
:104F300007463046FCF78EFF2A4906465046FCF7E6
:104F400087FF5946FDF742F9FDF78EFA1EAB80B296
:104F500003EB4000013430F82C3C0133E4B220F87C
:104F60002C3C214B1B78012B1CD1B8F80030124A85
:104F700011999BB202EB03139960B8F800309BB211
:104F800002EB0312109B5360B8F800309BB25A1C1E
:104F900092B2802BA8F8002004D1FFF72BFB00234E
:104FA000A8F800300F20FDF705FDB9F101097FF4E5
:104FB00027AF32E72E1E00202C160020CDCCCC3E91
:104FC000B55F03088B1E002092600308336003085E
:104FD0005E60030800007A44841E0020801E0020CA
:104FE000B2600308CDCC4C3FA40300202DE9F04370
:104FF000ADB014230DF10E0204A9ADF80E3012F07D
:10500000A3FE044648B902460146194B03200FF09F
:105010009FFB20462DB0BDE8F0830022154B164FB4
:10502000DFF85880DFF85890114603200FF090FB0E
:105030000025BDF80E30AAB29342EAD9AAB22CAB31
:1050400003EBC202032012F89C6C52F8A03C002E25
:1050500014BF3A464246CDE9003200224B46114683
:105060000FF076FB002E05F1010508BF3446E0E79E
:105070000C6103082F61030802610308076103083C
:105080005361030830B5102289B000252946044633
:105090000DEB0200039529F0BBF914F0FFF92A4645
:1050A000A34B0090294603200FF052FBFDF70AFCAA
:1050B00012F0C2FB8DF80C0012F068FC431B18BF05
:1050C000012301218DF80D30029012F07DFC029831
:1050D00012F01CFE029812F091FC0298FFF786FF76
:1050E000002840F0008102A812F060FC12F018FCC9
:1050F000029812F09FFC029812F0B8FC0298FFF799
:1051000075FF002840F0F38002A812F04FFC12F067
:1051100007FC029812F0C6FC0022864B11460320C1
:105120000FF016FB029812F0D9FC0298FFF75EFF11
:10513000002840F0E08002A812F038FC12F0F0FBEA
:10514000029812F0E7FC002211467B4B03200FF07F
:10515000FFFA0022794B114603200FF0F9FA02986A
:1051600012F064FD0298FFF741FF002840F0C7806D
:1051700002A812F01BFC12F0D3FB029812F072FD91
:10518000002211466E4B03200FF0E2FA00226D4B15
:10519000114603200FF0DCFA029812F07FFD02980E
:1051A000FFF724FF002840F0AE8002A812F0FEFBBB
:1051B00012F0B6FB029812F08DFD00221146624BF0
:1051C00003200FF0C5FA0022604B114603200FF0B8
:1051D000BFFA029812F0BAFC0298FFF707FF002806
:1051E00040F0958002A812F0E1FB12F099FB0298C2
:1051F00012F0C8FC00221146554B03200FF0A8FA0C
:105200000022544B114603200FF0A2FA029812F02C
:10521000D5FC0298FFF7EAFE00287CD102A812F024
:10522000C5FB12F07DFB029812F0E4FC002211464F
:10523000494B03200FF08CFA0022404B114603200B
:105240000FF086FA029812F0F1FC0298FFF7CEFEFA
:10525000002864D102A812F0A9FB12F061FB0298A9
:1052600012F000FD00221146354B03200FF070FABA
:105270000022344B114603200FF06AFA029812F014
:105280000DFD0298FFF7B2FE00284CD102A812F0E3
:105290008DFB12F045FB029812F01CFD0022114616
:1052A000294B03200FF054FA002211462B4B032008
:1052B0000FF04EFA01238DF8173003AB03CB002219
:1052C0002060186861600C23A060114600930320E1
:1052D000234B0FF03DFA02A812F068FB12F020FBFE
:1052E000002009B030BD01238DF80E3000E7012306
:1052F0008DF80F300DE701238DF8103020E70123E2
:105300008DF8113039E701238DF8123052E701236F
:105310008DF813306BE701238DF8143083E70123F8
:105320008DF815309BE701238DF81630B3E700BFE9
:105330006961030892610308C5610308F661030807
:10534000256203085262030887620308BA620308F1
:10535000ED6203081E6303084E6303087C630308C1
:10536000A963030802480122102103F0DFB900BF3E
:105370000004004802480022102103F0D7B900BF02
:105380000004004813B5134C23785BB9E37C03F0A9
:10539000FF023BB9104B1146022002B0BDE810409D
:1053A0000FF0D6B9FEF7ACF800380C4B18BF01204F
:1053B000400018701A78022A02BF00222270E2749C
:1053C0001B7800930022064B114603200FF0C0F912
:1053D00002B010BD2E210020C8630308F01E00207B
:1053E000E463030838B5184C23785BBBE37C03F017
:1053F000FF023BBB154D2B68012B0CD92B68042BEE
:1054000009D81146124B02200FF0A2F9114A0421CB
:10541000012000F0F5FE2B68042B13D900220E4B5F
:10542000114602200FF094F9FEF76AF800380B4B92
:1054300018BF0120400018701B78022B02BF002308
:105440002370E37438BD00BF2E210020EC1E002025
:10545000FB6303082064030825640308F01E002092
:1054600010B501214FF0904003F05AF90C4B0D4A52
:105470001870002414701B780B4ADBB202214FF025
:105480009040137003F04CF9084B094A18701470DF
:105490001B78084ADBB21370BDE81040FEF74CB928
:1054A0000A010020AA1E0020080100200901002096
:1054B000A91E00200701002010B5164B1A78022AF9
:1054C00026D91B78072B23D8FFF7B2FA1248134AC4
:1054D000037811785B1A124918BF01230B70037807
:1054E0001048DBB21370104B104A1C780378E31A93
:1054F00018BF012313700E4B04701B7823B10023D7
:105500000B700C490B701370BDE81040FEF714B916
:1055100010BD00BF060100208B1E0020881E002049
:105520008C1E0020101500201215002011150020DF
:10553000F01E00208E1E002008B501214FF0904083
:1055400003F0EEF8064B012816BF022218701A70FD
:105550001878044B1978BDE80840FEF759B800BF29
:10556000050000200000002038B5324D324C287B69
:10557000FCF720FD3149FCF775FDA060687BFCF766
:1055800019FD2E49FCF76EFDE060A87BFCF712FDCB
:105590002A49FCF767FD6062E87BFCF70BFD2849B0
:1055A000FCF760FD274BE0642361287CFCF702FDDB
:1055B0006060687CFCF7FEFCA061A87CFCF7FAFC4C
:1055C000E061E87CFCF7F6FC2062287DFCF7F2FC49
:1055D000A062687DFCF7F2FC1849FCF743FD2063EC
:1055E000A87DFCF7E7FC6063E87DFCF7E7FC144965
:1055F000FCF738FDA063287EFCF7DCFCE063687EE6
:10560000FCF7DCFC0D49FCF72DFD2064A87EFCF7BF
:10561000D5FC0A49FCF726FD6064E87EFCF7CAFC6D
:10562000A064287FFCF7C6FC074BE06202221A70D8
:1056300038BD00BF58030020301E0020CDCCCC3D2B
:105640000AD7233CCDCCCC3EA81E002038B5114D46
:10565000114C287BFCF7B2FC1049FCF703FDA0605D
:10566000687BFCF7ABFC0D49FCF7FCFCE060A87B19
:10567000FCF7A4FC0949FCF7F5FC6062E87BFCF749
:105680009DFC0749FCF7EEFC064BE06401221A7012
:1056900038BD00BF58030020301E0020CDCCCC3DCB
:1056A0000AD7233CA81E00207FB5394E394D3378E8
:1056B0000370394B1B784370044601214FF0904032
:1056C00003F02EF82B78A070E37002214FF0904089
:1056D00003F026F8314B20711B7863712B78012B76
:1056E00052D12F4B1868FCF7BFFE2E4BE080186894
:1056F000FCF7BAFE80B22C4BA0831B7884F82430D0
:10570000191F4A424A41A2779BB1284A03EB8303FF
:1057100002EB8303002200931146254B02200FF079
:1057200017F8244B1B8884F82530234B1B8884F8FA
:10573000263002A80FF06EFA204B1A78FAB1204AF0
:105740001168E1B112681F4A15681F4A12681B7878
:10575000AD1AC3EB0313B5EB830F10D900221B4B1B
:10576000114602200EF0F4FF194B258501221A7014
:105770001B78184A84F82730082313703370164BAF
:1057800001221A7004B070BD0020E080B3E700BFB2
:10579000050000208B1E0020060100208A1E00202C
:1057A000841E0020801E0020121500203E000020D4
:1057B000586403080A15002006150020A5030020E0
:1057C000A41E00209C1E0020981E00208664030852
:1057D0002B21002006000020E81E0020024B0122A1
:1057E000002103200EF0B4BFA6640308024B01227F
:1057F000002103200EF0ACBFDC64030808B50122D1
:10580000074B002103200EF0A3FFFFF7ABFDFFF7CE
:10581000ABFE044A00231370034A137008BD00BF97
:1058200022650308A81E00202921002010B5104B76
:105830000122002102200EF08BFF0E4B04225A7031
:105840006321012200241A7083F82A1083F82B2088
:105850001C635C6383F827401C85FFF783FDFFF71B
:10586000C5FFFFF7BBFFFFF7C9FF034B1C7010BD5F
:1058700058650308B01E0020292100201FB5114BD8
:1058800011491C6858681A7A5B7ACDE90223FCF743
:10589000E9FBFCF7E9FD0C4901902046FCF7E2FB2F
:1058A000FCF7E2FD0022094B0090114603200EF0A8
:1058B0004FFFFEF77DFD642004B0BDE81040FEF709
:1058C000A7B900BF2000002000007A448F650308BC
:1058D00070B586B00D460446FFF744FD01F026FE84
:1058E000FDF72EFB9620FEF793F90026AE420AD173
:1058F00001AB03CB1B882381094B20600022616030
:105900001A7006B070BDFEF75BF801A8FFF7BAFB8E
:1059100041F28830FEF77CF90136FFF7AFFFE5E78B
:105920002921002030B585B00446002503A8ADF834
:105930000C50FCF7CBFF70B19DF80C309DF80D209A
:10594000237062702946CDE900320320034B2A46BA
:105950000EF0FEFE012005B030BD00BFC465030897
:10596000022801D8FFF7FEBC7047022801D8FFF7D4
:1059700001BD7047022803D80248102102F0DBBEA7
:10598000704700BF0004004808B5FEF78DF8BDE879
:10599000084000F06DBE4FF0FF300FF023B87047A5
:1059A00070470000014BD870704700BF18010020FD
:1059B000014B1874704700BF1801002007B5064B53
:1059C00000221B5C00931146044B02200EF0C0FE27
:1059D00003B05DF804FB00BF03660308E965030834
:1059E00008B5002102200EF0C5FF0A4B1B7803F01A
:1059F000FF014BB9084B1A68042A05D81A68102011
:105A000001321A600EF0B6FFBDE8084003480FF0FF
:105A100019BA00BF2E210020EC1E0020902000208B
:105A2000002101200EF0A6BF13B5104A104C42F21F
:105A30001073002818BF03460E48236013600FF050
:105A4000B3F921680B480FF037FA0A480FF0FAF95A
:105A500023684FF47A72B3FBF2F3002200931146ED
:105A6000054B01200EF074FE02B010BD9C03002017
:105A700014010020902000200766030813B50D4C88
:105A8000206023680BB90C4B23600C480FF08CF995
:105A900021680A480FF010FA08480FF0D3F923687C
:105AA00000930022064B114603200EF051FE02B077
:105AB00010BD00BF9C030020A0860100F41E002042
:105AC0003366030837B50446002841D090F90650E4
:105AD000002D4AD128480FF067F9FDF789FD274BC3
:105AE00001221A70FDF73AFD2A462946244B02206E
:105AF0000EF02EFEE379012B0CBF224B224B2A46DF
:105B000029460220214D0EF023FEE3792B70204B15
:105B10001868FFF7B3FF1F4B1868FFF785FF297858
:105B20001D4A1E4B012908BF13460022009311464F
:105B30001B4B01200EF00CFE94F90530019394F9F3
:105B4000043000930022174B114603200EF000FE94
:105B5000154B0122002102201A700EF00BFF134892
:105B600003B0BDE830400FF06DB90022104B114674
:105B700002200EF0EDFDDFE73C1F002005000020B5
:105B8000786603088D660308AA6603082A210020A8
:105B90009C030020140100206F660308736603084D
:105BA000C7660308FF66030828210020241F002081
:105BB000E66603080A460149FDF77CB900F00308D0
:105BC00070B516480FF0F0F806F0AEFE044650B17E
:105BD0000022134B114602200EF0BAFDBDE87040C2
:105BE00010480FF02FB9104D104B0246014602200D
:105BF0000EF0AEFD01260E4B2E70224621460220ED
:105C00000EF0A6FD0B4806F023FD2878314606F07D
:105C100077FA02480FF016F9E0E700BF9020002065
:105C200028670308782000207C01002046670308CD
:105C30005A67030818010020F0B599B0FDF766FF18
:105C4000054606F057FB074600283ED16F4C0AA8D0
:105C5000FFF72AFD132323706D4B1A7802F0FF061D
:105C6000002A43D01F70142323706A4B62681B788C
:105C700063F07F031370636828B200EB400000EB11
:105C80004010FE22B0FBF2F058700223624A1278F4
:105C9000012A88BF00236370604C637A33B106F039
:105CA00015FB012802D120460FF07EF85C4B5748C7
:105CB000D978002206F034FB0146002840F091809C
:105CC0000122584B10460EF043FD002456480FF0B9
:105CD0006BF8564B54481968A14238BF21460FF063
:105CE000EBF851480FF0AEF819B0F0BD504A1178FA
:105CF00001F0FF030029C9D0464B16701B7862687B
:105D000063F07F03137063689DF828505D706268CC
:105D10009DF82930937062689DF82A10D1706268EE
:105D20009DF82B10117162689DF82C1051716268FA
:105D30009DF82D109171BDF82E206168120ACA716C
:105D40006068BDF82E200272BDF84420120A42722B
:105D5000BDF8442082729DF84620C2729DF84C2006
:105D600002739DF84F204273BDF85020120A8273CF
:105D7000BDF85020C27303EB83032E4A03EB830369
:105D8000134401932C4B05EB850503EB450300936E
:105D900032462A4B314601200EF0DAFC9DF84C3099
:105DA0000893BDF84A3007939DF846300693BDF836
:105DB00044300593BDF82E3004939DF82D300393A5
:105DC0009DF82C3002939DF82B3001939DF82A30DA
:105DD000009332461A4B314601200EF0B9FC1023D5
:105DE00054E706317FF471AF06F06AFA04460028E2
:105DF0003FF46BAF01224FF47A730021B0FBF3F351
:105E0000104600930F4B0EF0A3FC5FE70C0100203F
:105E100028210020841F0020F01E00203C1F0020AD
:105E200018010020B8680308902000201401002009
:105E3000E81E00207D010020F4020020796703089D
:105E4000A4670308C768030800B503468DB000289F
:105E50002CD0407802280AD003282AD0164B0022E2
:105E6000114602200DB05DF804EB0EF071BC1A7FF4
:105E70000B92DA7E0A929A7E09925A7E08921A7ED4
:105E80000792DA7D06929A7D05925A680492DA6842
:105E9000039293F914200292B3F9122001921B7C11
:105EA00000930022054B11460EF052FC0DB05DF838
:105EB00004FB034BD3E700BFE5680308FC68030855
:105EC0006E69030801284FF000020CBF024B034B20
:105ED000114602200EF03CBC8D6903089F6903083F
:105EE0001FB50446002831D00378002B2ED01D4862
:105EF0000EF0A8FF002211461B4B02200EF028FCDA
:105F000094F91830039394F90A300293237C019397
:105F1000E368009300221146144B03200EF018FC96
:105F20000022134B114603200EF012FC237A012BA2
:105F30000ED1617A0F4A104B002918BF1346002278
:105F4000009311460D4B03200EF002FC04B010BD6F
:105F500000220B4B1146032004B0BDE810400EF0A8
:105F6000F7BB00BF6C1F0020B8690308E96903088C
:105F70001A6A0308B4690308B3690308276A0308A7
:105F8000386A030808B5104B0122002102201A705C
:105F90000EF0F0FC0D480EF055FF0D4B1B788BB149
:105FA0000C4B1A7872B9DB7C63B90B4B1A68042A64
:105FB0009EBF1A6801321A600021BDE80840102017
:105FC0000EF0D8BC08BD00BF28210020F41E002020
:105FD0002A2100202E210020EC1E002008B50021DF
:105FE00040200EF0C7FC074B1B7853B1064B1A78C4
:105FF000012A06D100211970BDE8084002200EF0E8
:10600000B9BC08BD2A2100208C1E0020044B1B783F
:10601000022B03D1002108200EF0ACBC704700BF5A
:106020007C010020044B1B78012B03D00021802031
:106030000EF0A0BC704700BF0601002008B506F0B6
:106040007CFC80B906F042F901280CD1BFF34F8FD8
:106050000549064BCA6802F4E0621343CB60BFF304
:106060004F8F00BFFDE708BD00ED00E00400FA051A
:1060700038B504460D4607484FF40061FCF73AFF77
:1060800030B92A4621460348BDE83840FCF738BEFF
:1060900038BD00BF00F0030810B506F0E3FC10F1B6
:1060A000080F07D1064B0022BDE810401146022020
:1060B0000EF04EBB013001D1024BF4E710BD00BF22
:1060C000466A03085C6A030838B50F4C2378082B2E
:1060D0000DD10E4C23781E213BB10220FDF70AFBA7
:1060E000237883F00103237038BD0320F6E7084DC1
:1060F0002A7823789A42F7D020781E21FDF7FAFA01
:106100002378DBB22B70EFE7050000209803002016
:106110002C21002070470000022837B5044634D0F7
:10612000402853D0012854D12B4B1B78002B50D042
:10613000FA20FDF76DFD21464FF0904002F0F0FA95
:10614000264B214618704FF0904002F0E9FA2146A4
:1061500005464FF0904002F0E3FA214B214A002817
:1061600008BF1346CDE900531F4B00221146022001
:106170000EF0EEFA002120200EF0FCFB00210220A0
:1061800003B0BDE830400EF0F5BB184B1B7803B3ED
:10619000FA20FDF73DFD21464FF0904002F0C0FA95
:1061A000134B214618704FF0904002F0B9FA214687
:1061B00005464FF0904002F0B3FA0E4B0E4A00280D
:1061C00008BF1346CDE900530C4BCEE70021042055
:1061D000D6E703B030BD00BFAA1E00200300002098
:1061E000806A0308746A0308A66A0308A91E0020CF
:1061F00002000020996A03088C6A0308CC6A03082D
:1062000073B505460C46164606F074F8034600289A
:1062100040D000242A480EF0C7FD2A4B28481968B0
:10622000A14238BF21460EF047FE254802B0BDE826
:1062300070400EF007BE4A68F05CD0540133DAB209
:106240009442F8D8204B0D701A781B78012A88BF29
:1062500000244C700022CDE900341C4C1C4B11462C
:1062600001200EF075FA637A33B106F02FF8012899
:1062700002D120460EF098FD164B1748D97800221F
:1062800006F04EF8014638B9144B012203200EF0F7
:106290005FFABEE71049D2E70631BAD106F010F82E
:1062A00004460028B6D04FF47A730122B0FBF3F312
:1062B0000021009303200A4B0EF04AFAAAE700BF20
:1062C0009020002014010020F01E00203C1F002020
:1062D000F16A0308180100200C010020B8680308C7
:1062E000C7680308044B1B7823B9044A0521012021
:1062F000FFF786BF704700BFF01E0020226B030827
:1063000010B5002490B03C22214601A8009428F04A
:106310007FF8354B2022DA7219788DF80010597801
:106320008DF8011099788DF80210D9788DF8031046
:1063300019798DF8041059798DF8051099798DF82F
:106340000610D9798DF80710197A8DF80810597A46
:106350008DF80910997A8DF80A108DF80B202146D6
:106360000DF10B0258180131007B02F8010F1C29B6
:10637000F8D193F828208DF8282093F829208DF85B
:10638000292093F82A208DF82A2093F82B2093F8BF
:1063900028108DF82B20154A19BB93F8291001F00D
:1063A000FF00F1B9107093F82C206AB193F83F20E8
:1063B00052B10DF12B0100229818013290F82C00F7
:1063C00001F8010F142AF7D109484FF40061FCF7D6
:1063D00091FD20B9064840226946FCF791FC10B0B7
:1063E00010BD01211170DEE758030020A403002036
:1063F00000F8030810B5002204461146054B0220A0
:106400000EF0A6F920460449BDE8104040220EF0E7
:10641000A5BA00BF286B030800F8030873B54B4CFE
:10642000207963794D2BC0B25ED1C0EB00108000A3
:106430000A2838BF0A204FF47A735843444B186037
:10644000A379E2794D2ADBB256D1C3EB03139B004B
:106450004FF47A7202FB03F594F82C30002B53D1E1
:1064600094F83F30002B4FD142F21070FFF7DCFA66
:10647000384B1868FFF702FB237A374A3749DBB2FB
:106480001370374B01221A70637A364ADBB21370ED
:1064900094F82830344A03EB83035B00DBB21370BB
:1064A00094F82930314A03EB83035B00DBB21370AD
:1064B00094F82B302E4A03EB83035B00DBB213709E
:1064C0000023E21892F82C20D2B2CA540133142BC4
:1064D000F7D1A378012B37D1E37A202B34D102B046
:1064E000BDE87040FFF7A2B96379482B0ABF4FF4AB
:1064F0006163637958439BE7E279482A0ABF4FF406
:106500006162E2795343A3E71A4EFFF78DFA3560D3
:10651000336813B942F21073336017480EF044FC2D
:10652000316815480EF0C8FC13480EF08BFC336838
:106530004FF47A72B3FBF2F30022009311460F4B33
:1065400001200EF005F997E702B070BD5803002056
:10655000140100209C030020060100202E210020B1
:1065600005000020F01E0020A7030020A603002045
:10657000A5030020A00300200C1F00203C6B030893
:1065800010B590B000213C2201A8009127F040FFF7
:106590004022344968460EF0E1F99DF800203AB9EE
:1065A0009DF80100102803D19DF8021001290FD099
:1065B00000222D4B114602200EF0CAF8FFF7A0FE74
:1065C0004FF47A70FDF724FBFFF728FF10B010BDE1
:1065D000264B1A70587099709DF80310D9709DF869
:1065E000041019719DF8051059719DF806109971E4
:1065F0009DF80710D9719DF8081019729DF80910BF
:1066000059729DF80A1099729DF80B1001F03F0124
:10661000D972D87AD1B288421BD89DF8282083F845
:1066200028209DF8292083F829209DF82A2083F826
:106630002A209DF82B2083F82B200DF12B0100221E
:106640009818013211F8014F80F82C40142AF7D124
:10665000BAE701F140006844194410F8340C08739B
:106660000132D6E700F80308756B030858030020D1
:10667000F0B50C238BB0052600240125CDE9056378
:1066800018221023CDE9033221466D4B0294224695
:106690000327CDE90055022009940EF059F8694B03
:1066A000029422462146CDE9005702200EF050F810
:1066B000CDE901640226644B00962246214630460D
:1066C0000EF046F8614B009522462146CDE9017453
:1066D00030460EF03DF809A9204606F013F9099B53
:1066E000C3F307220292C3F307421B0E01920093E9
:1066F0002246574B214630460EF02AF809A9284673
:1067000006F000F9099BDAB20392C3F30722029262
:10671000C3F307421B0E0192009322464D4B2146C4
:1067200030460EF015F84C4B4C48009422464FF47E
:10673000FA710EF0DBFA4A4B4A48009422464FF4B5
:10674000FA710EF0D3FA484B484800942A464FF4A9
:10675000FA710EF0CBFA464B464800942A464FF4A5
:10676000FA710EF0C3FA2046FCF7C4FA08B1FCF740
:10677000E5FC414B009400224FF4FA613F480EF0D3
:10678000B5FA3F4A002101200EF0B0F93D4A002140
:1067900002200EF0ABF93C4A002104200EF0A6F9CD
:1067A0003A4A002108200EF0A1F900F019FE3849FC
:1067B000384806F05DF8384805F04AFF2B480EF0DF
:1067C00041FB364B0021187805F09AFC34490094BF
:1067D000344B0968344800220EF088FA32480EF033
:1067E00031FBFFF7CDFE314A002110200EF07EF97B
:1067F0002F4A002120200EF079F92E4A0021402056
:106800000EF074F92C4A002180200EF06FF92B4B0A
:106810002B4819682B4B009401220EF067FA284888
:106820000EF010FB284B29481968294B00940122CF
:106830000EF05CFA25480EF005FB0BB0F0BD00BF72
:10684000B56B0308F56B0308166C0308376C030877
:10685000586C0308796C03089F5900086C1F0020CE
:1068600015610008541F0020256000083C1F00200F
:10687000C9600008241F00200D6000087820002057
:1068800055C40008395C000899600008C15B000825
:106890000000030130010020180100207C010020CD
:1068A00014010020E159000890200020E553000861
:1068B00061540008B954000839550008A0030020AD
:1068C0000C1F0020DD5F00089C030020F41E002048
:1068D000855F000873B50D4D00262E60FEF7CEFFD4
:1068E000C820FDF795F928683146FBF74FFD0446AF
:1068F0000028F3D12868FBF791FD054B0090224654
:10690000214601200DF024FF02B070BDAC1E002016
:106910009D6C030830B50024A5B07C22214605A853
:10692000049427F075FD53238DF8103001254FF4A2
:106930008873ADF81230ADF800408DF81450FDF7B3
:10694000E5F8FE23B0FBF3F000EB400000EB401055
:106950003A4B8DF815002246214603200DF0F8FE33
:106960006846FEF7DFFF9DF800309DF801201343D5
:1069700014D158238DF81630072480220021304886
:1069800027F046FD224604A92D4827F0D7FD2C4AC2
:1069900021460120FFF734FC25B030BD0E232946E7
:1069A00001A8CDE901448DF81630ADF80C40FEF792
:1069B0008FFF01AB03CB234C1B88CDF81B10ADF828
:1069C0001F30CDF81700FEF759FF2068FBF74CFD8C
:1069D0000A254FF47A7380B2B0FBF3F0B0FBF5F305
:1069E00005FB130030308DF821002068FBF73CFDDB
:1069F000642380B2B0FBF3F0B0FBF5F305FB1300AA
:106A000030308DF822002068FBF72EFD80B2B0FBFD
:106A1000F5F0B0FBF5F305FB130030308DF82300E3
:106A20002068FBF721FD80B2B0FBF5F305FB1300F6
:106A300030308DF8240015249FE700BFD06C030888
:106A4000A8200020AC1E00202DE9F047044694B099
:106A5000BD480D46802200210DF08AFF2378592B76
:106A600040F04082052D5ED86378443B162B5AD8FF
:106A7000DFE813F07C015900590159006101590008
:106A8000590059005900BD005900440159005900EE
:106A90005900D70159005900E70059005900590021
:106AA0001700A678482E17D1A84A14210120FFF715
:106AB000A7FB41F28830FDF7ABF80022A44B11464A
:106AC00003200DF045FE40F6B830FDF7A1F814B0F4
:106AD000BDE8F047FFF7B2BA532E0DD1FFF71AFF0A
:106AE00041F28830FDF794F8974A1521012014B03F
:106AF000BDE8F047FFF784BB432E17D1002404A85C
:106B00008DF8104005F01CFD8F4A4C2313701023A4
:106B100093709DF81030547001204133D070137180
:106B20000521FFF76DFB14B0BDE8F087442EFAD1C4
:106B3000854C884DA670592323705A236370FFF744
:106B4000C9FE2868FBF76AFC0022834B00901146BF
:106B500003200DF0FDFD7F220021601C27F058FC72
:106B6000102326700126A370E6702671FCF7CEFF75
:106B7000FE23B0FBF3F000EB4000042300EB4010D9
:106B80006071A3712868FBF76FFC0A274FF47A73D2
:106B900080B2B0FBF3F0B0FBF7F307FB130030302B
:106BA000E0712868FBF760FC642380B2B0FBF3F06F
:106BB000B0FBF7F307FB1300303020722868FBF7B7
:106BC00053FC80B2B0FBF7F0B0FBF7F307FB130008
:106BD000303060722868FBF747FC80B2B0FBF7F3F7
:106BE00007FB13003030A07222460B217EE7A3780A
:106BF000303BDBB2092B96D8584C594A2370237886
:106C0000DBB25372504A592313704D2353702378CB
:106C10000321303301209370FFF7F2FA23780093B9
:106C20000022504B114601200DF092FDFFF768FB4A
:106C300023780BB1FCF7DCFC14B0BDE8F047FCF79F
:106C40007BBDA578482D1BD13F4C562323701023C4
:106C5000A37018236371052301200025A371224628
:106C60000C230821E3716570E0702071FFF7C8FA0A
:106C70003D4B00942A46114602200DF069FD52E773
:106C8000432D7FF450AF00213C2205A82E4C0491E7
:106C900027F0BEFB04A8FFF7ADFB9DF81030637032
:106CA0009DF81130A3709DF81230E3709DF81330F9
:106CB00023719DF8143063719DF81530A3719DF810
:106CC0001630E3719DF81730257023729DF81B5024
:106CD0009DF8183063729DF81930A3722A469DF80A
:106CE0001A30E37207A904F10D00257327F026FC82
:106CF00005F10D012246C9B2012012E7A07839281A
:106D00000CD83038C0B2FEF72BFE0F4A2378137030
:106D100063785370A37893700321E7E614B0BDE85D
:106D2000F047FFF7DFBAA0783928F7D83038C0B27B
:106D3000FEF71BFEE9E7A0783928EFD83038C0B25B
:106D4000FEF718FEE1E700BFA8200020E96C030869
:106D5000FE6C0308AC1E0020206D0308F01E00200E
:106D600058030020436D03086C6D0308A378303B83
:106D7000DAB2092AD2D8E578303DEAB2092ACDD86C
:106D80002179A1F14802D2B20B2AC7D87A4840FA39
:106D900002F2D007C2D40A224D2902FB03553BD18F
:106DA0003C235D43754B4FF47A7068431860744B15
:106DB0001860FEF739FE734A2378137063785370B6
:106DC000A3789370E378D3700521237913710120A0
:106DD000FFF716FA6C4B002610221E705A70012223
:106DE0009A70DA70A178303901EB8100E17830399E
:106DF00001EB4001C9B2197122795A71634A1278C4
:106E0000D2B21A72624A1278D2B25A72FFF778FA84
:106E1000604B009532462EE74829C3D14FF4616399
:106E2000BFE7A378303BDAB2092A3FF677AFE578BF
:106E3000303DEAB2092A3FF671AF2179A1F148024B
:106E4000D2B20B2A3FF66AAF4B4840FA02F2D207A1
:106E50003FF564AF0A224D2902FB03553DD13C2387
:106E60005D43474B4FF47A7606FB05F21A601868CB
:106E7000FEF704FE434A2378137063785370A378B7
:106E80009370E378D3700521237913710120FFF704
:106E9000B7F93D4B002710221F705A7001229A70DB
:106EA000DA70A178303901EB8102E178303901EBF9
:106EB0004201C9B299712279DA71344A1278D2B298
:106EC0001A72334A1278D2B25A72FFF719FAB5FB26
:106ED000F6F5314B00953A46CDE64829C1D14FF43D
:106EE0006163BDE7502B40F0A881022D7FF61BAEF9
:106EF0006178A1F13003012B3FF615AEA378312B59
:106F00007FF411AE052D4FD1E378302B40F0C480D3
:106F10001E4D224E00232B702B7803F0FF0253B935
:106F20002379303BDBB233703378009311461C4B2E
:106F300002200DF00DFC16491A4A00230B7033781D
:106F4000DBB213702B78104ADBB213720B78DBB212
:106F50005372FFF7D5F90B4B22781A7062785A708A
:106F6000A2789A70E278DA7022791A71FCF7E4FB61
:106F70000521044ABAE500BFDEF7FFFF1401002037
:106F80009C030020A82000205803002006010020B8
:106F9000F01E0020966D0308CD6D0308040000204C
:106FA000176E030805000020082D69D1E378462BF1
:106FB00040F0EC802579A5F13000C0B2092800F23C
:106FC0003A816179A1F13003092B00F23481A27971
:106FD000A2F13003092B00F22E81E379A3F13006F0
:106FE000092E00F2288105EB85067600B04D20368B
:106FF00001EB8101F6B249002E702031AD4E263AE8
:10700000C9B2D2B2317002EB8202AB4903EB830307
:1070100052005B000A802033A84ADBB21370A84AF2
:1070200082F828006379303BDBB282F82930A379FB
:10703000263BDBB282F82A30E379303BDBB282F8C0
:107040002B302B782BB9337803F0FF020BB99D4B13
:107050001A70FFF755F99C4B22781A7062785A70B3
:10706000A2789A70E278DA7022791A7162795A718C
:10707000A2799A71E279DA71FCF75EFB082178E770
:10708000042D2FD1E278A2F13003DBB2092B11D904
:10709000A2F14103192B0AD9FFF724F900228B4BE7
:1070A0001146012014B0BDE8F0470DF051BBA2F12C
:1070B0003703DBB286480370834B20785970312147
:1070C00018709970DA70824B7D4A1B78DBB21372AC
:1070D000804B1B78DBB25372FFF712F9FCF72CFBE5
:1070E000042146E71D2D4FD9A61C0025DFF8D091BD
:1070F000DFF8E4A13746A84617F8012F303AD2B29C
:10710000092A3ED809EB050303201A731B7BCDE93E
:1071100002533B780022CDE90053114653460DF04F
:1071200017FB01351E2DE7D1B8F1000FB4D1FEF7E2
:107130001BFA654B50221A7000225A7010229A7066
:107140000122DA7003F8042F203416F8012F03F817
:10715000012FB442F9D15A4B00221A7010225A70F2
:1071600001229A70DA705A4A1278D2B21A72594AC7
:107170001278D2B25A721E22DA72FFF7C1F82321B6
:10718000F7E64FF00108CCE7072D85D900254C4FD5
:10719000DFF8448102342E4614F8012F303AD2B27F
:1071A000092A46D8791903200A730B7BCDE90253CB
:1071B00023780022CDE90053114643460DF0C8FA6A
:1071C0000135082DE8D1002E7FF466AFFEF73EFAB8
:1071D0003D4B3B4C50221A7010229A700025012220
:1071E0005D70DA7003F8042F62190135127B082DE7
:1071F00002F1300203F8012FF6D10022502311468C
:1072000000930120354B0DF0A3FA002323701023C7
:1072100063700123A370E3702D4B1B78DBB22372E4
:107220002C4B1B78DBB26372E572FFF769F80D2116
:107230009FE60126C4E700219BE6412B7FF473AC57
:107240006378432B7FF46FAC162D7FF46CAC244D28
:10725000621C002312F8011FE9540133142BF9D1E9
:10726000FEF790F81F4B5B7D012B1DD114490023C5
:10727000EA5CC8180133D2B2142B80F82C20F7D165
:10728000144B00221A701B78DBB24B72FFF738F8F0
:107290000D4A631E153413F8011F02F8011B9C42AE
:1072A000F9D1094A162121E40A4B02221A70EFE7AC
:1072B000A7030020A60300203C000020A503002017
:1072C00058030020A4030020A8200020766E0308A5
:1072D00006010020F01E0020336E03085B6E0308D9
:1072E0002E210020AC09002070B5054688B00C4660
:1072F000002951D033480DF0A5FD26789EB3002D0E
:107300005ED068682E7870B3032E0BD0132E45D054
:10731000022E28D16978012925D00B0623D4FFF746
:1073200093FB20E06B78012B07D10078012802D075
:10733000022800D008B905F0BDF800250DF11F00A6
:107340008DF81F5005F0FCF81F4A4C2313701023D2
:1073500093709DF81F305570012041330521D07086
:107360001371FEF74DFF237C052B15D894F90A20E5
:10737000059294F909200492144A52F82330039399
:1073800094F90830CDE901630022E36800931146C7
:107390000F4B03200DF0DCF908B070BD6B78012BAA
:1073A000E1D102780B4B02F001021A702AB90A4BA4
:1073B000114603200DF0CCF9D5E7084B0022F7E782
:1073C0002E46D0E7541F0020A8200020006F03089D
:1073D000AE6E0308841F00209B6E0308A56E030891
:1073E000034B0022C3E902220122C3E900227047B5
:1073F0004421002000487047442100204FF0B04352
:1074000082B0DA6C0243DA64DB6C03400193019BC7
:1074100002B070472DE9F04186B000240220154DDE
:107420000594FFF7EBFF0420FFF7E8FF124F0394EA
:107430004FF4807601230DEB0001CDE9016328466E
:10744000032304934FF4005801F04AF801A9384689
:10745000CDF8048001F044F822464146384601F058
:1074600065F928462246314601F060F9204606B00B
:10747000BDE8F0810004004800080048032810B56A
:107480000ED8012810D868B902460B484FF4807115
:1074900001F04CF9002209484FF4005101F046F97F
:1074A000002010BD0122F0E7002203484FF4807154
:1074B00001F03CF90122EEE7000400480008004812
:1074C000022070470020704701207047002814BF39
:1074D00016200F20704700000D48854600F025F863
:1074E0000C480D490D4A002302E0D458C45004331F
:1074F000C4188C42F9D30A4A0A4C002301E01360F5
:107500000432A242FBD326F0EBFFFBF7F9FDFEE7C6
:107510000000012000000020C8070020E0D403087C
:10752000C8070020E0400020FEE7704710B50320A8
:1075300000F06EFC01F07CFA064B18600F20FCF79F
:107540005DFB044618B9FBF751FF204610BD01242E
:10755000FBE700BFA80300204FF0E022136923F0EF
:107560000203136170474FF0E022136943F00203F6
:1075700013617047014BD3F8900570470070FF1FEF
:10758000014BD3F8940570470070FF1F014BD3F8EF
:10759000980570470070FF1F024A536843F00103CB
:1075A00053607047002004E0024A536843F002032E
:1075B00053607047002004E0024A536843F004031C
:1075C00053607047002004E08068C0F3800070477B
:1075D000F7B5002301930446002800F0E980856D8B
:1075E00025B9FBF717FAE56584F8545023689A68C3
:1075F000D00040F1A1809A68D10000F1B480A26D62
:1076000042F01002A265E26D42F00102E26501253E
:107610001846FFF7D9FFA26D02F01002024340F0B6
:10762000C980A26D206922F4817242F00202A26533
:107630009A68D2075DD4226BA67E94F82CC0003ADB
:1076400018BF01221703D4E902120A43217E42EA3D
:107650008132617E42EAC13242EA4632002842EA81
:107660004C02B4BF20F000414FF400113A430A43EA
:1076700094F82010012903D1002E76D142F48032F3
:10768000616A21B1A66A01F4E07131430A43D96805
:10769000E66C21F4FE3121F4FF711143D96094F8B6
:1076A0003C206168012A01F0404C4CEA060609D1F1
:1076B000D4E910273A433243A66C324342EA0C0223
:1076C00042F001061F693E4A3A4032431A6121F0F6
:1076D0000042B2F1804F0CD0B1F1004F09D0394EC9
:1076E000D6F8082701F4701122F470120A43C6F884
:1076F00008275A69666BA16B22F0070232435A6170
:107700005A6922F0700242EA01125A61002835D10A
:107710009A6A62F00F029A625B6903F007039E4265
:107720003CD10023E365A36D23F0030343F0010381
:10773000A365284603B0F0BD9A68234922F01042A1
:1077400022F0170242F080529A60204A1268B2FB7F
:10775000F1F2013252000192019A002A3FF44BAF3C
:10776000019A013AF7E7002552E7A16D41F02001A7
:10777000A165E16D41F00101E16581E7B0F5001F10
:10778000CAD19A6AE269013A92006FF00F0102F0E1
:107790001C0201FA02F2216E0A43BCE7A36D23F03A
:1077A000120343F01003A365E36D43F00103E365A7
:1077B0000125BEE7A36D43F01003A365F8E700BF02
:1077C00002FCFF1F00200140400D0300A803002021
:1077D000F8B54569082D04460E460AD00368DB68F3
:1077E000D80705D5A36D43F02003A3650120F8BD9C
:1077F0000425FCF705FA074623681A682A4220D0B8
:10780000A26D42F40072A265DA6812F4406F14D1DE
:10781000A27E92B91A6812070FD51846FFF7D4FE58
:1078200020BB5A6822F00C025A60A26D22F48072CA
:1078300022F0010242F00102A265227EFAB100208C
:10784000D5E7711CD9D0FCF7DBF9C01BB04201D8D9
:10785000002ED1D123681B682B40CDD1A26D84F8B6
:10786000543042F00402A2650320C0E7A26D42F04A
:107870002002A265E26D42F00102E265DDE70C2222
:107880001A60DCE70368186C70470000F7B5002346
:10789000019390F85430012B044600F0C080056835
:1078A0000269012380F854302846FFF78DFE002836
:1078B00040F0AF80D1E90030022822F004027ED0EF
:1078C000B2F1004FC3F3110E35D1AA6A42EA0E029B
:1078D000AA628A68686902EA032222F07C4222F0E6
:1078E000FF0220EA03210A43002B6A611DDA4D4A98
:1078F0004D4DD2F80817AB4201F0E07043D10D02B4
:1079000013D4D2F8083723F0E073034343F40003A1
:10791000C2F80837454B1A68454BB2FBF3F20C230B
:1079200002FB03330193019B53BB0020002384F827
:10793000543003B0F0BD226E00F01F074FF00F0C63
:107940000CFA07FC6FEA0C0622EA0C0CBEF1000FE1
:1079500011D1C3F38462BA4042EA0C022266800865
:10796000E26901309042B4D8A86AC3F38362BA4096
:1079700006403243ACE793FAA3F2B2FA82F2EAE7A6
:10798000019B013BCEE72B4DAB420BD1C901CCD4BF
:10799000D2F8083723F0E073034343F08073C2F852
:1079A0000837C2E7244DAB42BFD14B02BDD4D2F859
:1079B000083723F0E073034343F48003EFE7B2F1A9
:1079C000004F01BFAA6AC3F311018A43AA62002BC8
:1079D000ABDA154813498342D1F8082709D1D1F809
:1079E000083702F0A07223F0E0731A43C1F80827A9
:1079F0009BE71048834204D1D1F8083702F44002D3
:107A0000F1E70D48834290D1D1F8083702F0C072F7
:107A1000E9E7A26D42F02002A265184686E702203F
:107A200087E700BF00200140001000B0A80300203D
:107A3000400D0300004000B8002000B4026838B5D3
:107A400004461046FFF7C0FD08B9002038BD936812
:107A5000990707D4936823F0004323F0170343F0FA
:107A600010039360FCF7CCF8054623689B685B071E
:107A7000EBD5FCF7C5F8401B0228F6D923689B68B4
:107A80005A07F2D5A36D43F01003A365E36D43F0ED
:107A90000103E3650120D9E773B500230268019370
:107AA0009368DD07044602D5002002B070BD9168DE
:107AB000214B194209D0A36D43F01003A365E36D78
:107AC00043F00103E3650120EFE7936823F00043EF
:107AD00023F0170343F001039360184BD3F80837E2
:107AE00018021CD4637E012BDED0FCF789F8144EFB
:107AF000054622681368DB07D6D49368D9075FBFB1
:107B00009368334043F001039360FCF779F8401B1E
:107B10000228EED923681B68DA07EAD4CBE7094BC1
:107B2000094A1B68B3FBF2F301330193019B002B5D
:107B3000D8D0019B013BF8E71700008000200140EE
:107B4000E8FFFF7FA8030020400D030038B504467E
:107B50000068FFF739FD054620BB94F85430012B2F
:107B600020D0012384F854302046FFF795FFB0B9A8
:107B7000A36D226823F4706323F0010343F4807340
:107B8000A3651C23E065136084F85400936823F018
:107B9000004323F0170343F00403936038BD84F8D7
:107BA0005450FBE70220F9E7026838B59368916802
:107BB0000446C80701D4002038BD9907FBD4936858
:107BC00003F00503012B19D1936823F0004323F040
:107BD000170343F00203936003231360FCF710F8CC
:107BE000054623689B68DB07E5D5FCF709F8401BD1
:107BF0000228F6D923689B68DA07F2D5A36D43F013
:107C00001003A365E36D43F00103E3650120D3E7AF
:107C100070B5044600284BD0836D43F002038365A2
:107C2000FFF70CFF054668B92046FFF7BDFF054684
:107C300008B90123A3652268936823F0104323F059
:107C40001703936023685A6822F4677222F00302D4
:107C50005A6040F29F321A60D968164A0A40DA60C8
:107C60001A6922F040421A615A6922F007025A61E9
:107C70001A6A02F0F0221A625A6A02F0F0225A627C
:107C8000DA6A02F0F022DA629A6A0B4A00269E62F1
:107C9000D2F8083723F0FE73C2F808372046FAF707
:107CA000CDFEE6652666A66584F85460284670BD5C
:107CB0000125FBE700023E830020014010B590F84B
:107CC0005430012B044615D0012380F85430FFF7BF
:107CD000B5FE58B92046FFF767FF38B9A36D23F406
:107CE000807323F0010343F00103A365002384F8AC
:107CF000543010BD0220FCE7F7B50023019390F843
:107D00005430012B04467FD0012380F85430FFF714
:107D10004BFF23689A6812F00102054607D0A36D55
:107D200043F01003A365002384F854302DE0A16DC7
:107D3000364F21F4817141F00201A165DE68D968F6
:107D400026F4FF4626F07C0621F40041360421F09B
:107D50000301360CD96008209968394041F0004190
:107D600099609968002913DA01990131019101990B
:107D7000B1F52E3FF5D3A36D23F0120343F01003AA
:107D8000A365002384F854300125284603B0F0BDD4
:107D9000D3F8B410013801F07F010A44DCD19968AE
:107DA0001A48014041F001019960D3F8B41021F064
:107DB0007F0141EAD202C3F8B4209A68024042F03F
:107DC00002029A60FBF71CFF074623689A68D207F5
:107DD00008D4DA683243DA60A36D23F0030343F07A
:107DE00001039FE7FBF70CFFC01B0228EDD92368B6
:107DF0009B68D907E9D5A36D43F01003A365E36D34
:107E000043F00103E365BFE70225BEE7E8FFFF7F1C
:107E10000749CA6822F4E0620302120403F4E06333
:107E2000120C134343F0BF6343F40033CB6070473D
:107E300000ED00E0164B30B5DC68C4F30224C4F159
:107E40000703251D042B28BF0423062D4FF0FF3503
:107E50008CBF033C002405FA03F321EA0303A54089
:107E600022EA0502A340002843EA0203ACBF00F166
:107E70006040084A4FEA0313B8BF00F00F00DBB2BE
:107E8000AABF00F56140135480F8003330BD00BF35
:107E900000ED00E014ED00E0002807DB044A410992
:107EA000012300F01F00834042F82130704700BFDB
:107EB00000E100E000280CDB4309064900F01F0048
:107EC00020330122824041F82320BFF34F8FBFF3BC
:107ED0006F8F704700E100E070B5D0E91345656031
:107EE000446D14B1D0E916456560D0E9105404F032
:107EF0001C060124B4406C60046863608368102B26
:107F00000BBFA260A160E160E26070BD0268416CDD
:107F1000D3B210B5083B1424B3FBF4F30B4CA242CC
:107F200088BF0B4A21F0030199BF01F1804202F59D
:107F30000232521807338264064AC26403F01F03F8
:107F4000012202FA03F3036510BD00BF07040240DB
:107F50001C0802408008024038B500285CD0026846
:107F60002E4B9A424FF014014AD82D4B1344B3FBC9
:107F7000F1F32C499B00C0E91013022380F825304F
:107F80001368056923F4FF4323F070031360D0E9FD
:107F9000024323432B43456911682B4385692B43D7
:107FA000C5692B43056A2B430B431360FFF7AEFFF4
:107FB000B4F5804F04BF002343604368816C03F035
:107FC0007F020A60D0E91314013B032B4C601ED8DA
:107FD000154B1649816513449B000121013A01FAB2
:107FE00002F200214365C2651960114B5A640023F7
:107FF0000122C36380F8243080F82520184638BD5C
:108000000C4B1344B3FBF1F30B499B00B3E7002384
:10801000C0E91533C365EAE70120F0E70704024031
:10802000F8FFFDBF000002403F82001040090240FF
:1080300000090240F8FBFDBF0004024038B50028EB
:1080400041D00268136823F0010313601F4B9A426A
:108050004FF0140130D81E4B1344B3FBF1F31D490C
:108060009B00C0E91013012403F01C0304FA03F37E
:10807000002515604B60FFF749FF836C41681D6068
:10808000D0E913325A604A1E032A06D8124B0B4419
:108090009B0094401D60114B5C640023C363C0E9E6
:1080A0001533C0E90B33C0E90D33C36580F82530C3
:1080B00080F82430184638BD094B1344B3FBF1F364
:1080C00008499B00CDE70120F5E700BF0704024007
:1080D000F8FFFDBF000002403F820010000902408F
:1080E000F8FBFDBF0004024070B590F82450012D4C
:1080F00004463BD090F825600125AE4280F824501C
:108100004FF000062CD1022580F825500568C66383
:108110002E6826F001062E60FFF7DEFE036BBBB172
:108120002B6843F00E032B60A36C1A68D20342BF86
:108130001A6842F480721A60636D1BB11A6842F4C7
:1081400080721A602B6843F001032B60002070BD21
:108150002B6823F004032B602B6843F00A03E2E74B
:108160008023C36380F824602846F0E70220EEE70E
:10817000034640B190F82520022A06D00422C263AB
:10818000002280F82420012070470268806C11686A
:1081900021F00E011160016821F480710160116805
:1081A00021F001011160D3E9100202F01C0101224B
:1081B0008A404260D3E9132151605A6D32B111688F
:1081C00021F480711160D3E9162151600122002051
:1081D00083F8252083F82400704708B590F82530EF
:1081E000022B03D00423C363012008BD03681A686F
:1081F00022F00E021A601A6822F001021A60826CE4
:10820000136823F480731360D0E9101303F01C0289
:10821000012393404B60D0E913325A60436D33B170
:108220001A6822F480721A60D0E916325A6001236B
:1082300080F82530002380F82430836B03B1984701
:108240000020D2E770B4426C046C036826681D6895
:1082500002F01C020421914031420FD015F0040FAE
:108260000CD01A6892065EBF1A6822F004021A60E7
:10827000036B6160002B33D070BC18470221914022
:10828000314217D015F0020F14D01A68940606D4A4
:108290001A6822F00A021A60012280F82520114A89
:1082A00093428CBF104B114B5960002380F824304F
:1082B000C36ADFE708219140314211D029070FD569
:1082C000196821F00E011960012303FA02F26260BD
:1082D000C36380F82530002380F82430436BC9E75E
:1082E00070BC704780000240000402400000024061
:1082F0000A4A536943F4802330B55361EFF3108485
:1083000072B60023CD58C5500433B3F5807FF9D140
:108310001369DB03FCD484F3108830BD004000589F
:10832000064B5A69002ABFBF054A9A6002F188329B
:108330009A60BABF5869C00F0020704700400058CB
:1083400023016745044B5A6942F000425A6158695B
:10835000C043C00F704700BF0040005870B50546CD
:10836000FBF74EFC124E04463369D90313D433692C
:10837000DA0744BF012232614CF2FA32134011D1C4
:108380000B4E306910F480200BD0FBF739FC001B3A
:10839000A842F6D304E0FBF733FC001BA842E3D36A
:1083A000032070BD024A1361024A01205360F8E7BE
:1083B00000400058542100202DE9F041184D984606
:1083C0002B78012B06460C46174626D001232B702E
:1083D0004FF47A7000236B60FFF7C0FFA0B9012E45
:1083E00016D1104A536943F0010353612760BFF36C
:1083F0006F8FC4F804804FF47A70FFF7AFFF094A1B
:10840000536923EA0603536100232B70BDE8F08112
:1084100039462046FFF76CFFEDE70220F6E700BF84
:108420005421002000400058054A536923F47E730C
:1084300043EAC00040F4803040F0020050617047D1
:10844000004000582DE9F041234F3B78012B0546B1
:1084500088463FD001233B704FF47A7000237B6045
:10846000FFF77CFF044688B92B68042B13D11B4A05
:10847000536943F4803343F0040353614FF47A703B
:10848000FFF76CFF0446154B1A681B6800233B700E
:108490002046BDE8F0814FF0FF33C8F800306E6829
:1084A000D5E901321344B3420AD93046FFF7BCFF85
:1084B0004FF47A70FFF752FF50B1C8F800600446DD
:1084C000064A536923F47E7323F002035361DAE70B
:1084D0000136E5E70224DBE7542100200040005884
:1084E0002DE9F04F524C00234FF00F090A6832FA81
:1084F00003F501D1BDE8F08F012505FA03F818EA6C
:10850000020200F08E804E68032706F003054FEA52
:10851000430E07FA0EFC6F1E012F6FEA0C0C32D8C7
:10852000876807EA0C0ACF6807FA0EF747EA0A07D6
:108530008760476827EA0808C6F300179F4047EAA4
:1085400008074760C76807EA0C088F6807FA0EF744
:1085500047EA0807022DC76017D14FEAD30800EB9E
:10856000880803F0070AD8F820704FEA8A0A09FA47
:108570000AFB27EA0B0B0F6907FA0AF747EA0B0712
:10858000C8F8207001E0032DDCD1076805FA0EF56C
:1085900007EA0C073D4316F4403F056041D023F045
:1085A000030707F1804707F5803703F0030CBD6828
:1085B0004FEA8C0C4FF0070E0EFA0CFEB0F1904F04
:1085C00025EA0E0E2FD01B4DA8422ED005F5806552
:1085D000A84214BF0725022505FA0CF545EA0E0549
:1085E000BD602568D74316F4801F0CBF3D4015437E
:1085F0002560656816F4001F0CBF3D40154365609B
:10860000D4F8805016F4803F0CBF3D401543C4F8A9
:108610008050D4F88450B60354BF3D401543C4F88D
:108620008450013362E70025D6E70125D4E700BF77
:108630000008005800040048374A2DE9F04F002395
:108640004FF0010A4FF0070B4FF00F0931FA03F416
:1086500001D1BDE8F08F0AFA03FC1CEA010654D0F0
:1086600023F0030404F1804404F5803403F003078D
:10867000A568BF000BFA07F8B0F1904F08EA050EA5
:1086800045D0264DA84244D005F58065A8420CBFD0
:1086900002250725BD40754517D1D2F8805025EA3F
:1086A0000605C2F88050D2F8845025EA0605C2F8C3
:1086B0008450156825EA06051560556825EA060503
:1086C0005560A56825EA0805A560056803265C00D5
:1086D00006FA04F423FA06F6254300EB8606056045
:1086E00003F00705376AAD0009FA05F527EA050723
:1086F0003762856825EA04058560456825EA0C052A
:108700004560C56825EA0404C46001339EE700257E
:10871000C0E70125BEE700BF00080058000400487C
:108720000369194214BF0120002070470AB181611A
:10873000704781627047436901EA030221EA03013D
:1087400041EA024181617047044AD168014208B59B
:1087500002D0D060FDF7E0FC08BD00BF0008005863
:10876000024A136843F48073136070470004005892
:108770000D4B10B55B690C4628B99A0507D500F07A
:1087800027F820B110BD9B0501D400F019F8074A65
:108790001369012C23F00403136101D130BFF1E709
:1087A00040BF20BF20BFEDE70004005800ED00E00F
:1087B000024B186800F4C060704700BF0004005806
:1087C000024A136843F48043136070470004005862
:1087D0000C4A136823F4804313600B4B1B6832214F
:1087E0004B430A49B3FBF1F35169890500D533B90D
:1087F000536913F4007F14BF032000207047013B2E
:10880000F2E700BF00040058A803002040420F0018
:108810000B4A136823F0070343F002031360094B6C
:108820001A69012842F004021A6105D130BF1A69A1
:1088300022F004021A61704740BF20BF20BFF6E754
:108840000004005800ED00E04FF0B0431868C0F39A
:10885000404070474FF0B0431868C0F34000704785
:108860004FF0B042536823F47F4343EA0023536040
:1088700070474FF0B0431868C0F340607047000085
:108880007FB54FF0B0432C4AD3F80831C0F3031042
:1088900003F00F0352F82040284A52F82330B4FB6B
:1088A000F3F4FFF785FF264B054693E80700B5F57F
:1088B000007F04AB03E9070010D0224B9C4218D381
:1088C00003F5B70303F67F539C4229D903F57413CC
:1088D00003F510639C4225D802230BE01A4B9C42FF
:1088E00007D91A4B9C421BD903F5370303F5D8531C
:1088F000F0E7002304AA02EB830353F80C4C144D59
:108900002B6823F0070323432B60FBF779F9064616
:108910002B6803F007039C4206D1002004B070BD11
:108920000123E7E70024EAE7FBF76AF9801B022846
:10893000EED90320F2E700BF186F0308786F030831
:10894000F8190308C0CF6A00BFEA21013F9334023F
:10895000004000584FF0B04310B59A68D96812F043
:108960000C0205D00C2A4AD101F00303012B51D18E
:108970004FF0B0412B480B6813F0080306D00B688A
:1089800013F0080337D1D1F8941007E00C682407DE
:1089900056BFD1F894300968C3F3032350F823304D
:1089A000002A0CBF184600204FF0B0418A6802F040
:1089B0000C020C2A1ED1CA6802F00302022A2ED031
:1089C000032A06D10B68184A13F4801F174B18BFEF
:1089D00013464FF0B042D068D168D268C0F3062089
:1089E0005843C1F302130133B0FBF3F0530F0133CB
:1089F000B0FBF3F010BD0B68C3F30313CEE7042AFA
:108A000005D0082A06D11B6813F4801305D0064848
:108A10000023C9E700231846C6E70448C4E7024B11
:108A2000D7E700BF186F03080024F4000048E801EE
:108A300008B5FFF78FFF4FF0B043044A9B68C3F3BC
:108A4000031352F82330B0FBF3F008BD786F03082E
:108A50002DE9F0410446002853D04FF0B0439D6803
:108A6000DE6803689B0605F00C0506F0030668D572
:108A7000026A1DB10C2D46D1012E44D1002A40D0EE
:108A80004FF0B043A16A1A68170756BFD3F8943065
:108A90001B681B0903F0F00399421FD90846FFF732
:108AA000EFFE00282DD14FF0B042136843F00803C9
:108AB00013601368A16A23F0F0030B431360606A2C
:108AC000FFF7CEFEFFF7B4FFAB4B1860AB4B186857
:108AD000FBF794F8002834D0BDE8F0814FF0B042A5
:108AE000136843F008031360136823F0F0030B438B
:108AF0001360606AFFF7B4FE0846FFF7C1FE002866
:108B0000E0D00120E8E74FF0B043002A54D01A68C3
:108B100042F001021A60FBF773F80746FFF79AFE6E
:108B2000002842D04FF0B042136843F008031360AE
:108B30001368A16A23F0F0030B431360606AFFF728
:108B40008FFE2368D80748D42368990700F18C80EA
:108B500023681E0740F1FA80A3694FF0B046002B4E
:108B600000F0E180D6F89430E16903F01002914200
:108B700000F0C48003F00302022AC2D0D80740F1FB
:108B8000B380D6F8943023F00103C6F89430FBF795
:108B900037F80746D6F89430990740F1A580FBF7DF
:108BA0002FF8C31B112BF5D904E0FBF729F8C01BE4
:108BB0000228B3D903208FE71A6822F001021A6055
:108BC000FBF71EF80746FFF745FE0028B9D0FBF774
:108BD00017F8C01B0228F6D9ECE7082D03D00C2D9E
:108BE00005D1032E03D16368002BADD189E74FF087
:108BF000B043A1681A6822F480120A431A606268BE
:108C0000B2F5803F10D11A6842F480321A60FAF748
:108C1000F7FF0746FFF718FE002895D1FAF7F0FF97
:108C2000C01B6428F6D9C5E7B2F5041F04D11A6841
:108C300042F400121A60E6E7196821F480311960E5
:108C4000196821F400111960002AE0D1FAF7D8FF61
:108C50000746FFF7F9FD00283FF476AFFAF7D0FF9B
:108C6000C01B6428F5D9A5E7042D236903D00C2D7A
:108C70000ED1022E0CD1002B3FF443AF4FF0B04287
:108C80006169536823F0FE4343EA016353605FE781
:108C90004FF0B046BBB1336843F480733360FAF7EA
:108CA000AFFF074633685A0505D4FAF7A9FFC31B7F
:108CB000022BF7D97EE77368626923F0FE4343EA2B
:108CC0000263736044E7336823F480733360FAF718
:108CD00097FF074633685B057FF53AAFFAF790FFD9
:108CE000C31B022BF6D965E74FF0B042E169D2F819
:108CF000943023F010030B43C2F894304FF0B04788
:108D0000D7F8943043F00103C7F89430FAF778FFAE
:108D10000646D7F894309A0718D4FAF771FF831BE8
:108D2000112BF6D946E7D6F8943023F00103C6F8A4
:108D30009430FAF765FF0746D6F894309B0705D5BF
:108D4000FAF75EFFC31B112BF6D933E723685807E8
:108D500054D50B4F3B68D90514D4FFF701FDFAF742
:108D60004FFF06463B68DA050CD4FAF749FF831B30
:108D7000022BF7D91EE700BFA8030020AC03002098
:108D800000040058E3684FF0B046002B58D023F0A1
:108D90008003052B02BFD6F8903043F00403C6F8D9
:108DA00090304FF0B046FAF72BFFD6F8903043F0F2
:108DB00001030746C6F8903041F28838D6F8903063
:108DC0009B0705D4FAF71CFFC31B4345F6D9F1E610
:108DD000E36823F00403812B1BD1FAF711FFD6F8C7
:108DE000903043F08003C6F8903007464FF0B0460D
:108DF00041F28838D6F89030180504D5E36A002B84
:108E00004AD1002068E6FAF7FBFEC01B4045F1D9C5
:108E1000D0E6FAF7F5FED6F8903023F08003C6F8D6
:108E2000903007464FF0B04641F28838D6F890307F
:108E30001905E3D5FAF7E4FEC01B4045F6D9B9E6BB
:108E4000FAF7DEFED6F8903023F080030746C6F826
:108E5000903041F28838D6F890301A0516D4FAF7D7
:108E6000CFFED6F8903023F00103C6F890300746C5
:108E70004FF0B04841F28836D8F890309B07BDD506
:108E8000FAF7BEFEC31BB342F6D993E6FAF7B8FE73
:108E9000C01B4045DFD98DE60C2D4ED0022B4FF084
:108EA000B0431A6822F080721A6033D1FAF7A8FE34
:108EB0000546FFF7DEFC38BBD4E90C314FF0B04279
:108EC0000B43D0682D4901400B43E16B0B43216CF0
:108ED0000B43616C0B43A16B43EA0123D36013681E
:108EE00043F080731360D36843F08053D360FAF784
:108EF00087FE0446FFF7BDFC002882D1FAF780FE0A
:108F0000001B0A28F6D955E6FAF77AFE401B0A2814
:108F1000CFD94FE6FAF774FE0446FFF7AAFC30B942
:108F20004FF0B042164BD1680B40D36069E7FAF7B7
:108F300067FE001B0A28F0D93CE6012B3FF4E1ADA7
:108F40004FF0B043D868236B00F003029A427FF4DD
:108F5000D8AD626B00F0700393427FF4D2ADA26B88
:108F600000F4FE43B3EB022F7FF4CBAD636C00F053
:108F70006040C01A18BF0120AEE500BF8C80C1114F
:108F8000FCFFFEEE2DE9F0410D46044610B901202C
:108F9000BDE8F081684E336803F007038B4216D3B7
:108FA00023689A0727D54FF0B047A268BB6823F023
:108FB000F0031343BB60FAF723FE0646BB68DB03EE
:108FC00019D4FAF71DFE831B022BF7D911E0336881
:108FD00023F007030B433360FAF712FE07463368AA
:108FE00003F00703AB42DBD0FAF70AFEC01B0228EE
:108FF000F5D90320CCE72368580617D54FF0B047C2
:109000006269D7F8083123F00F0343EA1213C7F857
:109010000831FAF7F5FD0646D7F80831D90305D42B
:10902000FAF7EEFD831B022BF6D9E2E723685A0715
:1090300013D54FF0B047E268BB6823F4E0631343F5
:10904000BB60FAF7DDFD0646BB689B0305D4FAF763
:10905000D7FD831B022BF7D9CBE72368180714D55C
:109060004FF0B0472269BB6823F4605343EAC20360
:10907000BB60FAF7C5FD0646BB68590305D4FAF78D
:10908000BFFD831B022BF7D9B3E72368DA070FD4A0
:10909000294C236803F00703AB4239D8FFF7C8FC1B
:1090A000264B1860264BBDE8F0411868FAF7A6BDBC
:1090B0006268022A1DD1FFF7C7FB00283FF467AFA3
:1090C0004FF0B04641F28838B36823F003031343EE
:1090D000B360FAF795FD0746B368626803F00C03C6
:1090E000B3EB820FD4D0FAF78BFDC01B4045F3D908
:1090F0007FE7032A02D1FFF7BCFBDEE712B9FFF7D7
:10910000A9FBDAE74FF0B0431B685B05D8D43EE714
:10911000236823F007032B432360FAF771FD06460B
:10912000236803F00703AB42B8D0FAF769FD801B50
:109130000228F5D95DE700BF00400058A8030020D1
:10914000AC03002008B5FFF773FC4FF0B043044AAE
:109150009B68C3F3022352F82330D84008BD00BFF8
:10916000586F030808B5FFF763FC4FF0B043044A9B
:109170009B68C3F3C22352F82330D84008BD00BF18
:10918000586F03084FF0B043D3F89000C0F340008D
:1091900070474FF0B0410209D1F8883002F47F22C5
:1091A000000123EA020300F47F200343C1F8883062
:1091B00070474FF0B041020CD1F88830120423EA16
:1091C000020343EA0040C1F8880070470368DA03ED
:1091D00070B5044639D5FFF7C3FAFAF711FD614EB1
:1091E00005463368DB0532D54FF0B043616BD3F8E9
:1091F000902002F4407291421DD0D3F89010D3F821
:10920000902042F48032C3F89020D3F8902021F4CB
:10921000407022F480328D07C3F89020C3F890008C
:1092200009D5FAF7EDFC41F288360546FFF7AAFFAB
:10923000012840F090804FF0B042616BD2F890303E
:1092400023F440730B43C2F89030002605E0FAF790
:10925000D7FC401B0228C4D903262568E8070AD595
:109260004FF0B0416268D1F8883023EA124392B2DD
:109270001343C1F88830A9070AD54FF0B041A2685E
:10928000D1F8883023EA124392B21343C1F88830F0
:10929000AA0609D54FF0B0422169D2F8883023F4EC
:1092A00040630B43C2F88830AB0502D5206AFFF754
:1092B00080FF680502D5606AFFF77BFF290502D5AC
:1092C000A06AFFF776FF6A0602D56069FFF761FFC3
:1092D0002B0602D5A069FFF75CFFE80502D5E0691F
:1092E000FFF757FFE90610D54FF0B042E168D2F81A
:1092F000883023F440730B43C2F88830B1F5807F87
:1093000002BFD36843F08073D3602A040ED54FF0B8
:10931000B042216BD2F8883023F040430B43C2F8AF
:10932000883019B9D36843F08073D3606B0410D5CB
:109330004FF0B042E16AD2F8883023F040530B433B
:10934000B1F1005FC2F8883003D1D36843F48033B1
:10935000D360304670BDFAF753FC401BB0427FF635
:1093600065AF79E70004005830B590F82C30012B38
:1093700002464FF0020022D0174B82F82D00CA247B
:10938000012582F82C505C6253245C62B1F5807F29
:10939000146B996914D121F488519961596C24F0A6
:1093A000010421F0004159641463DD650A4BFF217B
:1093B00059620020012382F82D3082F82C0030BD44
:1093C00021F408519961D96C24F0020421F0004184
:1093D000D9641463D865E9E70028004070B50B4EE6
:1093E000036B756D1D40EA07044603D50123F36541
:1093F000FAF77BFEAB0704D50223F365204600F0A5
:10940000C9F9012384F82D3070BD00BF0028004049
:1094100038B50A4CE36823F02003E360FAF7F0FB69
:109420000546E3689B0601D5002038BDFAF7E8FB46
:10943000401BB0F57A7FF4D90320F6E700280040FE
:10944000F8B5114DEC6814F0400406461AD1EB68EB
:1094500043F08003EB60FAF7D3FB23460746EC6842
:1094600014F0400401D1032B01D11846F8BDFAF7DE
:10947000C7FBC01BB0F57A7F234684BF032386F861
:109480002D30ECE70023F0E70028004038B50F4C02
:10949000E36823F08003E360A3699B06054606D4D6
:1094A000FFF7B6FF10B1032085F82D0038BDA36982
:1094B00023F02003A361FFF7ABFF10B1032085F871
:1094C0002D00A36943F02003A361EFE700280040CB
:1094D00038B5044600284BD090F82D3003F0FF0239
:1094E0001BB980F82C20F9F765FE0223214D84F882
:1094F0002D30EB68DB0636D4CA236B6253236B62D4
:109500002046FFF79DFF10B1FF236B6238BDAB69AA
:1095100023F08E6323F04003AB6121696368AA697D
:109520000B431343A2691343AB61D4E9022343EA1B
:1095300002432B61D4E90931EA680B4322F4F85263
:109540001343EB602046FFF7A1FF0028DCD1D4E9EC
:109550000713AA690B4322F0604213436269134365
:10956000AB61FF236B62012384F82D300020CDE72F
:109570000120CBE7002800400023092803D840EA57
:109580000310C0B270470A380133C0B2F5E70000DB
:109590002DE9F04790F82C30012B05464FF00200E2
:1095A00069D0012385F82C304E4B85F82D00DE68FC
:1095B00006F44076B6F5807F78D04C69087891F84B
:1095C000019091F802A091F82470002A55D19B696E
:1095D00013F0400308BFCB70FFF7CEFF804648462C
:1095E000FFF7CAFF02465046FFF7C6FF81463846DE
:1095F000FFF7C2FF0B6ACF78234343EA875343EA5E
:10960000090343EA084343EA022343EA0063354A75
:10961000CA205062532050628C6A8869B4F5807FFA
:10962000946945D124F4885494610124D465B6F535
:10963000807F09BFCB6913640343536418BF506430
:10964000284B4A681A672A6B42F001022A639A691A
:1096500042F488529A61244AD2F8803043F40033AD
:10966000C2F880301F4BFF225A620020012385F888
:109670002D3085F82C00BDE8F087B4F1803F07D08D
:10968000B4F5000F04D09B6913F0400308BFCB7002
:109690000B6ACA781C4344EA0A0444EA004343EADA
:1096A000092343EA825343EA0763B0E70023AEE7A6
:1096B00024F4085494610224D465B6F5807F09BF70
:1096C000CB6993640343D36418BFD064054B4A68E5
:1096D0005A672A6B42F002022A639A6942F40852DE
:1096E000B8E700BF002800400008005890F82C2080
:1096F000012A03464FF0020012D00A4A83F82D00D7
:10970000CA21516253215162916941F02001916156
:10971000FF2151620020012283F82D2083F82C00C4
:10972000704700BF0028004090F82C20012A034613
:109730004FF0020019D00D4A83F82D00CA21516262
:109740005321516291690A4841F080019161D0F83A
:10975000801041F48021C0F88010FF215162002068
:10976000012283F82D2083F82C0070470028004048
:1097700000080058064B5A6D520610B5044603D532
:109780004022DA65FAF7B4FC012384F82D3010BDCD
:10979000002800407047890001F1804101F5314106
:1097A0000A607047890001F1804101F53141086884
:1097B000704700002DE9F3471F468946904604464E
:1097C000FAF71EFA0A9D3D442D1AFAF719FA264BAC
:1097D0001E68C6F3CB366E438246019622689368B4
:1097E00039EA03030CBF01230023434501D10020C4
:1097F0002EE07B1CF3D0FAF703FAA0EB0A00A84294
:1098000029D323685A6822F0E0025A606268B2F5F0
:10981000827F0AD1A268B2F5004F02D0B2F5806F04
:1098200003D11A6822F040021A60A26AB2F5005F02
:1098300007D11A6822F400521A601A6842F40052E2
:109840001A60012384F85D30002384F85C30032023
:1098500002B0BDE8F087019A019B002A03F1FF33B3
:10986000019308BF1546B9E7A80300202DE9F74F7B
:10987000994600238DF80330044688461746FAF7C8
:10988000BFF90C9D4D442D1AFAF7BAF92C4BD4F8B8
:1098900000B01E6823235E43360D6E438246019658
:1098A0002268936803EA0803BB4201D100203AE032
:1098B000B8F5C06F07D137B99BF80C30DBB28DF823
:1098C00003309DF80330B9F1FF3FEAD0FAF798F979
:1098D000A0EB0A00A84229D323685A6822F0E002CC
:1098E0005A606268B2F5827F0AD1A268B2F5004F71
:1098F00002D0B2F5806F03D11A6822F040021A60DC
:10990000A26AB2F5005F07D11A6822F400521A6009
:109910001A6842F400521A60012384F85D30002373
:1099200084F85C30032003B0BDE8F08F019A019BFE
:10993000002A03F1FF33019308BF1546B0E700BFCB
:10994000A803002073B50B4600920D4616464FF44F
:10995000C05100220446FFF789FF024630B1236E52
:1099600043F020032366032002B070BD00962B460F
:1099700080212046FFF71EFF02460028EFD1009607
:109980002B464FF4C0612046FFF770FF0028EBD054
:10999000E5E74368B3F5827FF7B504460E46174600
:1099A0000BD18368B3F5004F02D0B3F5806F04D1BB
:1099B0002268136823F040031360009733460022A7
:1099C00080212046FFF7F6FE054628B1236E43F0BE
:1099D00020032366032514E06368B3F5827F10D16A
:1099E000A368B3F5004F02D0B3F5806F09D100979B
:1099F000334600224FF4C0612046FFF737FF0028AE
:109A0000E4D1284603B0F0BDF8B5044600287ED066
:109A1000436A002B50D14268B2F5827F00D0C36107
:109A200094F85D3003F0FF0223B984F85C202046EF
:109A3000F9F726FC2268E068022384F85D30136899
:109A4000B0F5E06F23F0400313604FF0000337D907
:109A50001D46B0F5706F18BFA362A7686368A1695F
:109A6000A66A07F4044703F482733B43276907F0AF
:109A700002073B43676907F001073B4301F40077A6
:109A80003B43E76907F038073B43276A07F0800745
:109A90003B4306F400573B43B6F5005F136014D117
:109AA000236B8BBBB0F5E06F0DD9022323631368E2
:109AB00043F40063136008E00023C0E90433AFE718
:109AC0004FF48055C7E701232363636A676B03F094
:109AD000100307F0080700F470603B43090C0343D0
:109AE00001F004010B432B43B6F5005F536004BF44
:109AF000A38D1361D36923F40063D3610020012394
:109B0000206684F85D30F8BD022BDED1CFE701205E
:109B1000F9E7000070B5044690F85C00012800F0F9
:109B2000CF80012084F85C0094F85D00666801280D
:109B3000C5B20AD0B6F5827F40F0C080A068002888
:109B400040F0BC80042D40F0B980002951D0002A9B
:109B50004FD0002B4DD094F85D00A16304281CBFAA
:109B6000052084F85D0000202066C4E91300A06A87
:109B7000E387B0F5005F2168A3872264A4F844302E
:109B8000A4F8463007D1086820F40050086008683F
:109B900040F400500860486820F4C0404860E06825
:109BA000B0F5E06FA06D29D94B6823F480534B606A
:109BB00094F85D30434E444D042B444B18BF1D4672
:109BC000434B18BF3346C0E90B35424B4363002378
:109BD0008363B4F846300C319BB2FEF785FA034636
:109BE000002848D0236E43F010032366012384F835
:109BF0005D300120002384F85C3070BD4D6845F471
:109C000080554D60656DAD69B5F5806F0AD113F073
:109C1000010F4B681ED123F480434B60E38FC3F3E5
:109C20004E03E3878369B3F5806FC1D14B6823F49A
:109C300080534B60B4F8463013F0010F4B6811D1DC
:109C400023F400534B60B4F84630C3F34E03A4F83A
:109C50004630ADE743F480434B60E38FC3F34E03DC
:109C60000133DEE743F400534B60B4F84630C3F3EE
:109C70004E030133EBE72268606D516841F001014A
:109C80005160C0E90B33C0E90D33E38FA16B9BB288
:109C90000C32FEF729FA0028A4D123681A6852066C
:109CA0005EBF1A6842F040021A605A6842F0200211
:109CB0005A605A6842F002025A609BE7022099E714
:109CC00002209AE70D9E0008DD9C0008E99C000830
:109CD000179D0008F59C00087047704708B5806A1A
:109CE000FFF7FBFF08BD704708B5806AFFF7FBFF71
:109CF00008BD7047806A026808B5536823F0030303
:109D00005360036E43F010030366012380F85D3057
:109D1000FFF7EFFF08BD7FB5064600230393846A73
:109D20008DF80B30F9F76CFF33681B689A0605460F
:109D300068D42268536823F020035360A36AB3F504
:109D4000005F13D101220090642311462046FFF7E3
:109D500031FD18B1236E43F002032366E3682668E1
:109D6000B3F5E06F2ED9F3680393039BA2682368D1
:109D7000002A43D16268B2F5827F3FD15A6822F04F
:109D800003025A6064212A462046FFF702FE08B10A
:109D9000202323660023A4F846302268012384F898
:109DA0005D309368DB0606D5236E43F0020323661D
:109DB0004FF6EF739360236E23B32046FFF799FFAE
:109DC00004B070BD337BDBB28DF80B309DF80B30E7
:109DD000236B022BCAD10122009564231146204631
:109DE000FFF7E8FC18B1236E43F002032366337BD0
:109DF000DBB28DF80B309DF80B30B7E75A6822F0D4
:109E00000102BEE72046FFF767FFD9E77FB50646A8
:109E100000230393846A8DF80B30F9F7F1FE336861
:109E20001B68990605465ED42268536823F0200318
:109E30005360A36AB3F5005F1BD1E368B3F5E06F2D
:109E40003ED1236B012B3BD1009064234FF4007271
:109E50004FF4C0612046FFF709FD18B1236E43F0AF
:109E60000203236623681B7BDBB28DF80B309DF861
:109E70000B302A4664212046FFF764FD18B1236E9B
:109E800043F02003236623685A6822F003025A60D5
:109E90000022E287A4F84620012284F85D209A6817
:109EA000D20606D5226E42F0020222664FF6EF720B
:109EB0009A60236EBBB12046FFF71BFF04B070BD54
:109EC000009564234FF480624FF4C0612046FFF791
:109ED000CDFC18B1236E43F0020323662368DB68D0
:109EE0000393039BC5E72046F8F7E6FCE6E700008E
:109EF000036830B559689A6802F04105012D85B0B4
:109F0000044606D14D0604D5C36C05B0BDE830400B
:109F10001847950704D5080602D5236D2046F4E7B7
:109F200012F4B07F59D08D0657D550060FD594F84E
:109F30005D0003284FF0000549D0206E40F004007A
:109F400020660095D8680090986800900098950663
:109F50000CD5206E40F00100206600200290986829
:109F60000290186820F0400018600298D00508D5CB
:109F7000226E42F008022266002203929A6803923F
:109F8000039A226E4AB35A6822F0E0025A60012214
:109F900084F85D208A0722D05A68A06D22F003025F
:109FA0005A6040B1104B8363FEF717F918B1236E66
:109FB00043F040032366606D78B10B4B8363FEF77B
:109FC0000CF950B1236E43F04003236605E0019580
:109FD000DA6801929B680193019B05B030BD204671
:109FE000FFF787FEF9E700BFED9F000808B5806A1C
:109FF0000023A0F84630C387FFF77BFE08BD0000B2
:10A00000034AD2F8903043F40043C2F890307047CE
:10A0100000040058034AD2F8903023F40043C2F8F9
:10A020009030704700040058074B1A6822F0400235
:10A030001A6040F441704FF4B85218605A601A68C0
:10A0400042F040021A6070470000015837B50546DB
:10A0500000284ED0837903F0FF046BB1032C0BD0A2
:10A06000254B4FF400629A612868FFF7DDFF00245A
:10A0700001232B71AC602FE000236B712846F9F7A8
:10A08000D3FC1E4AD2F8903043F48053C2F890308B
:10A09000002CE5D102234FF0B042AB71D2F89430DE
:10A0A00023F40043C2F89430154B1B681C214B432A
:10A0B000DB0C64214B430193019B93B90124AC60F9
:10A0C000FFF79EFF0C4B9A6842F400629A604FF4CF
:10A0D00000629A61002CC7D00123AB71204603B007
:10A0E00030BD019B013B0193D2F894305B04E3D473
:10A0F000E6E70124F2E700BF00040058000800581A
:10A10000A803002037B5174D2B6802461C20434397
:10A11000DB0C6420434314480193019B93B9012055
:10A120009060114C21732B681C214B43DB0C642184
:10A130004B430193019B6BB9012090600A4BDB6894
:10A1400003B030BD019B013B019383689C07E4D5BC
:10A150000020E6E7019B013B0193A368DB07E9D5FB
:10A16000ECE700BFA80300200000015837B5184DE8
:10A170002B6802461C204343DB0C642043431548F4
:10A180000193019BA3B901209060124CFF2323731C
:10A190002B681C256B43DB0C64256B430193019BEF
:10A1A00073B9012090600B4BDB680B7003B030BDBE
:10A1B000019B013B019383689C07E2D50020E4E703
:10A1C000019B013B0193A368DB07E8D5EBE700BFE8
:10A1D000A8030020000001580E4B0F491B681822ED
:10A1E000534382B01B0D6422534301934B69019A80
:10A1F000C3F3800322B902238360012002B07047B9
:10A20000019A013A01924A69920701D5002BEDD1DA
:10A210000020F3E7A80300200004005807B50379E5
:10A22000012B0FD10A4B1B68182253431B0C0193BF
:10A23000FFF7F0FE019B013B0193019B002BF9D13D
:10A24000FFF7DEFE03B05DF804EBFFF7C5BF00BF0C
:10A25000A8030020F8B51E468379012B1546044655
:10A260000F46DAB22DD14379012B2AD00223427155
:10A270008371FFF7D3FF0D212046FFF7CBFEFFF7D9
:10A2800041FF390A2046FFF73DFFF9B22046FFF7AC
:10A2900039FF2E44B5420ED12046FFF7B1FEFFF73D
:10A2A0009BFFA06801230038A3714FF0000318BF83
:10A2B00001206371F8BD15F8011B2046FFF722FF4E
:10A2C000E8E70220F6E7F8B51E468379012B15462C
:10A2D00004460F46DAB22FD14379012B2CD04271BC
:10A2E000FFF79CFF1D212046FFF794FEFFF70AFFB2
:10A2F000390A2046FFF706FFF9B22046FFF702FFB2
:10A3000000212046FFF7FEFE2E44B5420ED1204626
:10A31000FFF776FEFFF760FFA06801230038A37106
:10A320004FF0000318BF01206371F8BD2946204695
:10A33000FFF71CFF0135E8E70220F6E7F8B51F46F6
:10A340008379012B154604460E46DAB22CD14379A7
:10A35000012B29D04271FFF761FF06F0EF03A3F153
:10A36000840253425341237131462046FFF752FE87
:10A37000FFF7C8FE2F44AF4210D1FFF741FE842EF5
:10A3800002D02046FFF728FFA06801230038A37100
:10A390004FF0000318BF01206371F8BD15F8011BD1
:10A3A0002046FFF7AFFEE6E70220F6E7F8B51E46C7
:10A3B0008379012B154604460F46DAB227D143793B
:10A3C000012B24D04271FFF729FF39462046FFF7C1
:10A3D00021FEFFF797FE00212046FFF793FE2E4453
:10A3E000B5420ED12046FFF70BFEFFF7F5FEA06841
:10A3F00001230038A3714FF0000318BF01206371DF
:10A40000F8BD29462046FFF7B1FE0135E8E70220F6
:10A41000F6E737B50023ADF8043001AA0223122174
:10A420000546FFF7C3FFBDF80440022364BA01AA42
:10A43000A4B219462846FFF781FFE20702D5284655
:10A440000AF01EF8A30702D528460AF01FF8600795
:10A4500002D528460AF044F8210702D528460AF01A
:10A4600045F8E20602D528460AF046F8A30602D5CA
:10A4700028460AF02FF8600602D528460AF00CF8A4
:10A48000210606D514F4807118BF012128460AF070
:10A4900009F8A20502D528460AF014F8630402D58B
:10A4A00028460AF02FF803B030BDF8B51E46837970
:10A4B000012B154604460F46DAB227D14379012B0A
:10A4C00024D04271FFF7AAFE0E212046FFF7A2FD1D
:10A4D000FFF718FE39462046FFF714FE2E44B5421A
:10A4E0000ED12046FFF78CFDFFF776FEA068012312
:10A4F0000038A3714FF0000318BF01206371F8BD4D
:10A5000015F8011B2046FFF7FDFDE8E70220F6E7FE
:10A51000F8B51E468379012B154604460F46DAB27C
:10A520002BD14379012B28D04271FFF777FE1E21F2
:10A530002046FFF76FFDFFF7E5FD39462046FFF7A0
:10A54000E1FD00212046FFF7DDFD2E44B5420ED18E
:10A550002046FFF755FDFFF73FFEA06801230038B6
:10A56000A3714FF0000318BF01206371F8BD2946A5
:10A570002046FFF7FBFD0135E8E70220F6E7000083
:10A58000036A23F001030362036A70B544688269B9
:10A590000D6822F4803222F073022A438D6823F082
:10A5A00002032B43124DA84206D0124EB04203D0F4
:10A5B000A6F58066B04214D1CE6823F00803334379
:10A5C000A84223F0040306D00B4DA84203D005F5A2
:10A5D0008065A84205D124F44075D1E9054634438D
:10A5E0002C43446082614A684263036270BD00BFCD
:10A5F000002C01400048014000440140036A23F45C
:10A6000080730362036A426870B5C4690D6824F4FC
:10A61000803424F073042C438D6823F4007343EAE0
:10A6200005230F4DA8420ED1CD6823F4006343EA01
:10A63000052323F48063D1E9055622F440523543C3
:10A6400042EA051206E0074DA842F4D005F5806500
:10A65000A842F0D042604A68C461C263036270BD20
:10A66000002C014000440140036A23F4805303623C
:10A67000026A30B54468C3690D6823F0807323F41F
:10A68000E64343EA05238D6822F4005242EA05328C
:10A690000A4DA84207D005F5C055A84203D005F5DC
:10A6A0008065A84204D14D6924F4804444EA8514AD
:10A6B0004460C3614B680364026230BD002C0140FA
:10A6C000036A23F480330362026A30B54468436D41
:10A6D0000D6823F4803323F070032B438D6822F43C
:10A6E000003242EA05420B4DA84207D005F5C0559D
:10A6F000A84203D005F58065A84204D14D6924F431
:10A70000803444EA0524446043654B6883650262F3
:10A7100030BD00BF002C0140036A23F480130362A4
:10A72000026A30B54468436D0D6823F0807323F4EA
:10A73000E04343EA05238D6822F4001242EA055201
:10A740000A4DA84207D005F5C055A84203D005F52B
:10A750008065A84204D14D6924F4802444EA85240C
:10A76000446043654B68C365026230BD002C014004
:10A77000704710B5846A626A82420BD10123237745
:10A78000D2690AB984F83E302046F9F711F900235E
:10A79000237710BDA36A834208D102222277DB69A6
:10A7A000002BF1D1012384F83F30EDE7E36A8342C7
:10A7B00008D104222277DB69002BE5D1012384F83C
:10A7C0004030E1E7236B8342DED108222277DB6948
:10A7D000002BD9D1012384F84130D5E7704710B55B
:10A7E000846A636A834207D1012323772046FFF7F7
:10A7F000F5FF0023237710BDA36A834201D1022312
:10A80000F3E7E36A834201D10423EEE7236B83423B
:10A81000ECD10823E9E7704710B5846A636A834284
:10A8200009D10123237784F83E302046FFF7F3FF58
:10A830000023237710BDA36A834205D10223237727
:10A84000012384F83F30F0E7E36A83424FF00103CD
:10A8500004D10422227784F84030E6E7226B82425A
:10A8600003BF0822227784F8413084F83D30DCE7CA
:10A870001A4A0368904210B502D0B0F1804F09D156
:10A880004C6823F07003904243EA040309D0B0F10E
:10A89000804F06D0124A904203D002F58062904267
:10A8A00003D1CA6823F4407313434A6923F0800339
:10A8B000134303608B68C3620B688362074B984243
:10A8C00007D003F5C053984203D003F58063984244
:10A8D00001D10B6903630123436110BD002C0140CA
:10A8E0000044014010B5044650B390F83D3003F0E9
:10A8F000FF021BB980F83C20F9F75AFA02232068BE
:10A9000084F83D30211DFFF7B3FF012384F8483060
:10A91000002084F83E3084F83F3084F8403084F8DA
:10A92000413084F8423084F8433084F8443084F86D
:10A93000453084F8463084F8473084F83D3010BD07
:10A940000120FCE710B5044650B390F83D3003F009
:10A95000FF021BB980F83C20FFF70AFF02232068A2
:10A9600084F83D30211DFFF783FF012384F8483030
:10A97000002084F83E3084F83F3084F8403084F87A
:10A98000413084F8423084F8433084F8443084F80D
:10A99000453084F8463084F8473084F83D3010BDA7
:10A9A0000120FCE7036A23F010030362036A426894
:10A9B00070B584690D6824F0807424F4E64444EA98
:10A9C00005248D6823F0200343EA05130F4DA842A8
:10A9D0000ED1CD6823F0800343EA051323F0400332
:10A9E000D1E9055622F44062354342EA850206E089
:10A9F000074DA842F4D005F58065A842F0D042602A
:10AA00004A6884618263036270BD00BF002C01400C
:10AA10000044014038B590F83C30012B044673D017
:10AA200001200C2A84F83C004ED008D8042A2BD0F0
:10AA3000082A39D0BAB1002384F83C3038BD102A36
:10AA400052D0142AF7D12068FFF766FE436D0A69D9
:10AA500043F400634365436D23F480634365436DB2
:10AA600043EA02234EE02068FFF78AFD83690A6902
:10AA700043F008038361836923F0040383618369DE
:10AA8000134383610020D6E72068FFF78BFF8369BB
:10AA90000A6943F400638361836923F480638361FB
:10AAA000836943EA0223ECE72068FFF7A7FDC36947
:10AAB0000A6943F00803C361C36923F00403C36157
:10AAC000C3691343C361DDE72068FFF7CDFDC369A8
:10AAD0000A6943F40063C361C36923F48063C361FB
:10AAE000C36943EA0223EDE72068FFF7E9FD436D00
:10AAF0000A6943F008034365436D23F0040343658B
:10AB0000436D13434365BDE7022097E710B58468A2
:10AB10000A4324F47F4442EA03222243826010BDA8
:10AB200038B590F83C30012B04464FF0020000F09D
:10AB3000958084F83D000122206884F83C208568D7
:10AB4000474B2B4083600B68602B54D037D8402B89
:10AB50006BD019D8202B0DD00AD833F0100109D0B2
:10AB6000012384F83D30002384F83C30104638BD82
:10AB7000302BF5D1826822F4401222F070021A4381
:10AB800042F0070282602BE0502BE9D14A68CD6881
:10AB9000016A036A23F001030362836921F00A0159
:10ABA00023F0F00343EA05130A43836102628368DA
:10ABB00023F4401323F0700343F057030FE0B3F581
:10ABC000805F0DD0B3F5005F0CD0702BC8D1CB687F
:10ABD000D1E90121FFF79AFF836843F0770383608F
:10ABE0000022BDE7CB68D1E90121FFF78FFF836821
:10ABF00043F48043F3E7036A4D68C96823F0100308
:10AC000003628269036A22F4704223F0A00343EADC
:10AC1000051342EA013282610362836823F4401320
:10AC200023F0700343F06703D9E74A68CD68016AEF
:10AC3000036A23F001030362836921F00A0123F010
:10AC4000F00343EA05130A4383610262836823F435
:10AC5000401323F0700343F04703C0E7024685E743
:10AC60008800CEFF036A01F01F0110B501248C405B
:10AC700023EA04030362036A8A401A43026210BD96
:10AC800038B50D46082D044611461BD005D85DB1D8
:10AC9000042D14D094F8430008E00C2D15D0102D8D
:10ACA000F8D190F8420001E090F83E00A0F1020CCB
:10ACB000DCF1000040EB0C0050B1022076E090F88F
:10ACC0003F00F3E790F84000F0E790F84100EDE72F
:10ACD000082D1AD007D86DB1042D13D094F8432055
:10ACE000012A19D00CE00C2D27D0102DF6D194F8A4
:10ACF00042000CE094F83E20501E424242415AB9B4
:10AD0000012053E094F83F20F6E794F84000421EFB
:10AD1000504250410028F3D00029F1D0002BEFD051
:10AD2000082D4FF0020256D00AD885B1042D3ED02E
:10AD3000042D84F84320E3D13BE094F84100E6E79A
:10AD40000C2D5CD0102DF3D184F84220D8E7606A36
:10AD500084F83E203A4AC2623A4A02633A4A42635F
:10AD600022683432FDF7C0F90028C9D12268D368BF
:10AD700043F400732068D36029460122FFF772FF75
:10AD8000324A904250D0324B98424DD003F5806306
:10AD9000984249D0B0F1804F4DD182682D4B13407D
:10ADA000062B02D0B3F5803F45D1002038BD84F892
:10ADB0003F20A06A224AC262224A0263224A4263B8
:10ADC00022683832FDF790F9002899D12268D368BB
:10ADD00043F48063CEE7E06A84F84020184AC262F8
:10ADE000184A0263184A426322683C32FDF77CF934
:10ADF000002885D12268D36843F40063BAE7206B4A
:10AE000084F841200E4AC2620E4A02630E4A42632F
:10AE100022684032FDF768F900287FF471AF22689C
:10AE2000D36843F48053A5E7436C904243F4004356
:10AE30004364B2D0AEE7036843F001030360B4E7B4
:10AE400073A70008DFA7000819A80008002C01401C
:10AE50000044014007000100FFF712BF082938B580
:10AE600004460D464FD004D861B1042944D00120D6
:10AE700038BD0C29FBD10268006BD36823F48053E2
:10AE8000D36005E00268406AD36823F40073D3609E
:10AE9000FDF7A3F9206800222946FFF7E3FE2A4BBD
:10AEA000984207D003F5C053984203D003F580635E
:10AEB00098420DD1026A41F211131A4208D1026A76
:10AEC00040F244431A4202BF436C23F400434364FC
:10AED000026A41F211131A4208D1026A40F2444355
:10AEE0001A4202BF036823F00103036001238DB9F6
:10AEF00084F83E300020BBE70268806AD36823F400
:10AF00008063D360C4E70268C06AD36823F4006337
:10AF1000D360BDE70C2D13D007D8042D0AD0082D1F
:10AF20000BD0012384F84330E4E7102DF9D184F8E5
:10AF30004230DFE784F83F30DCE784F84030D9E77F
:10AF400084F84130D6E700BF002C0140FFF786BFF0
:10AF500070B590F83C30012B02464FF0020020D033
:10AF600082F83D000F4D106843688468A84202BF14
:10AF70004E6823F4700333430E6823F070033343A9
:10AF8000A842436002D0B0F1804F04D1896824F018
:10AF900080030B4383600123002082F83D3082F858
:10AFA0003C0070BD002C0140026852E8003F23F0D5
:10AFB000C00342E8003102680029F5D102F108031C
:10AFC00053E8003F23F4000302F1080C4CE8003181
:10AFD0000029F3D12023C0F88830704710B50268EB
:10AFE00052E8003F23F4907342E8003102680029E0
:10AFF000F5D10F4C02F1080353E8003F234002F162
:10B00000080C4CE800310029F4D1C36E012B07D1A4
:10B0100052E8003F23F0100342E800310029F7D145
:10B020002023C0F88C300023C366436710BD00BFE7
:10B03000FEFFFFEFF8B504461346D4F88850202DE4
:10B0400032D1F1B1EAB1E06FA4F85620A4F854204F
:10B0500000262122C4F890602165C4F88820226867
:10B0600088B1124FC762124F0763124F2832C0E9EE
:10B070000D76FDF739F830B11023C4F89030C4F8DC
:10B0800088500120F8BD236840221A62226802F12C
:10B09000080353E8003F43F0800302F1080141E850
:10B0A00000300028F3D1EDE70220EBE7B9B000084B
:10B0B00001B100080DB1000808B50346806A1B689D
:10B0C0001B6813F0200317D1A0F85630026802F174
:10B0D000080353E8003F23F08003083242E80031C0
:10B0E00002680029F2D152E8003F43F0400342E8F1
:10B0F00000310029F7D108BDF9F72EF9FBE77047B9
:10B1000008B5806AFFF7FBFF08BD7047806A38B555
:10B110000468D0F88830D0F88C50A268120606D5A2
:10B12000212B04D10023A0F85630FFF73DFFA36880
:10B130005B0606D5222D04D10023A0F85E30FFF770
:10B140004DFFD0F8903043F01003C0F89030FFF777
:10B15000DCFF38BD08B5806A0023A0F85E30A0F897
:10B160005630FFF7D2FF08BD704700000368D96969
:10B170001A682DE9F04140F60F0631429D680446F9
:10B1800010D18E0640F1978002F0200605F080571E
:10B190003E4300F09080436F002B00F08580BDE8B7
:10B1A000F0411847AB4EAC482E401040304300F001
:10B1B0008280CF0709D5D00507D501201862D4F8C1
:10B1C000900040F00100C4F890008F0709D5E8070F
:10B1D00007D502201862D4F8900040F00400C4F8AB
:10B1E00090004F0709D5E80707D504201862D4F866
:10B1F000900040F00200C4F890000F070BD502F059
:10B200002000304307D008201862D4F8900040F0A6
:10B210000800C4F890000E050AD5500108D54FF477
:10B2200000601862D4F8903043F02003C4F89030E6
:10B23000D4F89030002B37D08B0609D502F02002CD
:10B2400005F080552A4303D0636F0BB12046984721
:10B250002668D4F89020B36802F0280203F0400377
:10B2600053EA0205204621D0FFF7B8FEB3685F0617
:10B2700017D5226802F1080353E8003F23F040038A
:10B28000083242E800310029F3D1D4F8800040B1FF
:10B29000724B8363FCF7A1FF30B1D4F88000836B5D
:10B2A0007DE72046FFF731FFBDE8F081FFF72DFF76
:10B2B000C4F89050F8E7E06E012840F08980CE068F
:10B2C00040F18680D00640F1838010221A629A688D
:10B2D00051064BD5D4F8802011684A6892B2002AF2
:10B2E000E2D0B4F85C009042DED9A4F85E200A688F
:10B2F00092062FD453E8002F22F4807243E80021F5
:10B300000029F7D103F1080252E8002F22F00102D0
:10B3100003F1080040E800210029F3D103F10802FD
:10B3200052E8002F22F0400203F1080040E800211B
:10B330000029F3D12022C4F88C20E16653E8002FC5
:10B3400022F0100243E800210029F7D1D4F8800050
:10B35000FCF70EFF02232367B4F85E30B4F85C10EC
:10B36000C91A89B22046FFF7FFFE9DE7B4F85E20B8
:10B37000B4F85E00B4F85C1080B292B2002893D0AA
:10B38000891A89B200298FD053E8002F22F49072D5
:10B3900043E800200028F7D1314D03F1080252E8BC
:10B3A000002F2A4003F1080646E800200028F4D1C7
:10B3B0002022C4F88C206067E06653E8002F22F05A
:10B3C000100243E800200028F7D102232367C9E7D1
:10B3D000CF0209D56E0207D54FF4801220461A62BB
:10B3E000BDE8F04100F0A0BD08060BD502F08000DA
:10B3F00005F40005284305D0A36F002B3FF454AF9C
:10B400002046CCE64F0611D556060FD553E8002F3F
:10B4100022F0400243E800210029F7D12023C4F89C
:10B420008830A1672046F8F797FF3DE70D0206D563
:10B43000500004D52046BDE8F04100F077BDCB01B7
:10B440007FF532AF002ABFF62FAF2046BDE8F041AE
:10B4500000F06BBD010000102001000455B1000890
:10B46000FEFFFFEFD0F88C20B0F86010222A08B55C
:10B47000036855D15B6A826D0B401370836D013395
:10B480008365B0F85E30013B9BB2A0F85E30B0F847
:10B490005E309BB2002B42D1026852E8003F23F499
:10B4A000907342E8003103680029F5D103F10802E6
:10B4B00052E8002F22F0010203F1080C4CE80021B1
:10B4C0000029F3D12022C0F88C20184A416793420A
:10B4D000016705D1C26E012A0ED0F8F74BFF1EE0BE
:10B4E0005A681102F6D553E8002F22F0806243E833
:10B4F00000210029F7D1EDE70022C26653E8002FB2
:10B5000022F0100243E800210029F7D1DA69B0F8EF
:10B510005C10D20644BF10221A62FFF725FE08BD58
:10B520009A6942F008029A61F9E700BF0080004082
:10B53000D0F88C20B0F86010222A08B5036852D1E8
:10B540005A6A1140826D22F8021B8265B0F85E20B3
:10B55000013A92B2A0F85E20B0F85E2092B2002AC2
:10B5600040D153E8002F22F4907243E800210029D3
:10B57000F7D103F1080252E8002F22F0010203F193
:10B58000080C4CE800210029F3D12022C0F88C20BF
:10B59000174A41679342016705D1C26E012A0ED056
:10B5A000F8F7E8FE1EE05A681102F6D553E8002FBE
:10B5B00022F0806243E800210029F7D1EDE7002264
:10B5C000C26653E8002F22F0100243E80021002950
:10B5D000F7D1DA69B0F85C10D20644BF10221A62C3
:10B5E000FFF7C2FD08BD9A6942F008029A61F9E7C7
:10B5F000008000402DE9F84F0368B0F86060D3F890
:10B600001CB01F689D68D0F88C20222A044640F0A8
:10B61000B980B0F8683043B1DFF87491DFF874A1F5
:10B620004FF000081BF0200F20D1B4F85E309BB221
:10B63000D3B1B4F868209A4216D9226802F10803FF
:10B6400053E8003F23F08053083242E8003122687B
:10B650000029F2D1504B636752E8003F43F02003CA
:10B6600042E800310029F7D1BDE8F88F2368A26DC8
:10B670005B6A33401370A36D0133A365B4F85E3089
:10B68000013B9BB2A4F85E302368D3F81CB01BF0DA
:10B69000070F2ED01BF0010F09D0F90507D50122A5
:10B6A0001A62D4F8902042F00102C4F890201BF0F6
:10B6B000020F09D0EA0707D502221A62D4F89020B7
:10B6C00042F00402C4F890201BF0040F09D0E807F0
:10B6D00007D504221A62D4F8903043F00203C4F86C
:10B6E0009030D4F8903023B12046FFF70EFDC4F817
:10B6F0009080B4F85E309BB2002B93D1226852E860
:10B70000003F23F4807342E8003123680029F5D11B
:10B7100003F1080252E8002F02EA090203F10800CF
:10B7200040E800210029F3D120225345C4F88C20A1
:10B73000616721670AD05A68110207D553E8002FC4
:10B7400022F0806243E800210029F7D1E26E012A4D
:10B7500014D10022E26653E8002F22F0100243E8E1
:10B7600000210029F7D1DA69B4F85C10D20644BF91
:10B7700010221A622046FFF7F7FC53E72046F8F73D
:10B78000F9FD4FE79A6942F008029A616CE700BF41
:10B79000FEFFFFEF0080004065B400082DE9F84F80
:10B7A0000368B0F86060D3F81CB01F689D68D0F8DB
:10B7B0008C20222A044640F0B780B0F8683043B1AC
:10B7C000DFF87091DFF870A14FF000081BF0200F38
:10B7D00020D1B4F85E309BB2D3B1B4F868209A425D
:10B7E00016D9226802F1080353E8003F23F0805382
:10B7F000083242E8003122680029F2D14F4B6367DA
:10B8000052E8003F43F0200342E800310029F7D11D
:10B81000BDE8F88F2368A26D596A314022F8021BF7
:10B82000A265B4F85E20013A92B2A4F85E20D3F883
:10B830001CB01BF0070F2ED01BF0010F09D0F9052B
:10B8400007D501221A62D4F8902042F00102C4F810
:10B8500090201BF0020F09D0EA0707D502221A62D6
:10B86000D4F8902042F00402C4F890201BF0040F9A
:10B8700009D0E80707D504221A62D4F8903043F0C3
:10B880000203C4F89030D4F8903023B12046FFF77B
:10B890003CFCC4F89080B4F85E309BB2002B95D18C
:10B8A000226852E8003F23F4807342E800312368A5
:10B8B0000029F5D103F1080252E8002F02EA09023B
:10B8C00003F1080040E800210029F3D1202253456C
:10B8D000C4F88C20616721670AD05A68110207D525
:10B8E00053E8002F22F0806243E800210029F7D1BD
:10B8F000E26E012A14D10022E26653E8002F22F002
:10B90000100243E800210029F7D1DA69B4F85C108D
:10B91000D20644BF10221A622046FFF725FC55E7E5
:10B920002046F8F727FD51E79A6942F008029A612C
:10B930006EE700BFFEFFFFEF0080004031B500085A
:10B9400038B5044603682169A2681D68C0690A43C6
:10B9500061690A437749024329400A431A605A68D9
:10B96000E16822F440520A435A60734AA169934243
:10B970001CBF226A11439A6822F06E4222F43062A0
:10B980000A439A60DA6A616A22F00F020A43DA62B5
:10B990006A4A934219D14FF0B043694AD3F88830CC
:10B9A00003F0030343F44033934200F0B480B3F157
:10B9B000031F24D0013A934240F0B580B0F5004F08
:10B9C00040F08F80FCF7C6FF6EE05E4A93421CD1C8
:10B9D0004FF0B0435C49D3F8883003F00C0343F4D4
:10B9E00040228A4200F0978006D8002B7CD0574B2B
:10B9F0009A42E3D0012026E0B2F10C1FFAD1B0F553
:10BA0000004F53D04FF4004075E04B4A9342F1D1C0
:10BA10004FF0B043D3F8883003F44063B3F5006FC0
:10BA200018D006D85BB1B3F5806FE3D1FCF792FF75
:10BA300007E0B3F5406FDDD14FF400400BE0FDF7B8
:10BA400081FB40B900204FF00113A3660023C4E935
:10BA50001D3338BD3E4865683E4B626A05EB4501C3
:10BA600033F81220B0FBF2F39942C3D8B3EB053F91
:10BA7000C0D800231946F6F717FD090241EA106104
:10BA80006B080002C0182A464FF0000341F1000184
:10BA9000F6F70AFD304BA0F540729A42AAD8236807
:10BAA000D860CFE7FDF74EFB0028CBD06168294B6B
:10BAB000626A33F81220B0FBF2F24B0803EB420348
:10BAC0004FF6EF72B3FBF1F3A3F11001914291D85D
:10BAD00023F00F02216892B2C3F342031343CB60F9
:10BAE000B0E7FCF737FF04E0B0F5004FDAD0FDF720
:10BAF00029FB0028A6D06368616A164A32F8112033
:10BB0000B0FBF2F000EB5300B0FBF3F04FF6EF7335
:10BB1000A0F11002C1E7B0F5004F0D48EBD1C5E729
:10BB2000FDF720FBC0E7B0F5004FF9D0FDF71AFB99
:10BB3000DFE700BFF369FFCF00800040003801401D
:10BB4000020003000044004008000C0004000C0048
:10BB50000024F400B86F0308FFFC0F00836ADA07C3
:10BB600010B506D50168C46A4A6822F4003222433F
:10BB70004A609C0706D50168046B4A6822F480324B
:10BB800022434A60590706D50168446B4A6822F48B
:10BB9000802222434A601A0706D50168846B4A68EE
:10BBA00022F4004222434A60DC0606D50168C46BD9
:10BBB0008A6822F4805222438A60990606D5016879
:10BBC000046C8A6822F4005222438A605A060FD518
:10BBD0000168446C4A6822F480122243B4F5801F45
:10BBE0004A6005D14A68846C22F4C00222434A604C
:10BBF0001B0606D50268C16C536823F400230B436F
:10BC0000536010BD2DE9F843DDF8209005460F463E
:10BC1000164698462A68D36937EA03030CBF012306
:10BC20000023B34201D0002029E0B9F1FF3FF2D058
:10BC3000F7F7E6FFA0EB080048452C6802D8B9F1F9
:10BC4000000F1ED154E8003F23F4D07344E80032C3
:10BC5000002AF7D104F1080353E8003F23F0010361
:10BC600004F1080141E80032002AF3D12023C5F88D
:10BC70008830C5F88C30002385F884300320BDE877
:10BC8000F88323685A07C5D5E3691B05C2D54FF46D
:10BC90000063236254E8003F23F4D07344E8003289
:10BCA000002AF7D104F1080353E8003F23F0010311
:10BCB00004F1080141E80032002AF3D12023C5F83D
:10BCC0008830C5F88C30C5F89030D4E773B5044699
:10BCD0000026C0F89060F7F793FF23681B681A07E7
:10BCE000054619D423681B685B070AD56FF07E43AD
:10BCF000009300222B464FF480012046FFF782FF7D
:10BD0000B0B900202023C4F8883084F88400C4F837
:10BD10008C30E06620670CE06FF07E430093324683
:10BD200003464FF400112046FFF76CFF0028D9D0DE
:10BD3000032002B070BD10B5044650B3D0F888306F
:10BD40001BB980F88430F8F715FA22682423C4F868
:10BD50008830136823F0010313602046FFF7F0FDDD
:10BD6000012816D0A36A13B12046FFF7F7FE236817
:10BD70005A6822F490425A609A6822F02A029A6025
:10BD80001A6842F0010220461A60BDE81040FFF731
:10BD90009DBF012010BD000030B581658168A0F80D
:10BDA0005C200023B1F5805FA0F85E20436735D1A9
:10BDB0000369002B40F2FF1318BFFF23A0F8603087
:10BDC0000023C0F890302223C0F88C30016801F1C4
:10BDD000080353E8003F43F00103083141E8003411
:10BDE0000368002CF2D1456E84680169B5F1005FEB
:10BDF00032D1B0F8685095422ED8B4F5805F244A0D
:10BE000003D1244C002908BF22464267B1B153E850
:10BE1000002F42F4807243E80021F7E729B9036953
:10BE2000002B14BF7F23FF23C8E7B1F1805FC5D18A
:10BE30000369002B14BF3F237F23BFE703F10802F0
:10BE400052E8002F42F0805203F1080040E8002140
:10BE50000029F3D1002030BDB4F5805F0E4A03D134
:10BE60000E4C002908BF2246426741B153E8002F1B
:10BE700042F4907243E800210029F7D1EAE753E841
:10BE8000002F42F0200243E800210029F7D1E1E72A
:10BE9000F5B500089DB7000865B4000831B5000885
:10BEA000D0F88C30202B30B415D1B9B1B2B1002309
:10BEB0000468C3660A4B9C420AD063681B0207D51C
:10BEC00054E8003F43F0806344E80035002DF7D18B
:10BED00030BCFFF761BF022030BC70470120FBE798
:10BEE00000800040436E30B52BB90123A0F86A30C2
:10BEF000A0F8683030BD0368094D9A689968094C0C
:10BF0000490FC2F342626B5C615CDB00B3FBF1F38F
:10BF1000A0F86A30AB5CA25CDB00B3FBF2F3E7E7AE
:10BF2000D86F0308D06F03087047704770471FB57C
:10BF300004AB03E9060090F88430012B04463AD0A4
:10BF4000012380F884302423C0F8883003681A68FD
:10BF500022F001021A609A6822F440120A439A60A1
:10BF600071B95A68BDF80C009DF80E1022F010024D
:10BF700002435A605A6822F07F4242EA01625A60E4
:10BF80001A6842F001021A60F7F73AFE6FF07E423B
:10BF9000034600924FF4800100222046FFF732FE54
:10BFA00038B92023C4F88830002384F8843004B0E2
:10BFB00010BD0320F8E70220F9E790F88430012B48
:10BFC0000FD0012380F88430016851E8002F42F03F
:10BFD000020241E80023002BF6D180F88430184695
:10BFE00070470220704710B590F88430012B04464A
:10BFF00017D02423C0F8883003681A68196821F024
:10C000000101196042F000524FF0005141661A6080
:10C01000FFF768FF2023C0F88830002084F88400F0
:10C0200010BD0220FCE770B590F88430012B044667
:10C0300017D005682423C0F888302E682B6823F0B9
:10C0400001032B60AB6823F060431943A960FFF73D
:10C0500049FF20232E60C0F88830002084F8840037
:10C0600070BD0220FCE770B590F88430012B0446C7
:10C0700017D005682423C0F888302E682B6823F079
:10C0800001032B60AB6823F060631943A960FFF7DD
:10C0900029FF20232E60C0F88830002084F8840017
:10C0A00070BD0220FCE7000038B5084D052455F8A6
:10C0B000043B2BB9013C14F0FF04F8D1204638BDF5
:10C0C000DB6898470028F5D0F9E700BFA8220020D8
:10C0D000034BD870034B1B681B6C03B118477047A8
:10C0E000902200208C220020034B1874034B1B6805
:10C0F0005B6C03B118477047902200208C2200200F
:10C10000F0B5314D314B95F90420314E91B00C46CC
:10C11000012795F905108DF8047002288DF8092083
:10C120008DF80A1010D18DF80800D8711C7202F039
:10C1300063FD337803B114B101A803F0C1F9254BB5
:10C14000059A1A6011B0F0BD59714FF480711A71DF
:10C15000D9801C7233788DF8087053BB1F2306A852
:10C160008DF81C208DF8183002F024FF20238DF864
:10C17000183006A82B798DF81C3002F01BFF222303
:10C180008DF8183006A86B798DF81C3002F012FF7C
:10C1900021238DF8183006A86B798DF81C3002F039
:10C1A00009FF29238DF8183006A80B4B079302F0DE
:10C1B00001FF02F021FD012306A88DF818308DF84B
:10C1C0001C3002F0F7FEB4E790220020E0030020CC
:10C1D0006C21002060220020000400017FB50923AB
:10C1E00001A88DF8043003F06BF90038044B059A70
:10C1F0001A6018BF0120404207B05DF804FB00BF81
:10C200006022002070B504460B46144962784A70DB
:10C210000020A2780A7208701A884A729A788A7284
:10C22000DB780B746368CB600D4B1B68DA6A2AB14C
:10C23000237803F0FB030A2B00D09047094E00251A
:10C2400056F8043B1BB15B6A0BB120469847013599
:10C25000EBB2052B6DB2F3D170BD00BFB00300206F
:10C260008C220020A822002070B50446114801232A
:10C27000037063784370A3788372E368C360E378E4
:10C28000037623694376237943720B4B1B689B6AC1
:10C2900003B19847094E002556F8043B1BB19B6932
:10C2A0000BB1204698470135EBB2052B6DB2F3D1A7
:10C2B00070BD00BFC40300208C220020A8220020F3
:10C2C000014B1868704700BF6022002000B58BB09A
:10C2D000012368468DF8003002F046FD38B99DF81C
:10C2E0000400003818BF01200BB05DF804FB0020EB
:10C2F000FAE7000008B501F037FE40B9FFF7E6FFA6
:10C30000012806D0054B197AD879FFF7F9FE0120EC
:10C3100008BDBDE80840FFF7C7BE00BFE00300202E
:10C320002DE9F04186B005460E46174601F01CFE89
:10C33000002873D101F030FE044640B9FFF7C6FF74
:10C3400001280AD03D4B197AD879FFF7D9FE6FF052
:10C350000204204606B0BDE8F081DFF8E48088F8EA
:10C360000860003E18BF01268DF80460354E6878DD
:10C3700033798DF81230694602F094FC00283FD0E2
:10C380008DF804400394ADF810406FF0060495E872
:10C3900003002D4B83E80300337988F80A303946CF
:10C3A00001A803F091F9294B059A1A6011283FD88A
:10C3B00001A353F820F000BF23C400081DC40008E7
:10C3C00031C4000831C4000831C4000831C4000879
:10C3D00031C400084FC3000831C4000831C400084C
:10C3E00031C4000817C4000831C4000831C4000873
:10C3F0001DC400081DC400081DC4000837C400087F
:10C400002B788DF808306B78ADF810306B6803939B
:10C410004FF0FF34BBE76FF005049AE76FF00104BB
:10C4200097E70B4B00221A70E31D18BF144690E7E4
:10C430004FF0FF348DE76FF004048AE7E00300203B
:10C44000C403002090220020D4030020602200209A
:10C450005F22002037B501F0A9FD134D052455F8E2
:10C46000043B4BB11A693AB19B682BB1984718B19C
:10C4700055F8043C1B699847013C14F0FF04EED1C9
:10C48000FFF712FE68B9094D2B7853B1084BADF890
:10C490000040D978019422466846FFF741FF00B971
:10C4A0002C7003B030BD00BFA82200205F22002006
:10C4B0009022002030B58BB0044601F055FD0546B2
:10C4C000002835D1FFF702FF012834D168468DF8E6
:10C4D000005002F049FC40BB9DF80430A34204D058
:10C4E000012C22D0022C12D014B100200BB030BD90
:10C4F000002BFAD068468DF8044002F05BFDA0B92D
:10C500000E4B1B681B6B002BEFD09847EDE763B910
:10C5100068468DF8044002F04DFD30B9074B1B68AA
:10C520001B6B002BE1D02046EFE74FF0FF30DDE73B
:10C530006FF00100DAE76FF00200D7E78C220020ED
:10C5400010B504468AB018B94FF0FF300AB010BDDC
:10C55000002368468DF8003002F006FC0028F3D175
:10C560009DF804302370F1E77FB500220B46204987
:10C570008DF8072001220A7042784A700446002A8A
:10C5800033D102790A721A884A729A788A72DB78F1
:10C590000B740369CB60C378164D8DF80830037BAC
:10C5A0008DF80930836803932B68DB6A0BB102A80E
:10C5B00098472B689B6B13B1227E02B198470E4EB1
:10C5C000052556F8043B1BB1DB690BB120469847A3
:10C5D000013D15F0FF05F4D10DF10700FFF7B0FFA5
:10C5E000637913B1054B01221A7004B070BD00BF0E
:10C5F000B00300208C220020A82200205F2200200F
:10C6000010B504468AB018B94FF0FF300AB010BD1B
:10C61000202368468DF8003002F0A6FB0028F3D1F5
:10C62000024A9DF9043023701371EFE79022002035
:10C6300000B58BB02323019068468DF8003002F0DE
:10C64000B9FC003818BF012040420BB05DF804FB74
:10C6500070B5654C01468EB01822204606F08CF865
:10C66000624B00221A70FAF7C5FE23784068012257
:10C6700002FA03F1014004D15D4B084608F068F866
:10C68000FEE75C495C481A4602F0F8F818B14FF032
:10C69000FF300EB070BD272304A88DF8103002F0D3
:10C6A00089FC564E564D002870D1012333702B68FB
:10C6B000DB690BB100209847272304A88DF81030C0
:10C6C00002F052FB059B93F84820227093F8182142
:10C6D00093F81A316270A370464BD3E9020105F05A
:10C6E0003BFF05460028D2D1464E062304A88DF80C
:10C6F000103002F039FB059B736104A802F05AFC6C
:10C70000022304A88DF81030059602F02DFB0836A0
:10C71000032304A88DF81030059602F025FB0F26A0
:10C7200005F0E0FF012304A88DF814308DF81060A7
:10C7300002F040FC10230DEB03008DF810308DF853
:10C74000145002F037FC04238DF8103004A8A378AD
:10C750008DF8143002F02EFC3A238DF8103004A826
:10C760006369059302F026FC02A920788DF8086021
:10C7700004F09CF8003818BF0120E0711420FFF786
:10C7800057FFE07903F062F9284682E728238DF805
:10C7900010302B681B6943B104A802F0E5FA2B683E
:10C7A00005981B6940F2C4519847272304A88DF8C7
:10C7B000103002F0FFFB50B9012304A88DF81030AF
:10C7C00002F0D2FA9DF81430002B7FF46EAF33786C
:10C7D000002B7FF46CAF052204A88DF81020059380
:10C7E00002F0E8FB78E700BF902200205F220020E3
:10C7F000E06F0308642200207C2200206C210020CE
:10C800008C220020CC22002037B500230D46019356
:10C810000446D0B900F0A8FB0190019BD3B10F4AA8
:10C8200042F824300E4A9A620E4A1268916B1963DC
:10C83000916C596392690C49D9625A6128465B68C8
:10C840000A49F2229847002006E001A900F092FB75
:10C850000028E2D04FF0FF3003B030BDA822002006
:10C8600001C100088C220020DDC100086D210020DC
:10C87000194B07B51860194B194A1A60194A5A60C2
:10C88000194A9A60194ADA60194B02681A604268BC
:10C890005A6082689A60C268DA60164A1A618269D0
:10C8A0005A61154BC26B5A60144A019119609A6023
:10C8B0001946134ADA600020FFF7A6FF48B901A81D
:10C8C00000F056FB003818BF0120404203B05DF86D
:10C8D00004FB4FF0FF30F9E78C2200207C2200207F
:10C8E00069C2000869C500087DC9000805C20008C2
:10C8F000642200205D080108BC220020D1C000088D
:10C90000E9C0000849B118B1012804D000207047DF
:10C91000034B0B60FAE7034BFBE74FF0FF30704728
:10C92000000400010100010208B503F0ABF8002883
:10C9300014BF6FF00100002008BD08B502F084F9B3
:10C94000002814BF6FF00100002008BD10B5044698
:10C950008AB018B94FF0FF300AB010BD21236846E5
:10C960008DF8003002F000FA0028F3D1024A9DF958
:10C97000043023705371EFE7902200202DE9F0413D
:10C980002F4D304F00232B7043786B703B689B6AB0
:10C990008AB004460BB128469847DFF8AC800026E1
:10C9A00058F8043B1BB11B6A0BB12046984701366F
:10C9B000F3B2052B76B2F3D12378052B2FD00B2BB6
:10C9C00035D0012B25D1214C062368468DF8003047
:10C9D00002F0CAF90199E07905F004FE10B91C4B88
:10C9E000019A5A611B48FFF70BFE1B48FFF7AEFF89
:10C9F0006B788BB9A371194B5878FFF75BFD3B68D7
:10CA00005B6A0BB1114898476B7813B9E07905F070
:10CA10007BFE0AB0BDE8F081FF23A371EFE7104B66
:10CA200001225A74227A9A74627ADA74F1E763788E
:10CA3000002BEED00AB0BDE8F041FFF7CFBB00BF3E
:10CA4000C40300208C220020A8220020E003002044
:10CA5000CC220020E4030020E503002090220020E7
:10CA6000B003002030B58BB0FFF767FF0446F0B984
:10CA700003F0FCFE831C1DD0F8B9134D2B685B69D5
:10CA8000DBB1272368468DF8003002F06DF92B6882
:10CA900001985B694FF4B961984703F0F9FE78B9E2
:10CAA0002CB9094B1B68DB690BB101209847204664
:10CAB0000BB030BD6FF00704EFE74FF0FF34ECE749
:10CAC0004FF0FF34F3E700BF8C220020014B1878B1
:10CAD000704700BF00230020014B5878704700BF0B
:10CAE0000023002070470000044B9A7A0AB101220B
:10CAF0005A70034B5B6903B118477047002300204D
:10CB0000EC03002073B5224C6378002B33D008F07F
:10CB100007F966680546FFF7D3FB0644AE4214D218
:10CB2000A37A93B1E0228DF800208DF80130217AAC
:10CB3000E368019301226846FFF7F2FB08B1073072
:10CB400010D100236370A372656094F83430EBB1A8
:10CB5000002384F834300F4B5B6BBBB102B0BDE8EF
:10CB60007040184740F2DC510B4808F0A5F90A481C
:10CB700008F068F9E8E794F83520002AE5D094F841
:10CB8000360084F83530FFF795FCDEE702B070BD63
:10CB900000230020EC030020E422002037B5104DD4
:10CBA000104CC8B1C1B16272012300222860E1605B
:10CBB00023700D480D4B00924FF0FF3108F096F8AE
:10CBC00000250B4825822022294605F0E9FD6570E5
:10CBD000A574A58603B030BD00232B602370EFE75A
:10CBE000FC22002000230020E4220020E9CA0008E3
:10CBF000142300202DE9F0478E4C23788CB0002BB5
:10CC000056D0C2780AB9837B13B1238A01332382B9
:10CC1000437B002B4CD0E02A4AD10023A3728768C3
:10CC200097F80080B8F1220F27D8B8F1220F30D83A
:10CC3000DFE818F04100FB0052005A0061006E006E
:10CC400075008E009D00B400C7002F002F002F003C
:10CC50002F002F002F002F002F002F002F002F005C
:10CC60002F002F002F002F002F002F002F002F004C
:10CC70002F002F00C900D000D400B8F17E0F00F0C3
:10CC8000CC80B8F17F0F00F0DF80B8F17D0F00F0AD
:10CC9000AB80A57A002D00F05B81674C637A3BB9CD
:10CCA0004FF47A71204608F007F9204608F0CAF8D8
:10CCB0000CB0BDE8F087E36801220021A272197070
:10CCC000A37AE1689818A0720620C854A37AE16894
:10CCD0009818A072CA54DCE7584B9B6A002BD8D036
:10CCE000012102209847D4E77B7884F8363001236D
:10CCF00084F83530CDE704238DF804307B78003B91
:10CD000018BF012301A88DF8083002F053F9C0E7DD
:10CD10007878003818BF012002F098FEB9E7484E35
:10CD20000FCE01AD0FC50FCE0FC596E8070085E801
:10CD300007007B780A2BACD8424A12685268002A56
:10CD4000A7D00CA901EB830353F82C0C9047A0E764
:10CD50007878431E012B9CD83A4B01381B6818BFCA
:10CD6000012020729B68002B93D0984791E7E268DE
:10CD700001230821A3721170627A057BA17AAA426D
:10CD800028BF2A46934284D285685A1CEB5CE5682A
:10CD900001334E1CA6726B54D3B2EDE7E368012257
:10CDA000A27209221A70A37AE268218A581CA07222
:10CDB000D154A27A238AE1681B0A501CA0728B54BA
:10CDC00067E7238265E705238DF8043001A802F0A8
:10CDD00077FB5EE7194BDB6A98475AE7194B78787F
:10CDE0001B686075DB68BEE7037B072B7FF451AFE0
:10CDF00006238DF80430B7F80130ADF808307B79A0
:10CE00003A791B0443EA0223FA781343642253431A
:10CE10000393BB798DF81030D8E73B2201A88DF839
:10CE200004208DF8083002F0C5F8012384F834306E
:10CE30002FE700BF00230020E4220020EC030020A5
:10CE4000041A0308FC2200202A2301A88DF80430CC
:10CE500001F08AFF94F80A90E6689DF808009DF8B2
:10CE600009509DF80A709DF80BC09DF80D309DF893
:10CE70000E209DF80F109DF80CE009F1010A84F8CE
:10CE80000AA006F80980354E94F80A903668D4F85E
:10CE90000C8009F1010A84F80AA096F803A008F8AA
:10CEA00009A094F80A90D4F80C8009F1010A84F8DA
:10CEB0000AA096F802A008F809A094F80A90D4F8FD
:10CEC0000C8009F1010A84F80AA096F801A008F87C
:10CED00009A094F80A9009F1010A84F80AA096F8CA
:10CEE0000080E66806F8098094F80A80E66808F190
:10CEF000010984F80A9006F808C094F80AC0E668A8
:10CF00000CF1010884F80A8006F80C70A77AE6682C
:10CF100007F1010C84F80AC0F555A57AE6686F1C84
:10CF2000A7727055A07AE568461CA6722954A17AAA
:10CF3000E0684D1CA5724254A27AE168501CA072B0
:10CF40008B54A37AE268591CA17202F803E0A0E6B0
:10CF5000034807F029FF6570AAE600BFFC22002005
:10CF6000E42200207047000000487047EC030020D6
:10CF7000002070474FF0FF3070470000044B054A17
:10CF800093F81831022B18BF062382F890347047AB
:10CF9000A4290020682F0020034BD3F8483313B195
:10CFA0005B6903B118477047682F0020034A137864
:10CFB00043F004031370FFF7EFBF00BF4C230020C2
:10CFC0001FB50A4B8DF8090093F87C208DF80A20D4
:10CFD00093F88C2093F848000D3202A98DF80820B0
:10CFE00003F064FCC0B205B05DF804FBA429002086
:10CFF00008B5074807F0D8FE064B93F81A2412B17B
:10D00000012283F81924BDE80840FFF7C5BF00BF1F
:10D0100068330020682F002010B50C4CD4F8403342
:10D0200043F08003C4F8403394F81A3413B100205D
:10D03000FFF7DEFF94F8913423F0120343F012035C
:10D0400084F89134BDE81040FFF798BF682F0020A6
:10D050002DE9F041DFF8AC8098F81831022B064634
:10D060000D4602D0284BDB6A984702F0A6FD044625
:10D0700028B1022002F097FD002002F099FD98F8F7
:10D080001831012B17D102F09AFD074630B100206C
:10D0900002F08AFD002002F08CFD3C4602F091FD7A
:10D0A00048B1002002F081FD002002F083FDBDE8C0
:10D0B000F041FFF763BF002CF9D1144C94F8902491
:10D0C00094F81A34BAB90BB184F84164304602F0CE
:10D0D00017FFD8F82C0007F02DFED4F8B43398428F
:10D0E000E5D30B4807F060FE94F8913443F0100349
:10D0F00084F89134DBE70BB184F84154284602F000
:10D10000FFFEF1E7A429002058770308682F0020CC
:10D1100000330020074A10B5137843F00203137060
:10D12000FFF73AFFBDE81040034B01220021022027
:10D1300007F00EBB4C23002029700308074A10B5E6
:10D14000137843F008031370FFF726FFBDE8104083
:10D15000034B01220021022007F0FABA4C230020E1
:10D16000397003082DE9F0410F4616461D468046EA
:10D1700007F0D6FD0B4A0C4C1378278123F01103DE
:10D1800043F01103C4E90008137066812573FFF7AB
:10D1900003FFBDE8F041054B01220021022007F00A
:10D1A000D7BA00BF4C230020382300204970030861
:10D1B00013B507F0B5FD0D4B6C461860204607F01F
:10D1C00003FD94E803000A4A0A4B83E8030013783E
:10D1D00043F020031370FFF7DFFE074B012200210D
:10D1E000022002B0BDE8104007F0B2BA4823002088
:10D1F0004C230020A0320020567003082DE9F04196
:10D2000092B0064602F0D9FC002840F05881AD4D9E
:10D2100095F81831012B09D02B6BAB4C93B194F8D6
:10D220000431BBB1042B6FD0032003E002F0C7FC34
:10D2300018B10F2012B0BDE8F08102F0C2FC002846
:10D24000EAD0F6E7B5F82031D4F81C24013B53436B
:10D250002B63E4E79D4803F060FA002840F0128158
:10D2600094F80C3123802B6B0C930DF1180895F872
:10D2700039308DF83830404695F81C318DF83A3009
:10D2800007F0C8FCD5F82831009302AF98E80600F3
:10D29000D5F82431384607F054FC97E803000FAB6B
:10D2A00083E80300EB6A0D9300238DF84430238854
:10D2B000ADF8463095F8303101228DF839201BB990
:10D2C0008DF844208DF83930814B0093814B95F8CF
:10D2D0004800A3F179020CA903F05DFBC0B10B2853
:10D2E000A8D1D4F8941499B1002EA3D0D4F8403327
:10D2F000794843F02003C4F8403307F0DDFD764859
:10D3000007F0A0FD002095E7704803F03AFAA4E783
:10D3100095F8487095F9693095F9392095F87D10A0
:10D320006E4E384603F044FB009641B2EB6C95F824
:10D3300050203846183603F0DFFA0096EB6C95F86B
:10D34000502095F9701095F8480003F0D5FAD4F8FC
:10D35000C413AB6DD4F8DC230B44C4F8B033EB6DCD
:10D360001344C4F8B43394F80431042B07D02B6E63
:10D370000B44C4F8B0336B6E1344C4F8B4330023C9
:10D38000089395F83031002B40D100238DF81330ED
:10D3900095F839308DF8213095F838308DF82230F5
:10D3A000D5F880300993D5F884300A932388ADF8F6
:10D3B0002C3095F8303194F81B648DF82E3095F8A8
:10D3C0004800474B8DF820600DF1130208A903F0C7
:10D3D000A7FA012384F8413495F8393084F84234AF
:10D3E0009DF8133084F84334D4F81C34C4F85064E6
:10D3F000C4F84834C4F8583402F0E5FBC8B1D4F896
:10D400001C0402F0F2FBA0B1102013E708A802F000
:10D41000A7FC60B995F9390094F837629DF820703F
:10D42000FFF7CEFD3E44B042AFD2082002E7132002
:10D4300000E795F81831012B01D102F0D8FB02F07A
:10D44000C5FB0023059394F8043195F9395094F8FD
:10D450001B649BB1042B7FF4E7AE05A802F0B4FE79
:10D4600058BB94F8183413B1059B013B0593174B37
:10D4700005983246E9B202F00DFF02E0134802F0CF
:10D48000DDFE08B11120D5E6D4F8403394F80C1134
:10D49000218043F00203C4F8403394F81834114853
:10D4A0000133DBB284F8183484F845340E4B002580
:10D4B0009B6AC4F89854984724E71220BAE60E20D5
:10D4C000B8E600BFA4290020682F0020703000209B
:10D4D000D4290020FC330020D0320020203300204B
:10D4E000843300206A2F00205877030873B5134D4A
:10D4F000134E0096EB6C95F8502095F9781095F83E
:10D50000480003F0F9F995F83031337595F8480083
:10D5100040F2012306F13C023146738203F0F8F930
:10D5200050B196F83C3086F88230064B00205B6B99
:10D530009847F37C86F8A83002B070BDA42900207B
:10D540005033002058770308F8B5324C94F818315E
:10D55000012B05460ED0022B4ED0002B57D138B9E7
:10D56000D4E91B0104F1740383E803000020F8BD33
:10D57000012806D102F02CFB0028F8D184F81851BC
:10D58000F5E7022843D1244E84F8180106F5747C8F
:10D59000BCE80F0006F57A770FC79CE8030094F803
:10D5A000E92094F8003187E8030086F8FB53D2B1F4
:10D5B000022B18D1D4F804316367C6F8EC3394F821
:10D5C0007D3094F8082186F8F83394F88C3084F88C
:10D5D000782086F8F93396F81B2486F8E82340F281
:10D5E0000133A6F8FA33002386F81A340B4BDB6AB2
:10D5F0009847FFF77BFFB9E748B9074B84F8180154
:10D60000062283F89024054BDB6A9847AEE7032097
:10D61000ADE700BFA4290020682F00205877030839
:10D62000F0B5504C504EB4F8DC202287D4E92D01DF
:10D6300094F8B12084F8692004F16C0282E80300B8
:10D64000D4E92F0104F1740282E80300B4F8C42085
:10D65000A4F87C2091B0D4F8CC20D4F8C810C4F839
:10D6600084200025D4F8D020C4F888200123A4F811
:10D670002031C4F8801084F83051A56284F81B5121
:10D6800084F83A5084F81D5184F81E51C4F834517E
:10D69000C6F89854A6F8185486F81A54A4F83851C5
:10D6A0008DF8183004F50973039304F50A7394F8A0
:10D6B0004800049303A92D4B84F84551C4E94F5504
:10D6C000A4F84651059303F0FFF8E36EC6F8D4338F
:10D6D00094F87D3086F8E03394F88C3086F8E133A6
:10D6E0004FF48073A6F8E23386F8D05394F83031C3
:10D6F00086F8E43306F574770FCF06F57A740FC415
:10D7000097E8030040F2012384E80300A6F8FA3307
:10D71000D6F8483386F81B54CDE901551BB15A6839
:10D720005B6901920293124B0793A3F1480208929E
:10D73000A3F1140209920F4A0B9229330A93A2F122
:10D740009C030C93A2F198030D93131D0E9301A952
:10D7500002F14C0307A802F599620F9302F022FA36
:10D7600011B0F0BDA4290020682F00205023002014
:10D77000D0330020882A0020F8B50D4F0D4E0C46FE
:10D7800007F012FB3B6B98470B4A96F8480021467E
:10D7900003F0BEF850B1094D706D95F8243485F84A
:10D7A0006A347B6B9847E37C85F89034F8BD00BF02
:10D7B00058770308A42900208C330020682F00200C
:10D7C0000F4890F81B3480F8B8330E4B93F869205B
:10D7D00080F8BB2393F87D2080F8C82393F88C2031
:10D7E00080F8C92393F8303180F8CC330022A0F8B8
:10D7F000CA2300F56E7100F56070FFF7BDBF00BF72
:10D80000682F0020A4290020114890F89034EBB133
:10D8100090F81B3480F8D0330E4BDA6EC0F8D42366
:10D8200093F87D2080F8E02393F88C2080F8E123A2
:10D8300093F8303180F8E4334FF48072A0F8E2239B
:10D8400000F5747100F56670FFF796BF704700BF72
:10D85000682F0020A429002070B5344C24212046D4
:10D8600004F0A0FF636A984218BF60624FF01C0189
:10D870002F4814BF0125002504F094FF636C9842E3
:10D8800018BF60644FF480712A4818BF45F0020544
:10D8900004F088FFD4F84831984218BFC4F8480112
:10D8A0004FF0D401244818BF45F0040504F07AFF76
:10D8B000D4F82032984218BFC4F820024FF000017B
:10D8C0001E4818BF45F0080504F06CFFD4F8243258
:10D8D000984218BFC4F824024FF46071184818BF6A
:10D8E00045F0100504F05EFFD4F8A835984218BF43
:10D8F000C4F8A8054FF01401124818BF45F02005E0
:10D9000004F050FFD4F8C03598420F4B18BFC4F84C
:10D91000C005D3F8483318BF45F040052BB11B694B
:10D920001BB12846BDE87040184770BDA4290020EF
:10D93000CC290020EC290020F02A0020C82B002050
:10D94000CC2B0020502F0020682F00202DE9F04F15
:10D950008FB04FF00009012B06460F4690468DF818
:10D960000D90ADF8109002D84C46BC4202D30FB0D7
:10D97000BDE8F08F305D02F033FA2044B842F6DCA7
:10D98000335D651C023BEDB2112BF0D801A252F8B9
:10D9900023F000BFDDD9000807DA000805DB000826
:10D9A0002DDB0008ABDB0008D1DB000837DC00080A
:10D9B0005FDC0008E5DC00086FD900086FD90008BB
:10D9C00039DD00086FD900086FD90008E1DD0008D3
:10D9D00009DE000841DE000875DE0008052002F0BF
:10D9E000A7FA70B10521002002F068FA725DBA4B07
:10D9F000E51C0234E4B283F85C24325D83F85D24D4
:10DA0000EDB22C46B1E700238DF80E308DF80F30C3
:10DA10008DF814308DF81830B9F1000F6DD1AF4C7E
:10DA20004FF0050994F87C208DF831206B1E94F896
:10DA300039208DF83320334494F838200B938DF837
:10DA4000342094F81A3194F868208DF83520D4F8F1
:10DA50002C218DF832300A9273B37B1C5B1BDBB236
:10DA60008DF8303006AB019305AB009394F8480075
:10DA70000DF10F030DF10E020AA902F05DFF8DF802
:10DA80000D0000F00700072813D194F939209DF903
:10DA90000E3084F839309A429DF80F3084F83830CF
:10DAA000B8BF01229DF81430B8BF84F81D2184F856
:10DAB00068304FF0000A09E00523D1E701220DF19B
:10DAC0000D01032002F0A4F80AF1010A5FFA8AF2BC
:10DAD0009DF81830B3FBF9F19142EFD82B44DDB239
:10DAE0006B1EDBB29F420BD9F25C032A9AD0AF4285
:10DAF00088BF1D464FF0010983E70534E5B2F9E719
:10DB00001D46F7E7735D754903F00F03012281F8A5
:10DB10001B31023402FA03F3A1F82031E4B20022EF
:10DB200004A9042002F074F825466AE707238DF85B
:10DB30000D30735DC3F3021203F00F038DF828302C
:10DB4000E31CDBB28DF82920F25C231DDBB2651DDE
:10DB5000F35C0234E4B21B0443EA0223325D5F4CFF
:10DB600013436422534394F848000B930AA902F02C
:10DB7000F2FE00F00703072BEDB28DF80D000CD17B
:10DB80009DF8283084F8703084F878300B9BE36679
:10DB900063679DF8293084F869308DF81000012200
:10DBA00004A9052002F034F82BE74B4BD3F8483397
:10DBB00063B11B6853B1984708F03F038DF810001C
:10DBC0008DF81130022204A90620EBE7FF20F3E7CD
:10DBD00003238DF80D30735D8DF81C300AAB06936E
:10DBE000E31CDBB2A51DF25C231DDBB206A9F35CCE
:10DBF0001B0443EA0223A21CD2B20534B25C1343D5
:10DC000064225343E4B20A9300230B93335D8DF8EF
:10DC10003030324B93F8480002F0A3FEC3B2002824
:10DC2000EDB28DF80D30FFF6ECAE8DF8103001221C
:10DC300004A90720B6E7735D03F00F03012B4FF42F
:10DC40007A7238BF01235343244A0234936503F5A3
:10DC50007A73D365E4B2002204A9082062E7735DF9
:10DC60001E4DC3F340128DF8152095F84800C3F3FC
:10DC7000001205A903F00F038DF814208DF816305B
:10DC800002F075FE02340130E4B23FF44DAFBDF84E
:10DC90001430134AA5F87C309DF816309DF814A076
:10DCA000D05CF4F787F90223C5F880000AA995F83B
:10DCB00048008DF828308DF82AA002F0F7FD95F97C
:10DCC0003930069040B29842B8BF184685F83900FE
:10DCD000002204A9092025E7682F0020A42900209C
:10DCE0006370030803238DF80D30735D8DF82830C1
:10DCF000E31CDBB2651DF25C231DDBB20234F35C76
:10DD0000E4B21B0443EA0223325D1343642253430B
:10DD10000B93644B0AA993F8480002F02EFEC3B29D
:10DD20000028EDB28DF80D30FFF66BAE8DF8103097
:10DD3000012204A90A2035E7092002F0F9F8DFF8EA
:10DD400068B1002849D00921002002F0B7F800236B
:10DD5000ADF81E30A31CDBB2F25CE31CDBB216F89C
:10DD600003A0735D4FEA0A4A4AEA022A4AEA030A12
:10DD7000231DDBB2A51D0534F35CE4B24AEA036A55
:10DD8000335D4FF47A7253430AAC1B122046ADF850
:10DD90001C3006F019FF454B53440693DBF83C3327
:10DDA00000930DF1180A9AE80600DBF8383308A84A
:10DDB00006F0C7FE099B009394E80600089B5046B6
:10DDC00006F0A4FE9AE8030006F0D6FE01F00AFF72
:10DDD0000123EDB28BF8383413E68BF8380410E6E3
:10DDE0000C2002F0A5F800283FF40BAE0C21002017
:10DDF00002F064F82C4B93F89034043B012B7FF62F
:10DE000000AE01F0EBFEFCE5A31CDBB2725DF15C41
:10DE1000E31CDBB2651DF35C0434E4B21B04305D2B
:10DE200043EA012313436421594300F00F0001F03A
:10DE3000D6FEEDB28DF81000012204A91120B1E642
:10DE40000D2002F075F800283FF4DBAD0D21002015
:10DE500002F034F8A31CDBB2154AF05C735D126863
:10DE6000251D0334E4B243EA0020315DEDB201F038
:10DE7000B8FEC6E5725DA31C251D0334DBB2E4B217
:10DE8000F15C335D1B0443EA0123134364205843D0
:10DE900001F0A9FEEDB28DF81000012204A91320B3
:10DEA00080E600BFA4290020682F0020803DD51205
:10DEB000382300200E4B93F89124920703D593F852
:10DEC0008F24012A08D90B4991F81A2122B18A6AB4
:10DED000501C18BF01328A620022A3F8182483F86C
:10DEE0001A24D3F8402322F00202C3F840237047DB
:10DEF000682F0020A429002070B5184C1848194D2F
:10DF000006F052FFD4F84033D4F89804D5F8906066
:10DF100023F02003C4F8403338B106F00BFF8642EB
:10DF200003D2002385F83A3070BD0120FFF766F96F
:10DF30000028F9D00B28F7D095F8393084F842340E
:10DF4000092094F8183484F8453484F8410401F029
:10DF5000D7FFBDE87040FFF7ADBF00BF682F0020BE
:10DF6000D0320020A4290020094BD3F84023012AF5
:10DF70000AD008490978C90708D43AB993F8920435
:10DF8000013818BF012070470020704701207047FA
:10DF9000682F00204C230020034BD3F84003431E7E
:10DFA00058425841704700BF682F00202DE9F04FBC
:10DFB000A9B0EFF3108272B6DFF8F0B20021DBF8FF
:10DFC0000030CBF8001082F31088B94C002B00F021
:10DFD000E180DAB29B06039264D5B64D95F818310C
:10DFE000022B02D0B44BDB6A9847EFF3108872B66D
:10DFF000B24F06F095FE3E68D4F8B013361A31449D
:10E00000AF4806F059FFAE4806F01CFFD4F8B41331
:10E01000AC48314406F050FFAA4806F013FF88F3DD
:10E02000108894F81A34002B00F06B81152312A984
:10E0300095F848008DF8483002F038FCD4F8B41355
:10E040000F900144A04806F037FF9F4806F0FAFE03
:10E050003B6894F81B24EB620DAF38468DF87020B6
:10E060001D9306F0D7FDD5F82831009306AE97E84A
:10E070000600D5F82431304606F063FD96E803002B
:10E080001FAB83E80300D4F81C341E9395F830319D
:10E0900095F84800003B18BF01231CA98DF871308A
:10E0A00002F00DFC039BDF0648D5824DDFF81CA271
:10E0B000D5F8E42004929BF80020BAF90A809AF976
:10E0C0000C90A4F88C84002363F300020A9384F874
:10E0D0004434A4F8223484F82534C4F82834A4F84D
:10E0E0002C3484F82E34C4F8303484F82034C4F846
:10E0F000343484F83834C4F83C346F4B8BF8002047
:10E1000094F89024DB6A84F88E9484F88F24DAF8EB
:10E110000470BAF80860984794F88F3413B96948C6
:10E1200006F042FE3146384601F045FD83460028A0
:10E1300000F0EA80A4F87E8484F88094039B190799
:10E140001AD55C4B93F81831022B02D05A4BDB6A7C
:10E1500098470220FEF712FF84F8410401F0D0FE38
:10E1600094F81A3413B1012384F8193494F89134D3
:10E1700043F0100384F89134039B5A0703D506211A
:10E180000520FEF765FF039B9B0703D504210320B1
:10E19000FEF75EFF01F02DFD94F89124D7065FD5C0
:10E1A000002384F89234D4F840331E0644BF23F091
:10E1B0008203C4F8403312F0050F00F0FB820B20FD
:10E1C00001F0B6FE002800F0F58294F89134DD07E6
:10E1D00000F1F082580740F10783D4F8403323F070
:10E1E0000203C4F84033D4F8402382BB94F891541E
:10E1F00015F001011EBF2B4662F3000384F8913431
:10E2000094F891345E0744BF6FF3820384F891342D
:10E21000012384F8923421B1D4F844332C481B688C
:10E2200098476D070BD52B4801F08EFE01F0BCFE20
:10E2300028B194F8913443F0040384F8913401F048
:10E24000C6FC94F891346FF3041384F891340123DD
:10E2500084F8923494F8913443F0200384F8913494
:10E2600094F8913418070AD56FF3C3031A4984F858
:10E270009134D4F84433A1F12400DB68984794F832
:10E28000913499070AD56FF34103134984F8913407
:10E29000D4F84433A1F16C005B68984794F890344B
:10E2A000022B1BD1FFF722F918E000BF4C230020FE
:10E2B000682F0020A4290020587703084823002055
:10E2C000E83200200033002068330020382300208B
:10E2D000A8330020BC330020F433002094F891349C
:10E2E0009A0640F1C4826FF3451384F89134D4F850
:10E2F0004033002B40F0BB8229B0BDE8F04FFFF760
:10E30000ABBA84F84134A3E695F81831012B0CD14F
:10E3100001F055FC804668B1584601F045FC58466E
:10E3200001F047FC042384F88F347EB9012384F87C
:10E3300021344FE101F045FC0028F6D0404601F0C1
:10E3400034FC404601F036FC0523ECE73B780593AE
:10E350005B09013B062B00F21782DFE813F0070090
:10E36000150295001502920015020602102EDDD945
:10E3700095F830311297F6B28DF84C60002BD5D15C
:10E380001CA804F021F912AA1CA9FF2002F09EF893
:10E390009DF85830C3F3030307468DF82C3095F8E9
:10E3A000480095F87D308DF82D3007220BA902F03A
:10E3B00090FA002F5DD100285BD09DF853309DF876
:10E3C00052201599C5F8E4101B0443EA02239DF876
:10E3D000512002201343C5F8E03004F003F99DF802
:10E3E000583095F8480085F82E71C3F30212C3F334
:10E3F000030385F8703085F878309DF8593085F83A
:10E400006920012B38BF01234FF47A725343AB6567
:10E410001344EB650DF15A034FF001081093113EC0
:10E4200094F81B348DF83C300FA985F868808DF87E
:10E43000446002F056FA0223404685F8303101F07C
:10E4400077FD18B14146384601F038FD94F88F3415
:10E45000012B00F2A78194F81A34002B40F09A8126
:10E4600094F8913443F0100384F89134FEF786FD5C
:10E4700064E6012001F05CFD0028E7D001210720BF
:10E48000E2E7012384F8203495F87D308DF82E30B2
:10E4900094F824348DF82D3095F88C3095F8480098
:10E4A0000D330BA98DF82C3002F000FAA6F10D0304
:10E4B0001BB2099023EAE37300B283423FF736AF01
:10E4C0000B2E7FF633AFBA4B25931CA8FF231C9766
:10E4D0008DF874608DF8983002F0C4F80746002873
:10E4E0007FF424AF95F81831012B13D101F067FBAD
:10E4F000002872D0384601F057FB384601F059FB2E
:10E5000004239DF87C101E9884F88F34C1F3001109
:10E5100001F06EFB9DF87C301E99C4F8341413F0A2
:10E520000F0203D09DF89000002862D19DF898005A
:10E53000002861D0002A7FF4F9AE9DF89020002ACF
:10E5400014BF4FF003084FF0020800220A92D5F8DA
:10E55000EC2095F8E900914251D100284FD0D5F830
:10E560000C1195F8EAB009680A9195F8181102297A
:10E5700002D1032184F88F14B8F1030F7FF4D6AED3
:10E5800013F0600F7FF4D2AE0492012795F82E317C
:10E59000BBF1000F36D0BBF1010F13D1012B33D1EA
:10E5A0006FF0090646FA08F606F00106C6F1020603
:10E5B000F6B2BDF87E100AAA304601F011FE38B35B
:10E5C000072823D0012384F821340A9BC4F830346F
:10E5D000C4F86C34FEF720FDB0E501F0F2FA002833
:10E5E00098D0384601F0E1FA384601F0E3FA052305
:10E5F00087E74FF00008A8E74FF00108A5E74FF0C4
:10E60000010BC3E70426D4E70326D2E70823DAE7A1
:10E610001CAB009304990A9B3246584601F0A2FEB7
:10E6200020B1022814BF0B230A2380E60A9BC4F8FA
:10E630003034C4F86C349DF87C3084F82104C3F382
:10E64000401384F82E3484F8443494F88F3484F8DA
:10E650002274012B9EBF0122A86285F81E21012F82
:10E66000C4F8280484F82C0484F8410438D1022228
:10E6700084F8202495F83A20002A4AD19DF87C207D
:10E68000D60646D4012B94F840149DF87C2005D87A
:10E69000012901D1900601D501F04CFBB8F1020F20
:10E6A00094F88F3443D0B8F1030F0AD09DF87C1052
:10E6B000B8F1010F4A4601F00F0120A83BD0FFF747
:10E6C00045F99DF8903084F82334259BC4F828340C
:10E6D0009DF8983084F82C34012384F82D3430E0F0
:10E6E000059A02F0E002A02A1BD195F82E11012212
:10E6F00085F83A2009B927996963012B84F8202409
:10E7000007D9D5F89020C4F83C24DAF80020C4F8E2
:10E71000982495F81821002AB4D1012284F82524E0
:10E72000B0E7002285F83A2084F82024A6E79DF877
:10E73000981025984A46FFF709F99DF8903084F81B
:10E7400023349DF89020E02A08D195F81F312BB989
:10E7500084F82324C4F82834A4F82C3494F8913491
:10E7600043F0020384F8913470E6114D013EB2B2D9
:10E77000791C284604F000F80323A4F82034C4F8D8
:10E78000285484F82C64E9E7012384F82134FEF747
:10E7900043FC5BE694F84434002B3FF461AE002068
:10E7A000FEF726FC94F88F34022B3FF45FAE57E659
:10E7B000A031002094F89134590715D5012001F0BB
:10E7C000B7FB60B1012001F08BFB08B984F8180495
:10E7D000D4F8403323F00203C4F8403304E00620A9
:10E7E00001F0A6FB0028F3D194F89134DA077FF505
:10E7F000FAAC94F840240AB1032A18D11D4A94F8BF
:10E80000181492F86820914205D29B0723D594F8FA
:10E810008F34012B1FD8184806F0C6FAD4F84033BD
:10E8200023F02003C4F84033FFF744FBDBE4012A64
:10E8300011D194F81924002A3FF4D5AC0D4A94F86C
:10E84000181492F868209142E5D29F0703D594F8F6
:10E850004434002BDFD194F8913400206FF304137B
:10E8600084F8913484F81904FFF746FBBBE429B01F
:10E87000BDE8F08FA4290020D03200202DE9F04F10
:10E8800089468DB090460746002800F08F81002908
:10E8900000F08C810368002B00F088814368002B16
:10E8A00000F084818368002B00F08081C368002B16
:10E8B00000F07C81104601F0F5FF002800F078811F
:10E8C000BD4CBE4D384601F0AFFA40F2C4520021B3
:10E8D000204603F065FF40F21C520021284603F059
:10E8E0005FFFB74BC4F82C3104F50973089304F5A6
:10E8F0000A7300264046099308A9B24B84F8488061
:10E900000A9384F8186184F88C608DF82C6001F00B
:10E91000DBFF0F2306A994F848008DF8183001F0AA
:10E92000C5FF801B18BF01204FF00A0B84F81C01A3
:10E9300006A994F848008DF818B001F0B7FF4FF021
:10E94000060A84F8DC0006A994F848008DF818A09F
:10E9500001F0ACFF102384F8DD0006A994F848000C
:10E960008DF8183001F0A2FF1123C4F89C0006A90D
:10E9700094F848008DF8183001F098FF1223C4F87D
:10E98000A00006A994F848008DF8183001F08EFF19
:10E990001323C4F8A40006A994F848008DF8183091
:10E9A00001F084FF1423C4F8A80006A994F84800D5
:10E9B0008DF8183001F07AFF1623C4F8AC0006A9D0
:10E9C00094F848008DF8183001F070FF172384F890
:10E9D000B10006A994F848008DF8183001F066FFE0
:10E9E00018230DEB0301C4F8B400C4F8BC0094F87C
:10E9F00048008DF8183001F059FFC0B21D2384F88B
:10EA0000B80084F8C00006A994F848008DF81830C2
:10EA100001F04CFF1E2384F8C40006A994F84800B6
:10EA20008DF8183001F042FF1F2384F8C50006A9B5
:10EA300094F848008DF8183001F038FF2023C4F80E
:10EA4000C80006A994F848008DF8183001F02EFF90
:10EA50000B23C4F8CC0006A994F848008DF81830B0
:10EA600001F024FF0C2306A9A4F8D00094F8480074
:10EA70008DF8183001F01AFFD4F89C306365D4F893
:10EA8000A030A365D4F8A430E365D4F8A830236699
:10EA90004FF00108D4F8AC300590A4F8D2006366BA
:10EAA00084F8B080C4F894B084F898A0C4F84CB04E
:10EAB00084F850A084F8688084F81F81C5F84893D2
:10EAC000FEF7AEFDC5F84473C4E90B663E4B84F80F
:10EAD000198185F89164C5F8408332464FF0FF31C3
:10EAE000009605F55A7006F001F9384B009632464B
:10EAF0004FF0FF3105F5607006F0F8F8344B0096E2
:10EB000032464FF0FF3105F5667006F0EFF802AFC0
:10EB1000304B009632464FF0FF3105F5806006F02D
:10EB2000E5F8384606F076F897E8030004F59273A6
:10EB300083E80300284B294F1E60294BC5F84C334E
:10EB4000284BC5F85433284BC5F85C33274BC5F820
:10EB50005033274BC5F8583305F553703B68984739
:10EB600004F5A67003F04CFB20B1112630460DB021
:10EB7000BDE8F08F204601F003FB0028F5D101F03D
:10EB800039F8B8B91B4801F04DFB06460028ECD116
:10EB90007B69984703F0CEFDBB6D94F81901984747
:10EBA000FB6A9847012385F89234DFE70326DDE707
:10EBB0000926DBE71326D9E7A4290020682F0020C7
:10EBC0000004000150230020F9DE0008C1D700082E
:10EBD00009D80008F1CF00084C230020587703081B
:10EBE000B1D1000865D10008ADCF00083DD10008C3
:10EBF00015D100088C2A002008B5034B0020C3F86B
:10EC00004003FEF7BBF908BD682F002010B5FFF7E1
:10EC1000ABF90A4C60B90A4B93F81831022B02D1B8
:10EC2000084BDB6A98470123C4F84033002010BD2D
:10EC3000D4F84003013818BF0120F8E7682F0020FE
:10EC4000A42900205877030838B5124C204606F056
:10EC5000ABF804F1180006F0A7F804F1300006F054
:10EC6000A3F804F1980006F09FF800F0AFFF0A4BFC
:10EC70000025DB6A984744F8285CFEF7EDFD07495C
:10EC8000074840F2C45203F077FD012344F8283CC2
:10EC9000284638BDD032002058770308A429002028
:10ECA000E023002070B52E4B8AB0054693F8DD00B6
:10ECB0008DF8090093F8DC008DF80A0029489A6A5B
:10ECC00090F81804039200268DF80B0004960C4669
:10ECD000002940D00692D3F8882007921A8F93F823
:10ECE0001A118DF8151052BAADF8202093F87C2037
:10ECF00093F848308DF8243003AB8DF822008DF85E
:10ED0000232000930DF10A020DF10B030DF109010F
:10ED100005A88DF8146000F0D7FE9DF90900FEF7F4
:10ED20004FF9607004A801F01BF8B0B9049A0F2ADB
:10ED30000DD863789A420AD81544AB42A3EB02017E
:10ED40002CBF002001202170C0000AB070BD00233C
:10ED500023700820F9E70320F7E71320F5E700BF49
:10ED6000A4290020682F00201FB50446002800F0C9
:10ED700010810378412B00F20781DFE813F0420095
:10ED800049004D005100550059005E000501050184
:10ED90000501050105010501050105016500690081
:10EDA0006D0078007F00820085008A0088008C005A
:10EDB00090009300960099009C009F00AE00B20066
:10EDC000BA00B600BE00C100C500CE00CA00CC002B
:10EDD0000501D20005010501050105010501050137
:10EDE00005010501050105010501050105010501F3
:10EDF0000501DA00DE00E200E700EB00EF00F300BF
:10EE0000FC00664B93F818312371002004B010BD4C
:10EE1000624B93F83031F7E7406803F08FFBF4E77B
:10EE2000406803F0D1FBF0E75C4B93F81A31EBE755
:10EE30005A4BD3F8E0306360E7E7584B011D93F875
:10EE4000300103F0D9FBE0E7544B93F81931DBE7CD
:10EE5000524B93F88C30D7E71C238DF808304F4B7A
:10EE600002A993F8480001F021FD6060CDE74C4B0A
:10EE7000043493E8030084E80300C6E7494B0434F4
:10EE8000F7E7494B0434F4E7484B0434F1E71A231D
:10EE9000E3E71923E1E7414B93F86830B4E73F4BD0
:10EEA0005B6DC8E73D4B9B6DC5E73C4BDB6DC2E737
:10EEB0003A4B1B6EBFE7394B5B6EBCE702238DF804
:10EEC0000830364B02A993F87C2093F848008DF85F
:10EED0000A2001F0EBFC207197E7304B93F8DD300E
:10EEE00092E72E4B93F839308EE72C4B93F8DC30B9
:10EEF0008AE72A4B93F8383086E7284BDB6C9AE791
:10EF0000264B93F850307FE7244BD3F8843063606E
:10EF10007BE7224B8FE7264B8DE7204BD3F8CC3095
:10EF2000F5E71E4BD3F82C31436001F04DFDA06096
:10EF30006BE71A4BD3F890307DE7184B93F81F31ED
:10EF400062E7164BB3F88830A3805EE7134BB3F843
:10EF50008A30F9E7114BB3F8D030F5E70F4BB3F82F
:10EF6000D230F1E70D4B93F848200AB1062A12D1AE
:10EF7000B3F8A035E8E7094B93F848200AB1062A10
:10EF800009D1D3F8A43556E704B0BDE8104000F02D
:10EF900021BE03203AE7182038E700BFA42900204B
:10EFA000102A0020582A0020182A0020602A002059
:10EFB000E02300207FB5044610B9032004B070BDE3
:10EFC000A34DD5F840339A0700F16F820278412AA9
:10EFD00000F26882DFE812F04200470055005B0053
:10EFE0005F00640069007600810087008D00930057
:10EFF00099009F00A500AB00B5006602BA00DC00D6
:10F00000EF0016013801290142014B014F01530164
:10F0100057015B0166025F01710199018701AB0134
:10F02000B101B801BD01C201660228026602660292
:10F030006602660266026602660266026602660290
:10F0400066026602660266026602660234023902DF
:10F050003E02430248024D0252025C020079FEF772
:10F0600073FA30B1AAE70379022BA6D0794A82F865
:10F07000303195F8913443F0200385F89134002025
:10F080009CE7406803F04CFA0028F2D095E740680E
:10F0900003F08AFAF8E76F4B027983F81A21E8E760
:10F0A0006C4B4268C3F8E020E3E76A4E416896F88B
:10F0B000300103F097FA00287FF47FAF6368C6F849
:10F0C000E430D6E7416800293FF477AF002001F033
:10F0D000DDF90028CDD0112070E7416800293FF408
:10F0E0006CAF0120F3E7416800293FF466AF0820C8
:10F0F000EDE7416800293FF460AF0920E7E7416888
:10F1000000293FF45AAF0C20E1E7416800293FF4A1
:10F1100054AF0D20DBE7416800293FF44EAF0E20CD
:10F12000D5E7416800293FF448AF0F20CFE74A4CAC
:10F13000484B007983F81901A36D9847E36A984713
:10F1400097E7444B027983F88C2092E7414E037A8B
:10F150008DF8043096F8480096F87D308DF805302B
:10F16000072201A901F0B5FB00283FF426AF636830
:10F1700096F848000193002201A901F0AAFB00289B
:10F180003FF41BAF6C36D4E9010186E8030070E759
:10F19000304E037A8DF8043096F8480096F87D30AA
:10F1A0008DF80530072201A901F093FB00283FF4F8
:10F1B00004AFB436E7E7274E037A8DF8043096F8AB
:10F1C000480096F87D308DF80530072201A901F03E
:10F1D00080FB00283FF4F1AED4E9010106F174038D
:10F1E00083E8030096F81831022B7FF442AF96F8BB
:10F1F0003031002B3FF43DAF174BDB6A9847FEF7E9
:10F2000075F936E7134E037A8DF8043096F8480006
:10F2100096F87D308DF80530072201A901F059FBE1
:10F2200000283FF4CAAEBC36ADE743680293012321
:10F230008DF80C30074B02A993F8480001F056FBFB
:10F2400000287FF416AFB8E6436802930023EFE787
:10F25000682F0020A42900205877030803795A1E3C
:10F260000E2A3FF6AAAE934A82F8683001E7914B26
:10F2700042685A65FDE68F4B42689A65F9E68D4B08
:10F280004268DA65F5E68B4B42681A66F1E6894B0F
:10F2900042685A66EDE6874C037994F848008DF889
:10F2A0000430062201A901F014FB00283FF485AECA
:10F2B0009DF8043084F8DD30DBE67E4C03798DF870
:10F2C000043094F8480094F87C308DF8063005221C
:10F2D00001A901F0FEFA00283FF46FAE9DF804305A
:10F2E00084F83930C5E6734C037994F848008DF8FA
:10F2F00004300A2201A901F0ECFA00283FF45DAEC7
:10F300009DF8043084F8DC30B3E66A4C037994F855
:10F3100048008DF80430092201A901F0DAFA00282A
:10F320003FF44BAE9DF8043084F83830A1E6614BD1
:10F330004268C3F89420DA649BE65E4B027983F856
:10F34000982083F8502094E65A4B4268C3F88420F2
:10F350008FE6584B4268C3F8CC208AE6012B40F078
:10F36000A480554C2421204603F01CFA636A98427D
:10F3700001D0172022E61C2104F1280003F012FA24
:10F38000636C9842F5D14FF4807104F1480003F0AA
:10F3900009FAD4F848319842EBD1D42104F5A6708B
:10F3A00003F000FAD4F820329842E2D1002104F5AB
:10F3B000097003F0F7F9D4F824329842D9D14FF408
:10F3C000607104F50A7003F0EDF9D4F8A83598429D
:10F3D000CFD1142104F2AC5003F0E4F9D4F8C035D5
:10F3E0009842C6D1334E2146304640F2C45203F013
:10F3F000C3F9204640F2C452002103F0D1F995F838
:10F400001B3485F8E833736FC5F8EC3396F87D301C
:10F4100085F8F83340F20123A5F8FA33274B96F824
:10F4200019019B6D984724E68379012B3FF6C5AD02
:10F43000204B42684068C3F82C2100F0BDFE48E62E
:10F440001C4B4268C3F8902013E61A4B027983F8EC
:10F450001F210EE6174B8288A3F8882009E6154B7A
:10F460008288A3F88A2004E6124B8288A3F8D02071
:10F47000FFE5104B8288A3F8D220FAE50D4B93F8F4
:10F4800048200AB1062A12D1A288A3F8A025F0E5E7
:10F49000084B93F848200AB1062A08D16268C3F8DD
:10F4A000A425E6E500F098FBDBE5012086E51820C1
:10F4B00084E500BFA4290020E0230020587703083A
:10F4C0002DE9F04387B00023ADF800300646002850
:10F4D00000F0EE800361FEF747FD20B101242046D5
:10F4E00007B0BDE8F08300F065FD0028F6D100F01C
:10F4F0005BFD014618B96F48142203F051F96E4DB7
:10F5000095F89134012243F0040385F8552485F8D9
:10F51000913433788DF804300021013B8DF80520BB
:10F52000ADF806100C2B00F2BB80DFE803F007B942
:10F53000B9B97982B9B990B9AD9AA900D5F8407333
:10F5400017F02007CAD196F80480B8F1020F46D10F
:10F55000DFF868815A4CFEF763F896F9051098F8C1
:10F5600048003A4601F00FFA88F83900B37988F874
:10F570003830384607238DF80530FDF7E5FFFF23C7
:10F5800004F58670A5F80C31C5F8084185F80471BA
:10F5900003F01AF804F58A7002F0D0FF3846FDF740
:10F5A0002DFE0446002839D096F9051098F8480039
:10F5B000012201F0E8F988F83900D5F89434336174
:10F5C000002C71D000F0F0FC002888D195F891341F
:10F5D00085F81A0460F3820385F891347FE7B8F167
:10F5E000010F4FF00204E8D1DFF8D0908DF81440FD
:10F5F00099F8480089F81D7102A901F065F933797D
:10F6000089F830318DF805708DF80680FDF7C4FC5F
:10F6100095F8913443F0100385F891340024CCE739
:10F6200000226946022000F0F3FA0028F6D01324E5
:10F63000C3E7244BB288DB6B96F90C10B06898478F
:10F64000D5F8403343F00203C5F84033E6E702A99A
:10F650000D2000F053FB0028E0D0002269460D2069
:10F66000E1E7164B93F81831D3B9347904F0070069
:10F6700000F0ABFA8DF80040012269461020D2E775
:10F68000002269461220CEE78DF8072000F08EFA9E
:10F69000044638B900F087FA204600F089FABDE741
:10F6A00002248AE7012488E701A800F0D1FB16E7CD
:10F6B000032414E7BC330020682F0020A429002075
:10F6C0006A2F0020587703082DE9F04F99B0804643
:10F6D000059118B9032019B0BDE8F08F002303612C
:10F6E000FEF742FC0446002840F0A58046460FCEB7
:10F6F0000EAD0FC51422524898F800A0B8F80C704F
:10F7000098F90EB04F4E214603F04AF84E4B0122B5
:10F7100083F8412496F83021022A25460BD196F829
:10F720001821022A07D196F81E2122B9BAF1010F39
:10F7300038BF4FF0010ABAF1010F2BD0BAF1030F15
:10F740002AD0BAF1000F33D102229DF83C30DDF807
:10F750004090029362F34715012496F87C108DF8CF
:10F76000321002220CA996F848008DF8302001F0E2
:10F770009DF896F81A3196F830C196F81D1140B2EE
:10F78000002B63D0BCF1010F57D1002955D1002CBB
:10F7900061D153E00422D8E70023DDF83C90BDF8A6
:10F7A00040709DF942B0029365F01F050124D4E733
:10F7B0004FF0000BD946CDF808B0CEE74FF001006E
:10F7C00084F81A04D2E005F29A420BA900F0D4FAA8
:10F7D000002800F015811320049B33871A4B002268
:10F7E00083F81A2423E105F29A452A460BA900F072
:10F7F000C3FA0028EFD10B9B84F82801C4F82C51E0
:10F8000084F83031FCE0B9F1000F00F0F980002AF3
:10F8100000F0F6804946E01C02F0AEFF94F8373263
:10F8200001332380ECE01220D6E70220D4E7072042
:10F83000D4E71320D2E701204DE7FCB90220F6E01F
:10F84000A8330020A4290020682F0020002CF5D028
:10F850005845B8BF584696F87C308DF820000522F0
:10F8600096F848008DF8223008A901F032F80028F7
:10F870003FF430AF9DF8203086F839306F4A704B36
:10F88000D2F89804D3F8904038B105F053FA6C4B95
:10F8900084423CBF002283F83A20198F1A8F93F8D4
:10F8A00030010491996A099152BA0028BFD093F8A7
:10F8B0001B0100B9186393F81801ADF858200138FE
:10F8C00093F87C2093F81A411491D0F1000BD3F8EF
:10F8D00088108DF85B204BEB000B93F8482093F8D1
:10F8E0003A0093F868308DF85A3009AB0093554BC5
:10F8F00003904FF001008DF84C0015918DF85C20BD
:10F90000A3F12F01A3F1300213A88DF84D4000F0B0
:10F91000DBF8039B4FEA0B1B4BEA431B00264BEA29
:10F92000801B4BEAC413B145444C039308BF3746D0
:10F930003A46494604F59C70CDE90A669B46268006
:10F9400084F81A6402F018FFE9B2A570C5F34215F5
:10F95000FAB2042D3A4E039B84F837223FF42EAFBF
:10F96000072D3FF450AF022D7FF45FAF364D84F882
:10F970000D110420029984F80401FF2084F80C0181
:10F9800084F8281184F81431D6F8E410C4F808512A
:10F9900005F59B730AA8C4F8101184F83021C4F847
:10F9A0002C3100F011FC00287FF43DAF0A9BA4F835
:10F9B00044040BA8A4F81631C4F84C3400F0D0F974
:10F9C00000287FF408AF0B9BD3B196F93900FDF7FF
:10F9D000F7FA94F83732002B3FF405AF0B9B0F2B4F
:10F9E0003FF6F1AE05F58B720BA90F2000F0C4F9BC
:10F9F00000287FF4F0AE0B9B63F3030B84F814B183
:10FA00000598FDF7FBFB00287FF4E6AE099B86F81E
:10FA10003A00B36200F080F900287FF40AAF94F84E
:10FA2000913484F840A443F0010384F89134034BEB
:10FA3000D3F89434C8F810304DE600BF682F00208A
:10FA4000A42900200C2A00206A2F002037B50B4D76
:10FA50008DF8040004460F2295F8480001A900F033
:10FA600038FF40B1064A85F81C4192F8913443F0C2
:10FA7000200382F8913403B030BD00BFA4290020D8
:10FA8000682F002010B5FFF7C1F8044688B90A486E
:10FA900005F08AF9094805F087F9094805F084F965
:10FAA00000F094F8FDF7BCFD064BDB6A9847204652
:10FAB00010BD0124FBE700BFD0320020E832002057
:10FAC00000330020587703082DE9F04F8BB04778BA
:10FAD0000093149B90F90C8090F90D6090F80EB093
:10FAE0008A464168196004469146002F58D0022387
:10FAF0008DF8103004A9C37B007C8DF8123000F023
:10FB0000D5FEB4F808C0618943B26068984545469F
:10FB10006144B8BF1D46604534BF002701278842B5
:10FB200009D30A218DF81010207C019304A900F05C
:10FB3000BDFE019B46B2B4F808C0608961680CEB59
:10FB4000400E714519D3A1EB0C01B1FBF0FC00FB99
:10FB50001C1191B9984503DC2378CBB94FF0010B08
:10FB600021238DF81030207CE37B8DF8115004A9FF
:10FB70008DF8123000F09AFE45B2009B8AF80050D2
:10FB8000384689F8006083F800B00BB0BDE8F08F0C
:10FB90000223207C8DF8243006A900F095FEDDE7D5
:10FBA0004546EAE770477047704770470020704746
:10FBB0007047704770470020704700207047002052
:10FBC00070470020704700207047704770477047AB
:10FBD00002207047022070470220704770470020C3
:10FBE000704770477047002070470020704770478B
:10FBF0007047704710B5054C4FF403722046002142
:10FC000002F0CEFD0020C4E9000010BD84340020C5
:10FC10002DE9F8438146904600293CD01F4C202313
:10FC2000224604F1100012F8017F6FBB8242FAD124
:10FC30001B4E3368013403B93460736803B11C6030
:10FC400000252560C4F8088074601FFA88F284F8E3
:10FC50000490601D02F090FDB9F1110F4FF0000308
:10FC600098BF104D6373D6F8083298BF25FA09F58E
:10FC700003F1010398BF05F0010543442573C6F85D
:10FC800008323846BDE8F883013B13F0FF03044611
:10FC9000C6D10227F5E70127F3E700BF8B34002028
:10FCA000843400202007020010B518B3124A1368EC
:10FCB000984204D103681360002305E00B46002B33
:10FCC000FAD019688842F9D15168884208BF536058
:10FCD0000BB101681960D2F808328168013B002439
:10FCE0005B1A04602146C2F80832102202F058FD67
:10FCF000204610BD0120FCE784340020054B1B6822
:10FD000013B11A798242FAD1002B0B600CBF032089
:10FD1000002070478434002010B5054B186800B9E6
:10FD200010BD037B04680BB9FFF7BEFF2046F6E762
:10FD30008434002038B5084B084C186800B938BD29
:10FD400003790568112B05D824FA03F3DB0701D5E5
:10FD5000FFF7AAFF2846F1E78434002020070200BD
:10FD600028B1044BD3F8083203600020704701200B
:10FD7000704700BF843400202DE9F04107460E464D
:10FD8000154642B339B3154B1C6800232CB93046D5
:10FD9000FFF7E6FF0020BDE8F081A268F91A013202
:10FDA000914215D32279EA54581C22895FFA80F8CF
:10FDB000611D55FA80F002F0DFFCA36824689844C6
:10FDC0005FFA88F3E2E720462568FFF76DFF2C46CF
:10FDD000002CF8D1DBE70120DDE700BF84340020F0
:10FDE0000238C0B211289ABF014B185C002070473E
:10FDF0007370030830B50B4B93F820200446084677
:10FE000072B100211C330578A54208D00131984217
:10FE1000CDB214BF04301038AA42F4D8002030BD4F
:10FE20001046FCE79036002010B5084C00232060F7
:10FE3000142204F10C00FF2184F82030C4E90100F1
:10FE400002F0AEFC012384F8213010BD9036002072
:10FE500010B50E4A92F82010042915D8936804783A
:10FE60001C7044785C70C478807898700131DC70C4
:10FE700082F8201002F11C018B4214BF043302F1FE
:10FE80000C039360012010BD0020FCE79036002099
:10FE9000094B93F8200068B15A6803F11C018A42AB
:10FEA00000F1FF3014BF043203F10C0283F820008C
:10FEB0005A600120704700BF9036002010B5074BF4
:10FEC00093F820200446084632B15968FFF792FFA4
:10FED00010B101234470837010BD00BF9036002024
:10FEE00008B5064B93F820202AB15968FFF782FF26
:10FEF00008B1407808BD0120FCE700BF9036002023
:10FF000030B50A4A92F82010536882F8210061B196
:10FF1000916801241C32DD78587005B99C709342B9
:10FF200014BF0433103B9942F5D130BD9036002008
:10FF300008B5044B5968FFF75DFF003818BF012072
:10FF400008BD00BF90360020F7B50422154E0446C8
:10FF500000210DEB020096F8207002F021FC002534
:10FF6000EBB29F4201D803B0F0BD736819782170DD
:10FF70005A786270987838B1336820469B68984701
:10FF8000FFF786FF0135EBE7DB788DF804108DF87D
:10FF900005208DF80730FFF77BFF01A8FFF758FF1A
:10FFA000F0E700BF90360020014B93F82000704727
:10FFB00090360020034B93F82000042894BF0020C3
:10FFC00001207047903600201FB50024CDE902447F
:10FFD000C41F8DF800408DF801100C0AADF8042004
:10FFE000090C120C8DF803108DF806208DF80730DF
:10FFF00002461B0A012168468DF802408DF8083040
:020000040801F1
:1000000002F029FA002818BF0E2004B010BD2DE917
:10001000F04188B090460D460F9A0746002847D019
:1000200000240121CDE904448DF810109DF838100A
:100030008DF81510ADF81630190CCDE900441B0EE3
:10004000CDE902448DF81930ADF81A20130C120EC8
:1000500007948DF818108DF81C308DF81D20E3B230
:100060001E01002DF6B203DC002008B0BDE8F081CF
:10007000013310218DF81F3042466B460DEB010015
:1000800002F07FF90346A8B9102D28463E44A8BFC8
:1000900010206946327811F801CB013382EA0C0254
:1000A000984206F8012BF5DC103D2DB20134D6E75D
:1000B0000920DAE70E20D8E70138032815D8DFE851
:1000C00000F002080C100A4B1B681B690B60002033
:1000D0007047074B1B685B69F8E7054B1B689B691A
:1000E000F4E7034B1B68DB69F0E70520704700BFAE
:1000F000B43600202DE9F041C4B00C464A9E1746A4
:100100001D468046B8B3B1F5807F36D84FF488726B
:100110000021684602F044FB492300934FF48073AA
:10012000ADF804302B0C8DF80830330CADF80650C8
:10013000ADF80A608DF80C3022460023414604A831
:100140002D0E360E8DF80E308DF809508DF80D609D
:100150008DF80F4002F010FB04F110014B9A3B4662
:1001600089B2684602F0F7F810B1012818BF0E20D6
:1001700044B0BDE8F0810920FAE70D20F8E700005F
:1001800010B590B10A4C28220021206002F008FB33
:100190002368084A1A6000204FF0FF32C3E90302C7
:1001A000C3E90522C3E9072210BD0820FCE700BF10
:1001B000B436002000010101024B1B6818600020CA
:1001C000704700BFB436002030B1044B1B68DB68B9
:1001D000013303600020704709207047B4360020C7
:1001E00013B500230C460193CAB101A9FFF764FFC0
:1001F00018B9019B591C02D1146002B010BD99B20C
:10020000611A002901DD5C18F6E702D113600720AE
:10021000F3E71B0C1B0403F580331C44ECE70920B7
:10022000EBE7000028B1044B1B681C33436200203D
:1002300070470920704700BFB43600201FB5044640
:1002400000B3002303A8039302F05CF9104ABDF841
:100250000C30126820469380E38200F05EFA98B971
:1002600004F11803009321680123132202F068F8B7
:1002700060B9204600F051FA003818BF0120000193
:1002800004B010BD0920FBE71020F9E70E20F7E7C6
:10029000B4360020F0B5054687B01C4613B90920D6
:1002A00007B0F0BD2E4E3368DB68834255D894F812
:1002B0002020002A0CBF08220922834205D32046B1
:1002C00000F05FFA68B11020EAE700230190009384
:1002D000A36894F82810606AFFF799FE0028EED012
:1002E000DEE723792168B4F808C0A768043B9AB216
:1002F0000029D4D0B2F5807F2DD8ADF80EC08DF88E
:1003000017304FEA174C04F12C033F0E8DF8117093
:1003100000932F0C08234FF0490EADF80C008DF818
:1003200014708DF816002F0E0DEB0300CDF808E0C9
:100330008DF810C0ADF812508DF8157002F000F86D
:1003400008B10E20ACE7204600F01BFA0028BAD115
:100350003368DD60A4E70D20A2E70620A0E700BF18
:10036000B43600202DE9FF410A9D80460F4616460F
:100370001C46002D5AD0002303A910460393FFF713
:100380009BFE18B1062004B0BDE8F081039B9C429F
:1003900001D80133F6D1284600F064F9002847D18E
:1003A000264B1A78424503D01A79424542D10120A2
:1003B000AA68BA4240D103EB8002EB6A92F801804E
:1003C0002979CDE900430439927828683B4689B2FF
:1003D000FFF790FE0028D6D195F820300194002B2D
:1003E0004FF00103009314BF4246082295F82810ED
:1003F000686A3B46FFF70BFE0028C4D1013E032E7E
:10040000C1D8DFE806F002070B0F0D4B1B681C611B
:100410001C62B8E70A4B1B685C61F9E7084B1B6874
:100420009C61F5E7064B1B68DC61ACE70920AAE795
:100430000F20A8E70B20A6E70220A4E72404002051
:10044000B43600201FB50B294FF00003CDE900336F
:10045000CDE902330A4607D00C2914D00A2910D05E
:100460000A2005B05DF804FB012802D120238DF895
:1004700000300021684601F0EEFF002818BF0E2072
:10048000EFE73023F3E70B21F4E7000038B505462A
:1004900001F0DCFF044610B10E24204638BD002DCB
:1004A000FBD1094B1B680B219878FFF7CBFF002885
:1004B000F2D10C21FFF7C6FF0028EDD10A21FFF78A
:1004C000C1FF0028E9D0E7E7B43600202DE9F0436A
:1004D00080468FB00C461746002A6BD0002969D0A1
:1004E000002529461D2206A805951DF091FF8DF8CF
:1004F0001350344D2B680DF114099E88CDF80490EB
:100500000DF1130302933B7900933B683246214679
:10051000404601F0BCFF00284ED138683A79494680
:1005200002F02AF9384600F04FF8002846D13C7A0C
:10053000FA79BB79240444EA02241C432B689A68A4
:1005400094423DD99C609DF813000B21FFF77AFF80
:10055000034658BB0C21FFF775FF034630BB0A2149
:10056000FFF770FF034608BB7B7ABA7AFF7A3F0435
:1005700047EA02271F433A46334621460920FFF740
:1005800023FD034690B933463A4621460820FFF73B
:100590001BFD034650B92A689DF813109170002185
:1005A000D1604FF0FF31C2E90411916118460FB0DC
:1005B000BDE8F0830923F9E70E23F7E70F23F5E7FA
:1005C0000323F3E7B436002010B50446002845D0D5
:1005D0000168002942D011F8013B43710322063023
:1005E00002F0CAF82046032250F8091B043102F039
:1005F000C3F82168CB79E3600A7A43EA0223E36017
:100600004A7A43EA0243E3608A7A43EA0263E36098
:10061000CB7A23740B7B63742379212B1AD110229C
:100620000D3104F1120002F0A7F81D222168501CC0
:100630008B5C6362085C43EA0023901C6362085C85
:10064000033243EA004363628A5C43EA0263636203
:10065000002010BD112B03DC0D22E7E70220F8E794
:100660000120F6E710B50446002854D0016800299F
:1006700051D00B7843714B7883608A7843EA022328
:100680008360CA7843EA024383600A7943EA0263DB
:1006900083604B7903738B79C381CA7943EA022360
:1006A000027BC38102F00F020831103002F064F8BF
:1006B000237B002203F00F0384F8202084F82820F5
:1006C000227903F10800111A04290DDD216809338C
:1006D000043AD21A085C84F82000D2B2606A84F826
:1006E0002820194402F048F8237922681A4400208F
:1006F00012F8043CE36212F8031C43EA0123E362AC
:1007000012F8021C43EA0143E36212F8012C43EAA7
:100710000263E36210BD0220FCE710B5044660B33B
:10072000036853B30279162A29D942791A7001460F
:10073000082251F8060B013002F028F82146082261
:1007400051F80E0B093002F021F82368E28A5A743E
:10075000E38A22681B0A93742368A269DA74A36986
:1007600022681B0A13752368628B5A752368E27E20
:100770009A7517232371002010BD0120FCE7022089
:10078000FAE738B50446002863D00168002960D034
:10079000037B90F8282003F00F03002A57D1083379
:1007A000207904321344984255D363790B7023683F
:1007B000A2685A70A36822681B0A93702368628932
:1007C000DA702368E27A1A712368227B5A712368EF
:1007D000E2899A71E38922681B0A2146D371227B40
:1007E00051F8100B02F00F02083001F0C5FF237B17
:1007F00094F8282003F00F0303F108052AB12268BA
:1008000094F82010515503F10905206894F8282028
:10081000616A284401F0B0FF94F828302268E16A48
:100820002B44D1545A1CE16A206892B2090A8154BF
:100830009A1C2168E08D92B28854DA1C216894F8E1
:100840002F0092B2043388542371002038BD09333D
:10085000A6E70120FAE70220F8E70000024B1A8819
:1008600010431880704700BFB836002008B5074B0A
:100870001B883BB1FEF7CAF9002814BF6FF00200D5
:10088000002008BD6FF00100FBE700BFB836002074
:1008900010B5034B00241C80FEF7AEF9204610BDB6
:1008A000B8360020B0FA80F04009704782B018B91D
:1008B000084602B000F0CAB8002002B0704710B974
:1008C000084600F079B9704710B9084600F090B9B1
:1008D00070470346084611460BB900F0DDB9002009
:1008E000704710B9084600F039BD704710B9084686
:1008F00000F0FEB90020704710B4044608461146C7
:100900001A46019B14B910BC00F00CBA10BC704719
:100910000346084611460BB900F036BA002070476E
:1009200010B40446084611461A4614B910BC00F02B
:10093000A3BA002010BC704730B4054608461146E3
:100940001A46DDE902341DB9029430BC00F022BB26
:10095000002030BC704710B9084600F0D3BB00201F
:10096000704710B9084600F037BD0020704710B935
:10097000084600F0E2BB0020704710B9084600F0BE
:10098000DFBB002070470346084611460BB900F054
:10099000F9BB0020704710B40446084611461A46B9
:1009A000019B14B910BC00F0EFBB092010BC7047CC
:1009B00010B40446084611461A4614B910BC00F09B
:1009C0002DBDC8B210BC704700487047010001023D
:1009D000064B10B51B6A0446984730B10448054BD6
:1009E000204498428CBF0020012010BD5877030896
:1009F000403576C9405DC600F0B5114B85B00C4658
:100A000010491F56054601F017F80F4BE4B25E6A15
:100A1000072D4FF00103CDE9024301460AD105221B
:100A20000023CDE900234FF47A727A431846B04789
:100A300005B0F0BD08220020CDE900203A46F5E7D8
:100A40004071030820710308587703081FB500237D
:100A500000930378013B372B21D8DFE803F01C24F7
:100A60002020201E202020204143454E2055585B49
:100A70005E6164206C1E6E73787A7D207F832620F1
:100A800020202020202020202020202085878C202E
:100A900020858C208E92C3780BB10223009300989E
:100AA00005B05DF804FB8378F6E743788DF80430F1
:100AB00007238DF805308378003B18BF01235B00C6
:100AC0008DF8063010238DF80730314B1B6801A8D4
:100AD00003F55872CDE9022300F08EFF0090DEE7A7
:100AE0004023DBE72023D9E7827890F9013012B95F
:100AF000284AD35CD2E7284AFBE7827890F9013094
:100B0000002AF8D1254AF4E740F6B833C6E74FF497
:100B10007A73C3E74FF4FA63C0E741F28833BDE765
:100B200041F27073BAE71E484FF47A7101F008FE83
:100B300000F5FA60D2E71B4BB0E7154B1B6803F5D5
:100B40005873ABE7124B1B6803F55B73A6E71023E2
:100B5000A4E70F4B1B68A1E701239FE74FF08343F6
:100B600000939CE7104BFBE7104B97E740F2111303
:100B7000ADF8003093E7032390E790F901300C4A79
:100B8000B7E70C4990F9010000F056FFA6E700BF57
:100B9000C036002015710308057103080D710308A4
:100BA00018FCFFFF00EA06379A99094040F7093719
:100BB000407103082071030837B50B4B02781B689E
:100BC0000C2101FB02335B7A03EB4304074B1D68E6
:100BD00003690093C3684278816805EBC40000F0A4
:100BE000A7FC03B030BD00BFC0360020BC360020DB
:100BF00030B587B0027B6423ADF80030012A4FF096
:100C00000003CDE90133CDE903338DF802308DF8CF
:100C1000143028D0022A2FD01ABB03680BB34368C4
:100C2000FBB11A4C80682360194B18226946186082
:100C300001F0A2FD174B246893E807000C3384E809
:100C4000070093E8070004F10C05032385E807007B
:100C5000A4F86C33012204F55B7104F5587000F0C0
:100C600058FC07B030BD094908684360036100F5CE
:100C70005B7100F55870F2E7044B1B68B3F8602312
:100C8000B3F86C130A43A3F86023EAE7C0360020E8
:100C9000BC360020301A030808B503460A2924D8B8
:100CA000DFE801F006232323230B161B2321210059
:100CB000BDE808400068FFF78BBE90F90000997806
:100CC000072271B900F0E5FB003818BF012008BD0C
:100CD000052293F900000021F4E790F9000059780B
:100CE000EEE70221EEE70722F3E70020EFE700003E
:100CF00008B502791AB1012A0BD0002008BD084BB3
:100D000001681B68012203F5587000F002FC012005
:100D1000F4E7034B01681B6803F55B70F5E700BF60
:100D2000C0360020F7B50728144D1C46A8BF072081
:100D300058700E462946174600F07EFE94F90130A1
:100D4000A070072B13D1322000F076FD0C4BDB6D29
:100D50000546984704F10C020834034601920094BA
:100D60003A463146284600F06CFD03B0F0BD054A16
:100D700055F82310D05C00F057FDE7E72071030819
:100D800058770308407103082DE9F04F344F90F96C
:100D900001607B68D0F804908BB004468846984781
:100DA0000546002859D1E37C73B92E4A237812688E
:100DB00003EB4303990002EB8303D3F80490B9F1EA
:100DC000000F01D152F80190274B484613F906B0A5
:100DD000FB689847A37C2289D7F818A00993072EAF
:100DE00028D100230121CDE90223204A0693CDE931
:100DF0000431CDE907330521CDE900214FF47A72A2
:100E000002FB0BF24CF250311846D047637C13B30F
:100E1000174B995D7B6D0D31C9B228469847E07C30
:100E20003246494600F01AFE88F8006001200BB0F7
:100E3000BDE8F08F002101250823CDE90013CDE99D
:100E40000715CDE90511CDE903110292A1782B46D2
:100E50005A462846D9E7074BDBE70020E7E700BF03
:100E600058770308C036002040710308854501000B
:100E70000D710308157103082DE9F04F8DB090F93D
:100E80000130DFF8FCA0DFF8FC90CDE90A123E4A01
:100E900012F903B00278DAF800300C2505FB0233B2
:100EA0003A4A5B7A126803EB430302EBC30304463E
:100EB00093F9021090F9020000F0B9FD344906469A
:100EC00094F9010000F0B8FDA268616880463046E0
:100ED00000F0DFFC2178DAF80020D9F80C30694303
:100EE000074650589847D9F81C309C4694F9013071
:100EF0000025072B4FF47A63CDE90753CDE905555B
:100F00002DD10123CDE903530523CDE901534FF43E
:100F10007A7303FB0BF300933946434646F2A8125B
:100F200028466746B8472378DAF800200C214B435F
:100F300094F90110D05800F0B3FDA18994F9010093
:100F4000FFF75AFD0B9B217B1860D9F854302846D7
:100F500098470A9B01201E700DB0BDE8F08F01205C
:100F60000823CDE90350CDE901032A46CDF800B0AE
:100F7000654643463946A84701200546D3E700BFEA
:100F8000C03600205877030840710308BC360020A3
:100F9000207103082DE9F04F8FB0002405468A46E2
:100FA000914698460494ADF81440ADF802400726E7
:100FB0004FF0010B2B7AA34206D9686804A920449C
:100FC00000F0CAFB00285DD102238DF8083002A88A
:100FD0006B7A8DF80A30FFF739FDAB7A8DF81D304A
:100FE0009DF811308DF81E309DF812308DF81F30AD
:100FF0009DF810308DF82030EB7A8DF821302B7B66
:101000008DF822306B7B8DF8233010238DF81C6017
:101010008DF824303A4E8DF82C000DF102030A931E
:10102000072332688DF82D30ADF834302B680C92E0
:1010300006930DF1120204AB0DF1110106A800F0A8
:10104000A5FB072805460BD130680C22002100F5CE
:10105000587001F0A5FB3368BDF80220A3F86023A7
:101060009DF811308AF800309DF8123089F8003070
:101070009DF8103088F80030189B28461C700FB07F
:10108000BDE8F08F9DF81330BDF81470ADF8027014
:101090002044C4B2F3B917B3194A002011680726D7
:1010A00002464FF00C0C062B1BD10CFB00FE51F836
:1010B0000EE0BEF1000F04D00BFA00F23A4397B2F3
:1010C000012201301028EED1002A3FF473AFADF8B1
:1010D00002706FE75A1E042A01D9062BDCD00626BF
:1010E00068E747FA00FE1EF0010FEAD00CFB00FE95
:1010F00051F80EE0BEF1000F08BF0626E1E700BF81
:10110000C036002038B505464068FFF761FC07226D
:10111000841D002195F90000E4B200F0BAF908B985
:1011200004F0FD0495F901000722002100F0B1F957
:1011300008B904F0FB04204638BD002070470000C9
:1011400010B503780F2B044618D84068FFF740FC11
:1011500022780B4902EB42020968831C01EB8200F2
:1011600051F82220DBB21AB903F0FD0358B210BDCA
:10117000032B06BF626842600223F7E70020F6E710
:10118000C0360020022070472DE9F0413A4D044658
:10119000286896B00E46904600211F460122032380
:1011A00000F55870CDE90411CDE906118DF80C1049
:1011B0008DF80D10ADF80E3000F08DF930B92A68B9
:1011C000B2F8603343F00303A2F860332A68637A0D
:1011D0008DF8203002F55871CDE90912274A94F9AB
:1011E000083012680B921022ADF830200DF10E027B
:1011F0000D9222680E9262680F92D4E90301A27ADE
:101200008DF8402001228DF8412011AA82E80300C8
:10121000227DE18A8DF8213018468DF84C20FFF7A9
:10122000EBFB08AB15930DF10D0314900093CDF873
:10123000048003AB04AA39460EA800F099FB0446CB
:1012400078B99DF80C10013901F07AFA00F15803D1
:101250000DEB030010F8483C3370204616B0BDE893
:10126000F0810C2801BF2A68B2F8603343F0030311
:10127000A2F86033F1E700BFC0360020BC36002082
:10128000F8B50679012E054648D90F2E48D80368CF
:10129000187A40F303000722002140B200F0F9F869
:1012A0002B680446187A40F303100722002140B24D
:1012B00000F0EFF8B8B1B4FA84F4640929680B7A45
:1012C000086843F3030243F303135BB252B29A423A
:1012D000C8BF0124FFF77CFB80F00103DBB224B11F
:1012E0000533D8B2F8BD0124E8E7DBB90E4F296811
:1012F0003B6806EB460003EB80000C2201F03CFA51
:101300003A680C2303FB062320465C72B2F8601394
:101310000123B3400B43A2F86033E3E70620E1E783
:101320000320DFE70420DDE7C036002010B4017899
:1013300001290ED9084B18680C234B43C41800220E
:10134000C250C4E9012200F5587010BC102200F010
:10135000A9B8002010BC7047C03600202DE9F0412C
:1013600086B050238DF81430037A102B074630D105
:101370004368DD7B6DBB0224A8466426062C14D886
:101380007A68535D03932A44517843EA0123039317
:10139000927843EA02437343CDE9033863B9684660
:1013A0008DF80040FFF7C2FF0DE0CDF80C808DF8FE
:1013B0001480CDF81080F2E703AB01A801938DF8FB
:1013C0000840FFF75DFF0134E4B2102C05F103057E
:1013D000D4D106B0BDE8F0811FB502680379116869
:1013E00049B901A88DF80430FFF7A0FF78B10320B8
:1013F00005B05DF804FB02A802928DF80C30FFF7EF
:101400003FFF042805D0052805D00028EFD0002094
:10141000EEE70220ECE70120EAE70000C90020B96E
:10142000034B0B449856C0B27047024BF9E700BF1C
:10143000C570030885700308F0B59A42069D03DB6A
:101440009DF914309A4220DD0020F0BD03EB4303E8
:1014500031F814C005EB830300264CFA06F7FF07AA
:1014600007D51F7A07F00F0E964502DCB2EB171F67
:101470000DDD0136102E03F10C03EED10134E4B280
:101480002301DBB29842E1D8DEE70024F8E701202F
:10149000DBE7884204DB9042CCBF0020012070478C
:1014A0000020704710B51409B4EB111F03464FEA32
:1014B00011100ED391420CD202B201F00F0133F899
:1014C0001240012000FA01F124EA010123F8121070
:1014D00010BD0020FCE7F0B528B100EB4105012765
:1014E0000020914200D3F0BD002435F802CB234602
:1014F00007FA04F636EA0C0608BF013304F10104CA
:1015000008BFDBB2102CF3D118440131C0B2C9B20C
:10151000E7E710B500B149B910BD31F8134020F824
:1015200013400133DCB2A242F7D8F5E70023F9E714
:1015300082B030B504880493D2B9B3F5616F15D386
:1015400049F6AF2542F21072AB4298BF4FF47A725F
:10155000944238BF14466143BDE83040C3688B42B3
:101560008CBF5B1A0023C36002B070476422EFE7B0
:10157000012C38BF0124EEE72DE9F04F8FB015465E
:10158000199F03939DF8603007930C46804603F043
:10159000C7FB6A4A0590A7F5F633303BB3FBF2F37D
:1015A000534303F5F63B0493182313FB05430BF158
:1015B000300B069300254FF0FF3A069B9C4207D163
:1015C000002D14BF50464FF0FF300FB0BDE8F08F34
:1015D000BDF96830ADF82430099919973846089755
:1015E00003F02EFB2688B8F1000F5FD1B7F5616FCD
:1015F0005AD349F6AF2242F21073974298BF4FF484
:101600007A739E4238BF1E46642E59D1DFF830915E
:10161000A060A1680CA803F035FB0D9B0093DDE9E9
:1016200008120C9B0AA803F08CFA039A0A9B0AB9C9
:10163000079A2AB122694A4502D1424A93420ED9F9
:10164000414BC4F80C909F4209D90023ADF82C30CF
:101650000B99CDF828B0584603F0F2FAA060606804
:1016600008B9C4F80C90C4F81090B8F1000F04D079
:1016700003F060FBE3680344E360D4E90332934280
:10168000059B88BFE26063601B9BE16873439942DE
:1016900004D20398E8B9B8F1000F1AD001231D4411
:1016A0002375EDB2183488E76423AAE7039B0BB9CE
:1016B000234BE360012EDFF8889038BF0126CEE788
:1016C000B6F57A7F0ABFDFF88490DFF88490A060D7
:1016D0009FE700209342207506D85B1A9A4505F1D2
:1016E000010528BF9A46EDB2B8F1000FDAD1642E99
:1016F000184AADF82C801DD049F6B023B6F57A7F94
:1017000018BF1346974281BF049A02F5A83202F52A
:10171000C0729B180A931A9B00930AAE96E80600C3
:10172000199B304603F00DFA96E8030003F088FA9F
:101730008246B7E74FF46163E4E700BF80510100E0
:1017400040771B007F5101002FEC010080A812019F
:10175000002E930230EC01000378032B14D1437860
:1017600003F00F021B098A704B7083788B80C2785C
:1017700043EA02238B800379C3F3021203F00F03C1
:10178000CA700B7005207047002070472DE9F347A1
:101790009A464379057990F907609146044690F995
:1017A00006208846D3B190F90870002D37D00F2A53
:1017B0001BD194F909200F2E27D194F90A00072D87
:1017C00002D1002F08BF012788F8002089F8000007
:1017D00028468AF8007002B0BDE8F08790F90B70D7
:1017E00090F9092090F90A60DFE7A369019394F961
:1017F0001530009394F914302169207BFFF71CFE0B
:101800000028D8D105F0FD05D5E794F91D00B042B8
:10181000D5DC94F91C30B34203DA05F0FB05304601
:10182000D2E73046CBE70000024B03FA00F0B0FBF2
:10183000F1F0704740420F004FF4FA53B3FBF0F061
:10184000704730B54FF47A750C1F6A4300FB0422D1
:1018500052001EBF00F1FF341219B2FBF0F29142A8
:1018600038BF1146039A1160820048431CBF013003
:1018700040084FF47A71121A01FB1323002BCABFE0
:1018800003F2E73393FBF1F1B3FBF1F1049B196031
:1018900030BD38B5400014460D46F0F78BFB0146CD
:1018A0002846F0F7D5FA2146F0F7D2FAEFF74CFFC9
:1018B0001EF0BAFEF0F750FA40B238BD2DE9F74FEE
:1018C000019300239C469E46048A1E01F6B2B44250
:1018D00046D906EB46054FEA4309AD0000244768A8
:1018E00037F809702741FF0729D5876807EB050AF4
:1018F0007F5927B3077837B9476927B137F8097097
:101900002741FF071BD59AF8087090F901B047F3FB
:1019100003084FFA88F8D84511DC47F303177FB264
:101920005F450CDB9AF8097007EB4708C76807EBBF
:10193000C8073F7D5FB90CF1010C5FFA8CFC0134E4
:10194000102C05F10C05CAD10133DBB2BCE70EF156
:10195000010706EB040801F80E805FFA87FEEEE748
:10196000019B82F800E083F800C003B0BDE8F08F6F
:101970002DE9FF4704464068DDE90C671D468A46AD
:10198000914603F0D7F923681B1A3B604FF000081B
:101990000123337085F80080636813B123688342A4
:1019A00024D8D4F81CC0CAF80080A3699CF800E0D1
:1019B0000393D4E9030101AB83E80300237D009383
:1019C000DCF80C10237A627A7046FFF7D5FD3346B7
:1019D00038602A46E0694946FFF770FF2B782BB143
:1019E000C7F80080002004B0BDE8F0873378002BF2
:1019F0000CBF0C200B20F6E737B590F9002090F9CA
:101A00000250954204460FD0013A52B295420BD093
:101A1000A368019394F9013000936168E0782B4644
:101A2000FFF70AFD0028EFD0104603B030BD884212
:101A3000B8BF08467047000051F82000054B984297
:101A400005D0054BC31A5842584140007047012049
:101A5000704700BF90D0030020A1070005281FB5E4
:101A60000ED80C4B53F820300093CDE901120A4BED
:101A700001220021022002F06BFE05B05DF804FB9C
:101A8000CDE90012054B01220021022002F060FE88
:101A9000F3E700BFB07103084871030867710308DA
:101AA00007B5054BCDE9000101220021022002F01B
:101AB0004FFE03B05DF804FB8371030810B51022DC
:101AC00004460021F13000F06BFE0021C4F814112F
:101AD0002046F022BDE8104000F062BE02460846F3
:101AE000102100F0A5B92DE9F0430446D0F8140107
:101AF00085B00E46154604F2011988B3C0F11008EE
:101B00009045474628BF1746BAB2484400F034FE15
:101B1000D4F814313B440F2BC4F814312DD9A84507
:101B20002BD204F1F00304F5807113F8012F187C17
:101B30008B4282EA00021A70F7D104F1F1081022F8
:101B40004146684600F018FE22466946684600F0A5
:101B5000F1F910226946404600F00EFE3E44ED1BAE
:101B600004F5807804F1F107102D09D8AAB23146A6
:101B7000484600F001FEC4F8145105B0BDE8F083FA
:101B800004F1F003711E13F8012F11F8010F434502
:101B900082EA00021A70F6D110223946684600F037
:101BA000EBFD22466946684600F0C4F910226946FA
:101BB000384600F0E1FD1036103DD5E7F0B589B0AC
:101BC0000C46102200210546684600F0E9FD224639
:101BD0006946684600F0AEF99DF90030002B6A4670
:101BE0004FF0000143DA137812F8010F01315B0066
:101BF00043EAD0130F2902F8013CF4D19DF80F30CD
:101C00005B0083F08703D4F81401DBB210288DF851
